:020000040800F2
:10000000781E0020D50000089D2B00086D220008F6
:1000100000000000000000000000000000000000E0
:1000200000000000000000000000000099880008A7
:100030000000000000000000BF5100089D8800087B
:10004000E700000800000000E7000008E7000008E3
:10005000E7000008E7000008E7000008E7000008E4
:1000600000000000551D0008E7000008E700000838
:10007000E7000008E7000008E700000800000000B3
:10008000E70000080000000000000000E700000892
:1000900000000000E7000008E7000008E700000893
:1000A000E7000008E7000008E7000008A18A000850
:1000B000918C00080000000000000000000000001B
:1000C0000348854600F04CFB00480047ADB00008EF
:1000D000781E00200448804704480047FEE7FEE7FA
:1000E000FEE7FEE7FEE7FEE7258A0008C1000008FC
:1000F00000487047D4D0000810B50446FFF7F8FF59
:100100000068005DC007C00F10BD30B505462A4627
:100110000B4610781C78521C5B1C002801D0A042B2
:10012000F7D0002C03D0002802D06D1CEFE7284642
:1001300030BD10B5044605E00B780370401C002B61
:1001400000D0491C521EF7D2204610BD421C017837
:10015000401C0029FBD1801A704710B5002200E036
:10016000521C835C8C5CA34201D1002BF8D1D8B225
:10017000E1B2401A10BD03460A780270401C491CC7
:10018000002AF9D11846704730B5054600200346CD
:1001900000E05B1C934205D2EC5CC85C201A01D1E4
:1001A000002CF6D130BD0000F7B5009C0F460026AC
:1001B0002578641C002D05D0FFF79AFF0068405D8C
:1001C000C007F5D12B2D02D02D2D18D0641E394635
:1001D0002046029A00F050F8002F04D03968A1425E
:1001E00001D1009939607105022400290BDA4042DF
:1001F000002803DD0CF0C4F90460A007FEBD012057
:1002000080020643E3E70028F8DA0CF0B9F904604D
:100210000048FEBDFFFFFF7FF0B51FB4064600207B
:1002200082B005464024019100901BE001992246CE
:100230000F46304600F0FEFA049A059B801A994159
:1002400010D310461946224600F0E4FA361A8F41C0
:100250000197224601200021009F00F0DBFA3818A8
:100260004D4100902046641E0028DFDC019B009871
:100270002946324607B0F0BDF7B582B0029C002790
:100280002078641C15460197302802D0002D15D027
:1002900015E020780127641C782804D0582802D063
:1002A000002D09D00BE0002D01D0102D07D1002723
:1002B00010252078641C02E0082500E00A250026AD
:1002C000009610E00099012769430818020C29469E
:1002D00080B2714300908E183804864201D3012009
:1002E00001902078641C294600F0C8FA0028E9DA59
:1002F0000398002805D0002F01D0641E00E0029C66
:1003000004600198002806D00CF03AF9022101603F
:10031000C81E05B0F0BD009930040843F9E700009D
:100320000FB400B589B00A460DA9009100230C99BD
:10033000002ACB60234B0693234B079301D0042361
:1003400000E00023214A0292214A089201930246CA
:100350006B46002000F031FB09B008BC04B0184720
:10036000F0B585B007460020C04301901E4600202E
:1003700015460C460091029104903B466A46314670
:1003800004A8FFF7CDFF049902466018002D05D0A0
:10039000002901D0034600E023462B6000290ED03F
:1003A000002A02DD0099814209D0001B01900094CF
:1003B0003B466A463146029404A8FFF7B1FF05B0F8
:1003C000F0BD0000110C0008310C0008FFFFFF7F9A
:1003D000F9000008F0B507460846584087B0C00F3E
:1003E000049048000E46590040084908BC1A88414C
:1003F00005D2384631461E4617460B46024658007F
:10040000400810434CD0300D039040055900400D7A
:10041000490D0590401A0290402872DA1803012114
:10042000000B09050843019004980092002805D0AC
:100430000199524200208841009201900298402187
:100440000A1A0199009800F0E5F905460C466B463A
:1004500007CB00F000FAC0197141039A0E0D00237A
:10046000D71756401A467A40164344D0049A002AB9
:100470002DD0029A012A039A15DC1205C01A914167
:1004800001263605001C7141D20F059ED20700934C
:10049000019202962A46234600F0E9FB07B0F0BD20
:1004A00038463146FAE71605224A0F46B218C01AF6
:1004B000B74101210905001C4F4100187F41114639
:1004C00018187941E20F10436D19644113E0E207F7
:1004D0006D0815436408C2071443039A01261205E8
:1004E000C01A91413605001C7141CE0740083043C7
:1004F0004908C01851412A46234600F0ABFBCDE71E
:10050000FFE7049801224000C117121A00238B4113
:1005100004983146C417381AA141EEE730B40124DB
:10052000E407634030BC55E730B40124E407614080
:1005300030BC4FE70000E0FFF0B51FB488B00B9966
:100540000998002448400999C00F490049080991B9
:10055000C0070B990090490049080B910999089828
:10056000A64608431CD00B990A98084318D009984E
:1005700001244000420D4800410D09982405000364
:10058000000B204309900B980003000B20430B90B5
:1005900050181C494018002201901446104605E0EE
:1005A000002001460DB0F0BD032801DA034600E04B
:1005B00003239C46C11A0AAE0AE05F0008ADED5B5A
:1005C0004F00F75B7D430027AA187C41491C5B1E46
:1005D0006145F2DD410004AB5A522104120C0A437A
:1005E000240C401C0828DFDB01980290009970461B
:1005F00001910090059B049A0799069800F037FB3B
:10060000D0E700000DFCFFFFF0B50C465C4085B064
:10061000E40FE40703944C00002664085900944654
:10062000490802460296224321D062460A431ED060
:100630006200570D4A000E032303550D01240246A4
:100640002C492405781B1B0B360B401823432643EB
:10065000614600901C46501AB44103D30098401CD8
:10066000009002E0921800985B41002803DA002015
:10067000014605B0F0BD0020012109050746864668
:1006800011E064461D46141BB54106D36546521B56
:10069000B341744607430C43A646CD0740084908BA
:1006A000284392185B4105460D43EAD11046184392
:1006B00013D06046194650407140084306D060464A
:1006C000101AB34106D20122002306E000220123C2
:1006D000DB0702E00122D243531000987446010563
:1006E000381C6141029C039D0019694100F0B2FA77
:1006F000BFE70000FD0300004A0009030123090BC6
:100700001B0519430A4B10B5520D9A4202DA00201C
:10071000014610BD064B34339A4203DC9A1A00F0AE
:1007200089F810BD034BD21800F074F810BD00001A
:10073000FF030000CDFBFFFF10B5002904DB0124FF
:10074000E40740428C412146002B04DB1C46012378
:10075000DB075242A341994200D1904210BD0000F4
:10076000064C0125064E05E0E36807CC2B430C3C04
:1007700098471034B442F7D3FFF7A6FC58E60008B8
:1007800078E6000870B50446002903D00020202236
:10079000012310E0002801D00020C043C046C0461D
:1007A0000DE02546D5408D4205D30D469540641B8E
:1007B0001D46954040191546521E002DF1DC21467C
:1007C00070BD000070B5002504462E46002911D0EA
:1007D000002C01DA01254442002901DA01264942B0
:1007E0002046FFF7CFFFB54200D04042002D00D099
:1007F000494270BD002C02DA0121C90702E0002C39
:1008000000DD03490846C046C046214670BD0000D1
:10081000FFFFFF7F10B5202A04DB0146203A9140FC
:10082000002010BD914020239C1A0346E340194349
:10083000904010BD10B5202A04DB0846203AD04075
:10084000002110BD0B46D340D0402024A21A914075
:100850000843194610BD10B5202A06DBCB17084601
:10086000203A1041C1170B4306E00B461341D0401C
:100870002024A21A91400843194610BD3A2800D2FC
:100880003038202302469A43412A01D31046373894
:10089000884201D30020C04370470000FFB50878AC
:1008A00089B01546FF2805D0491C2D2804D0002208
:1008B000002407E000240BE00122F9E70A235C434F
:1008C0000419491C0878FF28F8D1002A00D0644296
:1008D000002004902A7801462D2A01D02B2A0FD11E
:1008E0006D1C2D2A02D00022049209E00122FBE7B0
:1008F00000260A2233466D1C00F00BFA38187141AD
:100900002F78FF2FF4D10C9AA218069202460A43C0
:1009100004D0FF23069A9133DA4205DA00210998C0
:100920000A4606C00DB0F0BD0024B74AB54D2646B4
:10093000079200F007FA029006980391002801DA66
:10094000474200E0074639050020AF4A001C5141EC
:100950000191009012E0F80707D022462B4630465E
:100960000799FFF7E9FD0646079122462B461046F8
:100970001946FFF7E1FD04460D467F10002FEAD12E
:100980000698019B0028009A0399029806DAFFF75F
:100990003BFE3246079BFFF737FE05E0FFF7CCFD35
:1009A0003246079BFFF7C8FD049A002A02D00122B5
:1009B000D2075140099A03C2B4E7FFB591B00020B5
:1009C00009900025ED432E209E685C681F4601902B
:1009D000B9696D1C129888470090396A88470028C9
:1009E000F6D10098401C0AD00D20C0018443002E8F
:1009F00012DD00982B2809D02D280DD103E000200E
:100A0000C04315B0F0BD012080020443B9696D1CDC
:100A100012988847761E009003A9600501D52D2005
:100A200000E02B206A461073491C0CA80F9102901D
:100A30000AE0B9696D1C12988847009001204002B5
:100A400004431398761E0560002E02DD00983028BE
:100A5000EFD001990098884245D18020044308E0F6
:100A60000998401E09900120400204431399681C14
:100A70000860B9696D1C761E12988847009030286E
:100A8000EED030E00199884205D1200603D48020C1
:100A90000443761E1DE000980BF0A2FE002825D02E
:100AA000012149020C43009807AA0F9903323038FC
:100AB000761E914208D208700F98401C0F902006B5
:100AC00007D50998401E03E0200602D40998401C6F
:100AD0000990A00502D51399681C0860B9696D1CBE
:100AE000129888470090002ECCDC59E0002E57DD8C
:100AF0000098652801D0452852D1A00550D5032083
:100B000000028443B9696D1C761E129888470090D4
:100B1000002E0CDD2B2804D02D2808D1FF20013019
:100B20000443B9696D1C12988847761E0090E00551
:100B300001D52D2100E02B21029801700298401C64
:100B40000290019025E00120400204430EA9029882
:100B50000131761E88420ED2009802993038000684
:100B6000000E087003D10299019881420AD90298B7
:100B7000401C029006E0E00501D5244801E023482E
:100B800040420990B9696D1C1298884700901398EB
:100B90000560002E04DD00980BF022FE0028D2D163
:100BA000F969129888470F99FF200870029903AAE3
:100BB000087000200A900B900CA90AA8099BFFF767
:100BC0006DFEA00502D40120C0431AE72420044290
:100BD00009D0E00713D138680B9A0A99031D3B60CE
:100BE000006806C00BE00B990A9800F0B9F80146BE
:100BF000E00704D13868021D3A60006801602846A9
:100C0000FFE60000000014400000F03FF1D8FFFFB5
:100C10004268002A08D001680B78491C002B03D0D9
:100C2000521E06C0184670470121C160881E7047D9
:100C30004268002A0BD0C3680168002B07D1836883
:100C40008B4204D0491E521C06C000207047002071
:100C5000C043704710B5002B08DA0024401C6141E6
:100C600092185B411A4301D14008400010BDF0B515
:100C70001FB482B005460C0003D008460BF068FC98
:100C800002E00BF065FC2030024600902146284629
:100C9000FFF7C0FD049B059A04460F461843114315
:100CA000084314D0184610431BD0009840210A1A5C
:100CB00018460599FFF7BEFD05460E46009A0599B0
:100CC0000498FFF7A7FD084305D0012004E0204663
:100CD000394607B0F0BD0020C11705430E432C4331
:100CE000374300990E986305401A7905E40A0022FB
:100CF0000C43FD0A0A3002D500200146E9E7010550
:100D0000101969410C9C0D9D00196941FFF7A2FF64
:100D1000DFE730B5434351435C18010C130C0D461B
:100D20005D432C1980B292B20546554351430A0CDB
:100D300009044D1962415843010C00044019514106
:100D400030BD00000EB5054A029200220092134603
:100D50000192FFF78CFF03B000BD000033040000D8
:100D6000CB0FDB07490010B5490802460A4307D0FC
:100D70000A0D07240903E401090B121B002A01DCF8
:100D8000002010BDC900440F0C43C100E018D2057B
:100D9000801800F001F810BD002904DA401C490059
:100DA00001D140084000704770B40024050C05D103
:100DB0001024000402D1002921D01124050E01D1F4
:100DC00000020834050F01D10001241D850F01D157
:100DD0008000A41C002801DB4000641C002908D00E
:100DE00020252E1B0D46F540A14000D001212943AE
:100DF000084301061B1B000ADB1D02D5002070BC46
:100E00007047DB05181880180029F8DA401C4900E3
:100E1000F5D170BC400840007047F8B50024254665
:100E2000002904DA0E46012400214042B141002B82
:100E300004DA1E46002352420125B341FFF7ECF9C4
:100E40008C4617461E46AC4203D0002540428D41D9
:100E5000AC46002C02D0002657429E4161463A46DD
:100E6000334601B0F0BD10B5431A934209D283183E
:100E7000881803E0401E01785B1E1970521EF9D2DB
:100E800010BD03460B439B0703D009E008C9121F9E
:100E900008C0042AFAD203E00B780370401C491CF6
:100EA000521EF9D210BDD2B201E00270401C491EA0
:100EB000FBD270470022F6E710B513460A460446F7
:100EC0001946FFF7F0FF204610BDF8B502464A402C
:100ED000D40F42004B0052085B089A4202D20246ED
:100EE000084611464A0023D0C30D4A00DDB2120E57
:100EF000AD1A202D35DA49020126490AF6058A196C
:100F0000002C00D0524220214F1B1146B9402A41EB
:100F10001018C20D9A4221D0002C17D0012D08DCE8
:100F2000DA05801AD20F8019D207DBB2FFF73CFF37
:100F3000F8BDDA05801A012340001B06C01880188E
:100F40005A428018CA0F1043490007E04908C207F7
:100F50001143DA05801A801940088018FFF71CFF3A
:100F6000F8BD61000122511A001BF7E70122D207E8
:100F70005140AAE70122D2075040A6E7024670B5C9
:100F80004A40D30FDB0740002DD04A002AD0010E83
:100F9000140E000212020919400A520A8418E501CF
:100FA00004465443000A120A2E045043A41942195D
:100FB000200CC543AA18120C0125AD03521C52196E
:100FC00012047F39240400D0521C104301D4400085
:100FD000491EC2B20C06C0092018401C4008802AD5
:100FE00002D003E0002070BD40084000002900DA74
:100FF0000020184370BD70B502464A40D50F40002E
:101000004A00ED0740085208002814D0002A12D0E8
:10101000C40DD30D41020120C0055202490A520AF3
:10102000E41A091812187D34914201D3641C00E0BF
:101030004900002C01DA002070BD0023914201D349
:10104000891A0343400849000028F7D100290AD033
:10105000914202D10121C90705E0914201D201214B
:1010600001E00121C943E005C0184019FFF794FED3
:1010700070BD0122D207002800DB101A002900DB16
:10108000511A814201D2012070470020704701228D
:10109000D207002800DB101A002900DB511A814218
:1010A00001D901207047002070470122D207002893
:1010B00000DB101A002900DB511A814201D1012006
:1010C000704700207047C217C10F504010B540183C
:1010D000CA0796230021FFF767FE10BD10B5002256
:1010E00096231146FFF760FE10BD0A4670B5C9177A
:1010F000D30F4A4048400025C11814466C41DA0716
:1011000096232046002C03D0B623FFF74DFE70BD7A
:1011100008460021F9E700000EB5C217C10F504084
:10112000CA0740180021054B0293019200910A461C
:101130000B46FFF79CFD03B000BD00003304000028
:101140000EB505490291002100910A460B46019116
:10115000FFF78DFD03B000BD330400003EB5CA1794
:10116000CB0F002450405140C0186141DA07054BB5
:1011700002930192009422462346FFF778FD03B0C4
:1011800030BD000033040000C20F410040020123C3
:10119000400ADB05D207090EC0187F2901DA0020BA
:1011A0007047962903DC9623591AC84001E0963906
:1011B0008840002AF4D0404270474100400201229A
:1011C000400AD205090E80187F2901DA00207047F5
:1011D000962903DC9622511AC840704796398840F8
:1011E0007047000070B5CD0F4A0009030123090BB9
:1011F0001B0519430B4BED070024520D9A4201DAEF
:10120000002070BD074B34339A4203DC9A1AFFF773
:1012100011FB02E00449511888402C43F1D04042B0
:1012200070BD0000FF030000CDFBFFFFC20FD2071F
:10123000400040080BD0C10D0723DB01C918400254
:101240000905400A1143C2084007114370470020B6
:1012500001467047FEB51D4613460C4607460CA2D4
:101260000C4E08461946B04706460B4938460AF068
:10127000A3FA4119684609F09FFD0246204631460F
:10128000044DA8470146A44A2046A847FEBDC046D3
:1012900042000000E5C1000808E30008F0B58FB087
:1012A0000A9305920991814907900AF085FA002175
:1012B00008910B910490401C0690099D28467C499A
:1012C0000AF07AFA07460E460CA8394609F074FD72
:1012D00004467A1C089846412846754933460AF068
:1012E00087FB284621460AF0ABFA00280FD00746B4
:1012F000069AD317079C20466C490AF079FB0BAA83
:10130000204639460A9BFFF7C9FF0A90D6E769498C
:10131000694C099F3846A047029068493846A04763
:10132000009067493846A047019066493846A04773
:10133000064665493846A047089064493846A047A4
:10134000054663493846A047039062493846A0479E
:10135000069061493846A0470990012001020BA878
:1013600009F024FB0446009800280CD05BA120461D
:10137000049F3A4609F096F80BA80A9922460AF00B
:1013800031FF0A9000E0049F002E0CD056A12046A9
:101390003A46334609F086F80BA80A9922460AF025
:1013A00021FF064600E00A9E019B002B0AD051A1B6
:1013B00020463A4609F076F80BA8314622460AF054
:1013C00011FF0646029B002B0AD04DA120463A464B
:1013D00009F068F80BA8314622460AF003FF0646DA
:1013E000002D19D049A120463A4609F05BF849483A
:1013F000214609F09AFA294609F0B2FA464909F05D
:10140000AFFA054602460C320BA831460AF0EAFE56
:101410000646284609F04CF9039B002B0AD03FA151
:1014200020463A4609F03EF80BA8314622460AF01B
:10143000D9FE0646069B002B0AD03BA120463A4621
:1014400009F030F80BA8314622460AF0CBFE0646DA
:10145000089B002B0AD037A120463A4609F022F813
:101460000BA8314622460AF0BDFE0646099B002B1A
:101470000AD033A120463A4609F014F80BA83146A9
:1014800022460AF0AFFE06467A1ED3170749079890
:101490000AF0AEFA059831460AF0C8FE04460BA8D9
:1014A00008F0C1FD20460FB0F0BDC04614E30008AF
:1014B0008BE300082FE200086FB8000805E500087C
:1014C000F4E30008C0E20008AAE40008F3E2000820
:1014D00065E4000892E30008FEE400082564204C5F
:1014E0005354200A00000000256420524546202560
:1014F000730A00002564204F50542025730A000011
:1015000025642052554E2025730A0000256420537F
:1015100054522000D8D00008BBDD000825642042CA
:1015200059542025730A00002564204E554D20256E
:10153000730A00002564204F55542025730A0000CB
:10154000256420494D502025730A0000F0B599B05C
:101550000F46069000250A950AA828220AF01DFFCA
:1015600001460D950DAE304601F09EF8FC4902F0A3
:10157000E9FC0446304608F056FD002C4FD00AAE78
:10158000F84C304621460AF051FE0890304621467C
:101590000AF04CFE07900DAC204602F05CFC2046A1
:1015A000394602F0C5FC204602F03AFC2C462E4695
:1015B0000DA8808884422CD2099434460DAE304662
:1015C00002F05CFC129F3846E5490AF07EFD0125D9
:1015D000002802D0307C032814D0E0B201280BD0C0
:1015E00026460028099C0FD10AA808993A460AF015
:1015F000F9FD0890002607E00AA807993A460AF084
:10160000F1FD07902E46099C179809F09BFC641C7D
:10161000CEE70DA802F014FC079C089DB3E0D14C66
:10162000D14D20462146A847079020462146A8478D
:10163000089020462146A847099000250C950BA844
:1016400005800CA8394601F02FF80446C74902F07E
:1016500079FC002802D00BA82B250570C449204630
:1016600002F070FC002802D00BA82D250570C1499E
:10167000204602F067FC002802D00BA82A2505703E
:10168000BD49204602F05EFC0028059703D00BA858
:101690002F21017002E0002D00D16CE20DAC20463C
:1016A00002F0D9FB2046394602F042FC204602F007
:1016B000B7FB002635460DA88088854230D20DA89C
:1016C00002F0DCFB129C2046AA490AF0FEFC01272E
:1016D000002818D12046A8490AF0F7FC002812D1AA
:1016E0002046A2490AF0F1FC00280CD12046A0496E
:1016F0000AF0EBFC002806D1002E0AD008982146FB
:1017000009F02EF908903E46179809F01BFC6D1C55
:10171000D1E70798214609F023F907900026F3E75F
:101720000DA802F08DFB079C0C34944D09982146BE
:10173000A8470BA9A8479249A84708990C31A84780
:101740009049A847054609900C3500260CA808F0DA
:101750006AFC002D04D00AA829460AF067FD05900E
:10176000002C05D00AA821460AF060FD054600E0DD
:101770000025854C0898A0470798A0470998A047DE
:10178000002E059C04D1814906982A460AF05AF990
:1017900000270C970CAD7A4A7A4B284605942146CF
:1017A00008F0C0FE01467A4A7A4B284608F0BAFE95
:1017B00005460DAE304602F04EFB3046294602F09B
:1017C000B7FB304602F02CFB734E07970397019747
:1017D0000297049709973C4608973D460DA88088D4
:1017E000854242D20DA802F049FB129F384631468D
:1017F0000AF06BFC002801D0012424E0384664493B
:101800000AF063FC002802D0012009901BE00DA81B
:10181000007C032802D10120089014E00DA9097F63
:10182000042902D1012007900DE0012809D00528E4
:1018300009D138780121222801D0272808D1039125
:1018400001E001200490179809F07CFB6D1CC5E7AE
:101850007978272901D0222904D1622802D10120D8
:101860000190F0E701200290EDE7002C35D00DA8A3
:1018700002F0E6FA0CA808F0D6FB059D2846FEF714
:1018800065FC01460AA809F091F804462846FEF7CF
:101890005DFC6A1E0021012808DB135C202B05D0AB
:1018A0006354135C401E491C202BF4D1C80F081848
:1018B00040104A1E0023834206DAE55CA65CE6542B
:1018C000A554521E5B1CF6E7002060543349069D68
:1018D000284622460AF0B6F8B9E10898002800D157
:1018E0003EE10DA802F0ACFA0CA808F09CFB059EA6
:1018F0003046FEF72BFC04460AA8214609F056F8AC
:101900000746002001460246A2420DDAB35C292BAD
:1019100000D1401E050602D17B54B35C491C282B24
:1019200000D1401C521CEFE70020785409900C9025
:101930000CA80897394600F0B7FE0746F74D1E265B
:10194000002E2DD03846294602F0FCFA002804D09B
:101950000CA829460AF06AFC0990761E0935EFE7C3
:1019600061E10008D8D000082BA9000857E1000861
:101970005AE1000854E100085DE1000861A900088F
:10198000A4DE000823E00008B1A60008AAE40008CD
:10199000E9E10008EBE1000895DE0008FEE400083C
:1019A000DF4909980AF091FB002805D1DD49099823
:1019B0000AF08BFB002833D00DAD284602F04BFA1D
:1019C0002846089902F0B4FA284602F029FA0026BF
:1019D000D34FD44C0DA8808886421ED20DA802F0A9
:1019E0004DFA129D284639460AF06FFB002804D0B4
:1019F0000CA839460AF01AFC0990284621460AF03C
:101A000064FB002804D00CA821460AF00FFC0990C2
:101A1000179809F097FA761CDCE70DA802F010FA87
:101A20000AAD284609990AF001FC04460CA808F002
:101A3000FAFABD490698089422460AF003F82846A7
:101A400005990AF0F3FB0546B34C2046214608F001
:101A50006CFF09902046214608F067FF06460DAC52
:101A6000204602F0F8F920460795294602F060FA70
:101A7000204602F0D5F900252F460DA88088854222
:101A800013D20DAC204602F0F9F9207A002807D1D4
:101A9000129908980AF019FB002801D00DA887793F
:101AA000179809F04FFA6D1CE7E70DAC204602F0DD
:101AB000C7F9204602F0CFF92046079902F038FA1C
:101AC000204602F0ADF900250DA88088854217D286
:101AD0000DAC204602F0D2F9E488BC4204D212993F
:101AE000304608F03DFF0646BC4204D912990998D9
:101AF00008F036FF0990179809F024FA6D1CE3E707
:101B00000DA802F09DF9354631460C310AA80AF0BD
:101B10008DFB0890099E34460C342046FEF716FBD8
:101B2000421C079F38462146FFF79DF9284608F0DA
:101B3000BFFD304608F0BCFD069D28460AF0B8F906
:101B400028460AF093F90899FFF700FD28460AF0A5
:101B5000AFF928460AF08AF93946FFF7F7FC76E034
:101B600009980028059E0AD00DA802F069F90CA872
:101B700008F059FA6AE0002501262C46E6E50798A8
:101B800000286AD00DA802F05BF90CA808F04BFA07
:101B90000AAD28242846314622460AF0FEFB0246BA
:101BA0006249069809F04EFF29232846314622460D
:101BB0000AF051FB01465E4A28460AF013FB07462D
:101BC0005548014608F0B1FE06460DAC204602F02D
:101BD00042F92046394602F0ABF9204602F020F9DE
:101BE00000250DA8808885422AD20DAC204602F03F
:101BF00045F9207A129F002804D03046394608F073
:101C0000AFFE17E038464A490AF05FFA0028F4D0E0
:101C1000069C20460AF04CF920460AF027F9314686
:101C20000C31FFF793FC304608F042FD3A4801467C
:101C300008F07BFE0646179809F084F96D1CD0E782
:101C40000DA802F0FDF8304608F032FD069D0AA806
:101C500008F0E9F9284619B0F0BD0398002827D00C
:101C60000DA802F0EDF80CA808F0DDF90AA831463D
:101C70000AF0DCFA0546441C2046FEF767FA00210C
:101C800029545C2120460AF049FA00280DD00AADFB
:101C900028A229A3284621460AF0AAFB014627A22A
:101CA00027A328460AF0A4FB0446069D25490FE613
:101CB0000198002815D00DA802F0C2F80CA808F071
:101CC000B2F9711C0AAC272220460AF004FB014637
:101CD000222220460AF0FFFA02461B49069D2846AA
:101CE000F8E50298002807D00DA802F0A9F80CA882
:101CF00008F099F915490AE00498002800D133E763
:101D00000DA802F09DF80CA808F08DF91049069D69
:101D100028463246DEE5C046D8D00008E9D800089B
:101D200027E000082BE00008F4E300082FE2000899
:101D300029E000085C220000220000005C2700006F
:101D400027000000F3E2000865E4000892E30008C1
:101D5000C0E20008F8B52848016C1C230B4004279A
:101D60003C469C4025490A1F1668026815683442A3
:101D700001D069071DD402249C40344201D0A90738
:101D800023D4DE40310736D5290734D52421002459
:101D9000445411680E24A143116001210A469A405F
:101DA000164C236813432360C16325228154416B81
:101DB0001DE01168890602D41168B94311600F4A09
:101DC000116821431160016B11E01168890606D486
:101DD00011680A23994311602521012242542421CC
:101DE00000224254054A116821431160C16A00294A
:101DF00001D001488847F8BDB80000200400024027
:101E0000B0B57D20C2009F48C16B8B180D490C688E
:101E1000E40304D5C46B9C42F9D30320B0BD0B6826
:101E2000094C651C0D60234201D00120B0BDC36B7D
:101E30009A180B685B0303D5C36B9342F9D3ECE7A5
:101E40000020B0BD10200240FA8300001CB50446FB
:101E500029490AF077F9002803D0154801680122C2
:101E60001CE0264920460AF06DF9002803D01048EE
:101E70000168022212E0224920460AF063F9002894
:101E800003D00B480168042208E01E4920460AF0EE
:101E900059F900280AD00648016808221143016058
:101EA000006810400190019800201CBD01201CBD5D
:101EB0003410024010B504460F490AF043F90028D7
:101EC00002D00520000710BD0C4920460AF03AF95F
:101ED000002801D0CC4810BD094920460AF032F94B
:101EE000002801D0C94810BD064920460AF02AF949
:101EF000002800D0C04810BD81E1000888E100083A
:101F00008BE100088EE1000870B5054601F0ACF8E1
:101F10000446A91C0AF08AF9054643490AF0D5F897
:101F2000002801D0012579E0404928460AF0CDF883
:101F3000002801D0022571E03D4928460AF0C5F885
:101F4000002801D0042569E03A4928460AF0BDF886
:101F5000002801D0082561E0374928460AF0B5F885
:101F6000002801D0102559E0344928460AF0ADF880
:101F7000002801D0202551E0314928460AF0A5F873
:101F8000002801D0402549E02E4928460AF09DF856
:101F9000002801D0802541E02B4928460AF095F819
:101FA0000126002801D0350238E0284928460AF0E9
:101FB0008CF8002801D0750230E0254928460AF047
:101FC00084F8002801D0B50228E0224928460AF00A
:101FD0007CF8002801D0F50220E01F4928460AF0CD
:101FE00074F8002801D0350318E01C4928460AF08F
:101FF0006CF8002801D0750310E0194928460AF052
:1020000064F8002801D0B50308E0164928460AF014
:102010005CF8002801D1054600E0134D204608F089
:1020200091FFA8B270BDC0461FE100082FE1000873
:1020300035E1000838E100083FE1000842E100080E
:1020400046E100084AE100084EE1000852E10008BC
:1020500012E1000823E1000831E1000837E100083F
:102060003AE1000841E100080080FFFF401C01D375
:102070000020C0430349CA6BCB6B9B1A8342FBD33E
:102080007047C04618000020F0B589B001905A4A48
:10209000904201D0052000E0032000900023079328
:1020A0001C4618460D682A46C24000D1A1E0012610
:1020B0000696089086403540039500D191E004943F
:1020C0004A68122A05935CD8069F97404D480742FC
:1020D00057D003279F4008461D46019CA368BB4379
:1020E000C968A9401943A1601109089B9940636818
:1020F000B3430B4363600146FF43E06838400E463C
:102100008B680295AB400343E36010211143122911
:102110000FD11C21079801400F228A400898C3085C
:102120009B00E318186A904332698A4002431A629E
:1021300072683146314D20683840032713463B40D2
:10214000029EB34003432360D000059B049C48D506
:10215000182222400F209040089BBB43EE18376E98
:102160008743603605200007019B834210D0264834
:10217000834210D0254883420098214B0DD1022084
:102180000BE003269E40F74308984500019CB4E706
:1021900000201B4B01E01A4B0698904038433060FA
:1021A0001C684A68D00302D5039E344301E0039EB5
:1021B000B4431C605C68900301D5344300E0B44331
:1021C0005C602C68D00201D5344300E0B4432C603D
:1021D0006C68900201D5344300E0B4436C60059B09
:1021E000049C9B1C0798001D079008340898401C0D
:1021F00058E709B0F0BDC046000C0050001802407E
:10220000801802400600060000040050000800503C
:10221000F8B50446104D68687D21C900FEF7B2FA92
:10222000421E0120110E16D10C490D4E72600D4A4E
:1022300013680B400327BF07DB1913600023B3604B
:1022400007273760032C06D810680840A1074018FC
:1022500010602C601846F8BD10000020FFFFFF0042
:1022600010E000E020ED00E007F0ECFC01A00AF037
:10227000A5FEFEE75B6572726F725D3A206861725F
:1022800064206661756C742C20706C6561736520C8
:10229000726573657420746865206465766963652A
:1022A0002E0D0000F0B587B00593154602920491FB
:1022B000044603902A2027498847A01C06AC60707A
:1022C000000A2070681E80B2801CE070000AA070B6
:1022D000214E022535603148202101910160042101
:1022E00000911E4A204690472B201A49884705989E
:1022F000401E80B2401CE070000AA0700498401C90
:102300006070000A20703560019F244807602046F5
:102310002C460099114DA8472C200E49884734605F
:102320001E48076005980499401A0399029A511AA9
:10233000414349000C98A8470948416D25310A7866
:10234000012AFCD15D22825C012AF8D1103E346062
:1023500007B0F0BD6523000828040050D9770008B5
:1023600014010020B0B50C4C022525610349202240
:102370000A6005F00FFB2560B0BDC0462800005084
:10238000B0B5054C02252561044920220A6005F0FC
:1023900001FB2560B0BDC046180400501800005075
:1023A000B0B5044618A109F090FE194D002828D1B7
:1023B00018A1204609F089FE002802D01F2005023E
:1023C0001FE016A1204609F080FE002801D0F82564
:1023D00017E013A1204609F078FE002802D0124D24
:1023E000F8350EE012A1204609F06FFE002801D05A
:1023F000002506E010A1204609F067FE002800D065
:102400000A4DA8B2B0BDC046776869746500000087
:10241000FFFF0000626C75650000000072656400DB
:1024200079656C6C6F77000007E0FFFF07E0000044
:10243000626C61636B000000677265656E0000008E
:1024400081B005490A6802430A60096801400091A9
:10245000009801B07047C04640100240FCB5002211
:1024600001910C682346D34048D0012393401C407F
:1024700042D04E68731E022B0092234612D2634351
:1024800001998F685F4303255D438268AA433A43FD
:1024900082600199CA6862434768A743174347604F
:1024A000019902E0634303255D43ED430A695A4302
:1024B000C7682F401743C7600199022E16D1260A1C
:1024C00001D0242200E020224F698458002E1146BA
:1024D00002D07643764301E01E465E430F227243EC
:1024E000944377432743475001994E6873430268EA
:1024F0002A401A430260009A521CB2E7FCBD000059
:1025000081B005490A6802430A60096801400091E8
:10251000009801B07047C0463410024070B50446C0
:102520000068C00700D08FE00D4620684749014091
:10253000A86808432969014368690843E9690143B8
:1025400021600320010362688A43E96811436160E6
:102550000102A2688A43A9691143A1603C498C42E7
:1025600013D03C498C4269D13B4EF16C01400004D0
:1025700008183C4988423AD03B4988423DD03B4903
:10258000884240D104F0A2FF13E004F09FFF3249DB
:102590000A680968890A1C230B403049C9581F235F
:1025A000194092093C2616402D4A92591A40D040B3
:1025B000C840002842D06E68002E3FD029680B2901
:1025C0003CD889002BA25158FEF7DCF80121C90341
:1025D000EA698A422BD17108400040183146FEF763
:1025E000D1F8304901400007400F401825E0012094
:1025F000C103706D80030840DBE7083E306840058A
:102600001CD51B48D7E704F061FF31683268920A95
:102610001C231340114AD2581F231A4089093C2613
:102620000E400F4989591940C840D040C1E7710890
:1026300040183146FEF7A6F880B2E060E06A0F214C
:10264000884329880143E16270BDC046F369FFEF0A
:10265000004400400038014008100240B4D800088F
:10266000CCD40008030003000200030001000300B3
:102670000024F4000100000002000000040000003B
:1026800006000000080000000A0000000C00000026
:10269000100000002000000040000000800000004A
:1026A00000010000F0FF0000F0B591B00F4600906F
:1026B0008A48014608F039F909903846FDF746FD89
:1026C00004460025E8431090661E0D950295069776
:1026D00007940196A54200DBE0E10022012D10469F
:1026E00002DBE819401E00780C90795D0E91691CA0
:1026F000A142134600DA7B5C0893AB1CA3420B9209
:1027000002DA2046FE5C0B9605930A91E91CA14271
:10271000104600DA785C2B1DA342164600DAFE5CF8
:10272000039604916E1DA642134600DABB5DA91DF7
:10273000A14200DA7A5C109C671C2F4600D0274625
:1027400010970D9902290CD0012912D00029079C5D
:102750000E992ED1272921D10C995C291ED0012058
:1027600024E002210D910E99222907D0069F079C93
:1027700092E101210D910E992729F7D10C985C283F
:10278000069F079C00D187E110AB099839460A9A49
:1027900000F0A4F9099000200D907DE10E99222906
:1027A00007D10C995C290E9903D002200D90069F49
:1027B00072E10C9028291CD110AB0998069F39466C
:1027C0002A4600F08BF90FAA002111800E99117092
:1027D000042100F0BFF90E990990282902D102982E
:1027E000401C0290292900D056E10298401E029018
:1027F00052E1084620381E284AD8800001A1085816
:102800000E9987463F290008832800087F2A000880
:102810007F2A00087F2A00088328000883280008F0
:102820007F2A00087F2A0008812800081129000853
:102830008328000881280008832800087F2A0008D0
:10284000112900087F2A00087F2A00087F2A000833
:102850007F2A00087F2A00087F2A00087F2A0008B4
:102860007F2A00087F2A00087F2A000881280008A4
:102870007F2A00085D290008832800084B290008EA
:102880009AE72F29069F089A6CD12F2A76D069E003
:1028900008465B3806280DD9692900D180E06E29E9
:1028A00000D199E06F2900D1ADE07C29E9D07E29E3
:1028B000E7D0E4E0800002A108580E998746C046A0
:1028C000E32800087F2A0008E3280008E128000820
:1028D0007F2A00087F2A0008E5280008D8D00008D1
:1028E000CFE769E708986E280B9900D0AEE064291D
:1028F00000D0ABE00C9A202A00D0A7E010AB0998DA
:10290000069F39462A4600F0E9F80321704A75E02F
:102910000898814220D10B983D281DD13D2000040C
:102920000F900FAC6170217010AB0998069F39466B
:102930002A4600F0D3F803212246079C93E0BD42CB
:1029400000D095E00A98109099E0089A3D2A069FD9
:1029500014D03E2A12D068E02A2992D1089A9142D6
:10296000069F0BD0084621381C285CD801218140E5
:10297000584801420E9956D03D2A56D10FAE72707A
:1029800031700020B07010AB099839462A4600F02B
:10299000A5F80321324600F0DDF809900A9D7BE09E
:1029A00008986D286BD10B98702868D10C986F2807
:1029B00065D10398722862D1742B60D1202A5ED130
:1029C00010AB0998069F39462A4600F087F8032184
:1029D0003C4A00F0BFF85DE008986F284FD10B9893
:1029E00074284CD10C98202849D110AB0998069F27
:1029F00039462A4600F072F80321374A00F0AAF857
:102A00000990049D48E00898722838D10B98202836
:102A100035D110AB0998069F39462A4600F05EF87A
:102A20000321294A1FE02529A6D00FAC00202080D1
:102A3000217010AB099839462A4600F04FF803215F
:102A40002246079C00F086F8099025E07328069F2F
:102A500015D1202913D110AB099839462A4600F028
:102A60003DF80321194A00F075F80990059D13E01F
:102A700010AB099806992A4600F030F80990019E9B
:102A8000B54200D093E610AB0998069F394622461E
:102A900000F024F8099035466D1C1BE602980006EC
:102AA00002D00024099D06E0099D29460C310098BA
:102AB00009F0BCFB0446284607F0FAFD204611B099
:102AC000F0BDC04695DE00087EDE000883DE00080B
:102AD00063DE0008015600188FDE0008FEB51C46B4
:102AE00017460E460546002202921868411C29D05E
:102AF000B84227D00192391A02A807F057FF22687E
:102B0000B1180646BA1AFEF7AEF933780521222B22
:102B100012D0272B10D01A46303A0A2A0CD3622B37
:102B200009D173780521222B0A4600D00122272BD8
:102B300002D0114600E001212846324600F00AF892
:102B40000546019AD043206002A807F06CFA284697
:102B5000FEBD00007CB516460446002001906A4682
:102B600051701F211170907021460C3101AD284623
:102B700009F038FB01462846324609F033FB01468E
:102B8000054807F0D2FE0646204607F091FD28468C
:102B900007F049FA30467CBDD8D00008FEE780B582
:102BA00000F020F880BD000010B500F06BF904467D
:102BB00005A1084A08F081FE07A1094A204608F04D
:102BC0007CFE204610BDC04650696B615374644C56
:102BD000696200001D2D00086D616368696E650003
:102BE0009530000810B5042008F0E6FF044600F018
:102BF0003BFA2060204610BDB0B5FFF7F3FF044656
:102C000014A1174A174DA84717A11D4A2046A847E7
:102C10001C491D4A2046A8471CA1204A2046A84717
:102C20001F49204A2046A8471FA1274A2046A847F7
:102C300026A12A4A2046A84729A12D4A2046A8476E
:102C40002CA12F4A2046A8472EA1334A2046A84748
:102C50002046B0BD5F5F64656C5F5F28290000009F
:102C6000995800085BAD00085F5F6765745F5F2877
:102C70005F5F6B65793A616E79292D3E616E7900EF
:102C8000A9580008A6DE0008D55800085F5F6974DF
:102C900065725F5F28292D3E616E7900F558000846
:102CA00014E500081D5900085F5F7365745F5F28B5
:102CB0005F5F6B65793A616E792C5F5F76616C3A24
:102CC000616E7929000000005D590008617070652F
:102CD0006E64286172673A616E7929009D59000817
:102CE00067657428693A696E74292D3E616E7900B2
:102CF000D55900086C656E28292D3E696E74000058
:102D0000F559000873657428693A696E742C61720C
:102D1000673A616E792900008D5A0008B0B5FFF757
:102D200061FF04460AA10F4A0F4DA8470FA1134A9D
:102D30002046A84712A1164A2046A84715A11A4ABC
:102D40002046A84719A11D4A2046A8472046B0BDE5
:102D50004D656D436865636B657228292D3E616E14
:102D600079000000AD6400084DAD000850696B614A
:102D70004F626A28292D3E616E7900006165000866
:102D800052616E67654F626A28292D3E616E790037
:102D900079650008537472696E674F626A28292D3D
:102DA0003E616E7900000000F96500085379734FA9
:102DB000626A28292D3E616E7900000025660008B0
:102DC000B0B5FFF70FFF04460AA10E4A0E4DA84703
:102DD0000EA1124A2046A84711A1134A2046A8472F
:102DE00012A1144A2046A84713A1164A2046A84714
:102DF0002046B0BD6765744D617828292D3E666C0C
:102E00006F617400C56400085BAD00086765744EAF
:102E10006F7728292D3E666C6F617400E9640008A5
:102E20006D617828290000000D6500086E6F772815
:102E3000290000002D65000872657365744D617886
:102E4000282900005565000880B5FFF7CBFE80BD3E
:102E500010B5FFF7C7FE04460849024A07F07DFF98
:102E6000204610BD9165000810B5FFF7BBFE044673
:102E70000249034A07F071FF204610BD14E500081F
:102E800011660008B0B5FFF7ADFE04462A492B4A8B
:102E90002B4DA8472B492C4A2046A8472B492C4AA2
:102EA0002046A8472B492C4A2046A8472B492C4AA4
:102EB0002046A8472B492C4A2046A8472BA12E4A3A
:102EC0002046A8472D492E4A2046A8472D492E4A7C
:102ED0002046A8472D492E4A2046A8472D492E4A6C
:102EE0002046A8472D492E4A2046A8472D492E4A5C
:102EF0002046A8472DA1304A2046A8472FA1344A92
:102F00002046A84733A1364A2046A84735A13A4A69
:102F10002046A84739A1404A2046A8473FA1444A35
:102F20002046A84743A1484A2046A84747A14B4A04
:102F30002046A8472046B0BD6AE500082D67000876
:102F40005BAD0008B0DF00085567000824E5000805
:102F50004D68000855E40008A168000805E4000871
:102F60003569000820E40008796A00086469637420
:102F700028292D3E616E7900CD6A000894E400088E
:102F8000156B000832E40008A16B0008EDE40008AE
:102F90000D6C0008DBE40008416C000857E50008F0
:102FA000116D0008C9E40008DD6D00086C697374D8
:102FB00028292D3E616E79005D6E00086F726428CD
:102FC00076616C3A737472292D3E696E740000004C
:102FD000A56E00087072696E74282A76616C2900EB
:102FE000BD6E00087072696E744E6F456E6428760F
:102FF000616C3A616E792900E56F000872616E6755
:10300000652861313A696E742C61323A696E7429AF
:103010002D3E616E790000004970000872656D6F89
:10302000766528617267506174683A73747229001A
:103030009D700008737472286172673A616E792915
:103040002D3E737472000000F97000087479706589
:10305000286172673A616E79290000008971000861
:1030600080B5FFF7BFFD80BD80B5042008F0A4FD4A
:103070000021016080BD000010B5FFF7F5FF044698
:1030800003490022134607F0F9FD204610BDC04653
:10309000D6E30008B0B5FFF7A5FD044614A1174A12
:1030A000174DA84717A11A4A2046A84719A11C4A3C
:1030B0002046A8471BA11E4A2046A8471DA1204A1A
:1030C0002046A8471FA1234A2046A84722A1254AF7
:1030D0002046A84724A1274A2046A84726A1294AD6
:1030E0002046A84728A12B4A2046A8472046B0BD25
:1030F00041444328292D3E616E790000BDAF000890
:103100004DAD00084750494F28292D3E616E79008A
:10311000D5AF00084B455928292D3E616E79000036
:10312000EDAF00084C434428292D3E616E79000024
:1031300005B0000850574D28292D3E616E790000DA
:103140001DB00008506F696E7428292D3E616E799C
:103150000000000035B0000852474228292D3E618A
:103160006E7900004DB000085461736B28292D3E24
:10317000616E790065B0000854696D6528292D3E9F
:10318000616E79007DB000085541525428292D3ECA
:10319000616E790095B00008F8B5FFF723FD04468D
:1031A0001749184A184FB8471849194A2046B847CE
:1031B0001849194A2046B8471849194A2046B847BD
:1031C0001849194A2046B847184D194A2046294639
:1031D000B847184E184A20463146B84717A11B4A2F
:1031E0002046B8471A491B4A2046B8471A4A204683
:1031F0002946B847194A20463146B8472046F8BD07
:10320000A6DE0008B95A00085BAD0008FEDE000823
:10321000C15A0008E3DE0008CD5A000862DF00084A
:10322000E95A0008ECDE0008F15A0008D2DE000876
:10323000015B0008B1DE0008115B00087265616483
:1032400028292D3E666C6F6174000000215B000828
:10325000A0DF0008455B0008BD7A0008257C000857
:10326000F8B5FFF7BFFC04463549364A364DA84746
:103270003649374A2046A8473649374A2046A847A4
:1032800036A13A4A2046A84739A13D4A2046A847D8
:103290003CA1404A2046A8473FA1414A2046A847B2
:1032A0004049414A2046A84740A1424A2046A847F3
:1032B0004149424A2046A8474149424A2046A84738
:1032C0004149424A2046A8474149424A2046A84728
:1032D000414E424A20463146A847414F414A204686
:1032E0003946A84740A1434A2046A8474249434A95
:1032F0002046A84742A1474A2046A84746A14B4A34
:103300002046A8474AA14F4A2046A8474E4A204691
:103310002949A8474D4A20462949A8474C4A2046F2
:103320002949A8474B4A20462949A8474A4A2046E6
:103330003146A847494A20463946A8472046F8BDA5
:10334000A6DE0008615B00085BAD0008FEDE000839
:10335000695B0008E3DE0008855B00086765744967
:103360006428292D3E696E7400000000A15B0008EE
:103370006765744D6F646528292D3E737472000073
:10338000B55B000867657450696E28292D3E73741B
:1033900072000000C95B000868696768282900009E
:1033A000DD5B000862DF0008595C00086C6F77285D
:1033B00029000000615C0008ECDE0008895C000860
:1033C000D2DE0008995C000818DF0008A95C00083C
:1033D00069DF0008B95C0008B1DE0008C95C0008BC
:1033E000C0DE0008D95C00087265616428292D3EA2
:1033F000696E7400ED5C0008DDDF0008155D0008F3
:103400007365744D6F6465286D6F64653A7374728B
:1034100029000000355D000873657450696E2870DE
:10342000696E4E616D653A7374722900C95D00085A
:1034300073657450756C6C2870756C6C3A7374722B
:1034400029000000F15D0008217E0008DD7E0008F3
:10345000997F0008E17F0008258000087D80000832
:1034600010B5FFF7BFFB044605A1084A07F075FC3D
:10347000B849074A204607F070FC204610BDC046F8
:1034800067657428292D3E696E740000C1510008DB
:1034900009520008B0B5FFF7A5FB044606A10B4A88
:1034A0000B4DA8470BA1184A2046A847A949174A1F
:1034B0002046A8472046B0BD636C65617228636FE3
:1034C0006C6F723A73747229000000009152000808
:1034D0005BAD000866696C6C2878303A696E742CB4
:1034E00079303A696E742C68696768743A696E74E9
:1034F0002C77696768743A696E742C636F6C6F72AD
:103500003A73747229000000D15200086553000814
:10351000F8B5FFF767FB04462B492C4A2C4DA8470A
:103520002C492D4A2046A8472C492D4A2046A84719
:103530002C492D4A2046A8472C492D4A2046A84709
:103540002CA1314A2046A84730A1344A2046A8473A
:103550003349344A2046A8473349344A2046A847CD
:103560003349344A2046A847334E344A2046314630
:10357000A847334F334A20463946A84732A1374A35
:103580002046A84736A13B4A2046A8473AA13F4AD1
:103590002046A8473EA1444A2046A84743A1484A9E
:1035A0002046A8474749484A2046A847474A204658
:1035B0001F49A847464A20463146A847454A204663
:1035C0003946A8472046F8BDA6DE0008855E0008FB
:1035D0005BAD0008FEDE00088D5E0008E3DE00083B
:1035E0009D5E0008B7E40008AD5E000883E40008B3
:1035F000C15E00086765744672657175656E6379B2
:1036000028292D3E696E7400D95E00086765744EE6
:10361000616D6528292D3E7374720000ED5E00080F
:1036200062DF0008515F0008ECDE0008595F000807
:10363000D2DE0008695F00088EDF0008795F0008AD
:1036400077DF0008895F00087365744368616E6EF8
:10365000656C2863683A696E742900009D5F0008F4
:103660007365744475747928647574793A666C6FFF
:1036700061742900BD5F0008736574467265712826
:10368000667265713A696E7429000000F55F000882
:103690007365744672657175656E637928667265C7
:1036A000713A696E74290000416000087365744EB8
:1036B000616D65286E616D653A7374722900000052
:1036C0005D600008A0DF00087D6000081981000827
:1036D000458500089585000880B5FFF783FA80BD11
:1036E000B0B5FFF77FFA04460EA1104A104DA84767
:1036F0001049114A2046A84710A1124A2046A8475F
:1037000011A1134A2046A8471249134A2046A84748
:1037100012A1144A2046A84713A1154A2046A847DB
:103720002046B0BD626C756528290000415700082D
:103730005BAD0008E3DE000859570008666C6F7740
:103740002829000095570008677265656E282900D2
:103750003D58000862DF0008595800087265642867
:10376000290000005D580008776869746528290001
:103770007958000870B5FFF735FA04461549164A1E
:1037800008F09BF81549164A164E2046B0471649D0
:10379000164A2046B04716A1204A2046B04720A12D
:1037A000294A2046B047294D294A20462946B04794
:1037B00028A12C4A2046B0472BA12E4A2046B047CC
:1037C0002DA1344A2046B047334A20462946B04707
:1037D000204670BD6DE40008F92B0008A6DE000845
:1037E0009D7200085BAD00080BE00008F172000854
:1037F00063616C6C5F706572696F645F6D7328667E
:10380000756E5F746F646F3A616E792C7065726962
:103810006F645F6D733A696E742900005D73000810
:1038200063616C6C5F7768656E2866756E5F746F38
:10383000646F3A616E792C66756E5F7768656E3A73
:10384000616E792900000000B173000827DF0008CD
:103850000974000872756E5F666F7265766572280E
:10386000290000002D74000872756E5F6F6E63652D
:10387000282900008174000872756E5F756E746986
:103880006C5F6D7328756E74696C5F6D733A696EE9
:10389000742900008974000811860008F8B5FFF744
:1038A000A1F904461B491C4A1C4FB8471CA11F4ADA
:1038B0002046B8471EA1244A2046B84723A1294ADA
:1038C0002046B84728A12F4A2046B8472EA1324AA1
:1038D0002046B8473149324A2046B847314D324A2E
:1038E00020462946B847314E314A20463146B8472E
:1038F00030A1344A2046B84733A1374A2046B8475A
:10390000364A20462946B847354A20463146B84708
:103910002046F8BDA6DE00089D6000085BAD0008EB
:1039200061736374696D652829000000A160000857
:103930006374696D6528756E69785F74696D653A41
:10394000666C6F6174290000B1600008676D74696E
:103950006D6528756E69785F74696D653A666C6F20
:1039600061742900D16000086C6F63616C74696DCB
:103970006528756E69785F74696D653A666C6F610C
:1039800074290000F16000086D6B74696D65282969
:103990002D3E696E740000001561000827DF0008E5
:1039A00035610008FADF000875610008EBDF0008E8
:1039B0009961000874696D6528292D3E666C6F61F8
:1039C00074000000BD61000874696D655F6E732846
:1039D000292D3E696E7400004562000825860008A6
:1039E00039860008F8B5FFF7FDF804462749284A4C
:1039F000284DA8472849294A2046A8472849294A46
:103A00002046A8472849294A2046A8472849294A44
:103A10002046A8472849294A2046A847284E294A2F
:103A200020463146A8472849284A2046A847284F1B
:103A3000284A20463946A8472749284A2046A84709
:103A400027A12D4A2046A8472CA1344A2046A84742
:103A500033A13A4A2046A84739493A4A2046A8475E
:103A600039A13D4A2046A8473CA1454A2046A847DF
:103A7000444A20461049A847434A20463146A847B1
:103A8000424A20463946A8472046F8BDA6DE00082F
:103A90007D6200085BAD0008FEDE0008856200085C
:103AA000E3DE00089562000862DF0008D5620008C6
:103AB000ECDE0008DD620008D2DE0008ED620008DE
:103AC000B1DE00081163000839DF0008FD6200085C
:103AD00008DF0008396300084DDF0008256300088F
:103AE00072656164286C656E6774683A696E7429E2
:103AF0002D3E737472000000A1630008726561645A
:103B00004279746573286C656E6774683A696E747F
:103B1000292D3E6279746573000000004D63000832
:103B2000736574426175645261746528626175647D
:103B3000526174653A696E7429000000E1630008FF
:103B4000DDDF00080164000877726974652864612C
:103B500074613A7374722900716400087772697431
:103B600065427974657328646174613A6279746539
:103B7000732C6C656E6774683A696E742900000076
:103B8000216400085D8600089D8700084D880008B4
:103B900070B505463C48294608F097FA01240028EC
:103BA00070D13A48294608F090FA00286AD138487E
:103BB000294608F08AFA002864D136A0294608F080
:103BC00084FA00285ED13448294608F07EFA00289D
:103BD00058D13248294608F078FA002852D13048A6
:103BE000294608F072FA00284CD12E48294608F0E0
:103BF0006CFA1024002845D12BA0294608F065FA5C
:103C000000283FD129A0294608F05FFA002839D1C1
:103C10002748294608F059FA002833D12548294673
:103C200008F053FA0126340200282BD122A029469D
:103C300008F04BFA002825D120A0294608F045FAC3
:103C400000281FD11E48294608F03FFA002819D144
:103C50001C48294608F039FA3403002812D11AA06A
:103C6000294608F032FA00280CD118A0294608F09D
:103C70002CFA002806D14848294608F026FA0028E0
:103C800000D1134C204670BD4CE1000815E100083E
:103C900044E10008504236003DE100081DE1000803
:103CA0002AE1000850E1000850413100504237003D
:103CB00048E1000810E1000850413200504238004D
:103CC00019E1000821E10008504133005042390059
:103CD0009F860100B0B504462648214608F0F5F954
:103CE000254D002843D12548214608F0EEF900284B
:103CF0003DD12348214608F0E8F9002837D1214872
:103D0000214608F0E2F9002831D11F48214608F089
:103D1000DCF91E4D00282AD11D48214608F0D5F9AE
:103D2000002824D11B48214608F0CFF900281ED1D5
:103D30001948214608F0C9F9002818D1174821462A
:103D400008F0C3F9002801D0154D10E015482146B0
:103D500008F0BBF9002801D0134D08E013482146B4
:103D600008F0B3F9002801D1054600E0104D2846BF
:103D7000B0BDC0464CE10008002C014050E10008F5
:103D800010E1000821E1000844E1000800040040BF
:103D900048E1000819E1000826E100083DE10008BB
:103DA000002000401DE10008004401402AE1000815
:103DB00000480140B0B51546044601200203914277
:103DC00010D0102918D0000281421FD0012912D131
:103DD000E06AFDF783F92946FDF7D0F8FDF7EDF924
:103DE0006063B0BDE06AFDF779F92946FDF7C6F8D2
:103DF000FDF7E3F92064B0BDE06AFDF76FF92946ED
:103E0000FDF7BCF8FDF7D9F9A063B0BDE06AFDF796
:103E100065F92946FDF7B2F8FDF7CFF9E063B0BDCB
:103E200010B504460168C06A01F0C4F9E06A21686F
:103E300001F0C0F90146394806F077FD606210BD17
:103E400010B50446406A002801D006F031FCE06A53
:103E500007F078F810BDB0B50446002545628562CC
:103E6000056045600572FFF7FFF8E0622562257482
:103E7000E56025776561A561B0BD000070B50446B9
:103E8000C088401CE080FFF7EFF8A062616A0C3147
:103E900008F0CCF9E060A06A216801F08BF9A0611C
:103EA000606A06F005FCA1691C4E304606F03DFD37
:103EB0006062E068017821740029354600D0451C15
:103EC0006561A06901782177002900D0461C26622F
:103ED0001349284608F0F9F8002802D0207A401C3F
:103EE00020721049284608F0F0F8002802D0207A05
:103EF000401E20720C49284608F0E7F8002802D03E
:103F0000207A401C20720949284608F0DEF8002873
:103F100002D0207A401E207270BDC046D8D0000862
:103F2000A4DE000823E00008E9E10008EBE1000856
:103F300010B50446C06AFEF7B7FB206004F07AFDB6
:103F4000A08010BDF8B50D460746002400946846D1
:103F5000394608F06BF90646384604F06BFD074613
:103F6000002F0FD06846314601F024F9017803296B
:103F700005D1401C294608F0A8F8002801D17F1E71
:103F8000EEE70124684606F04EF82046F8BD000032
:103F9000F0B5B1B00F4605461BA807F0BCFFFE4EBA
:103FA0003046314606F0C1FC04903846FCF7CEF8A6
:103FB00007900A21384608F060F80446304631463A
:103FC00006F0B3FC0F901395143509950025A0B2A7
:103FD000069029460D950A950895059708981A9018
:103FE0000C9179181AAC0A22204608F0D6F901463D
:103FF00020460B9108F01AF90446002D12D00F98B4
:10400000214606F0ADFC054601460C311AA808F021
:104010000DF90446284606F04BFBDF48014606F042
:1040200084FC0F900D9D6D1C2046FCF78FF8001945
:10403000401E00785C280D950ED12046FCF786F8CE
:104040000019401E002101700F98214606F088FCDF
:104050000F90012501F05BF81AA82146CF4AD0A3A2
:1040600008F0C6F90446A8B2069988420BD020464B
:10407000FCF76CF82146002864D04A1C401E0978E1
:1040800020291146F7D02046FCF760F80021814234
:104090001BD20A46635C222B01D0272B13D1511C63
:1040A000655C9D42F3D11519AE789E42EFD1002A8E
:1040B00003D06A1E1278202AE9D1EA78202313431C
:1040C000202BE4D13AE0511CE1E70A98002804D003
:1040D0000025FF200A9001F01AF80027219721AD52
:1040E00028462146FEF7E0FA0646284605F09BFFE3
:1040F000002E01D101F027F81AA80D2221460392C3
:1041000008F0E9F80546FCF721F83A4639468842B6
:1041100028D06B5C222B05D0272B07D1FBB25F4246
:104120005F4109E0D3B25A425A4105E03C0603D14F
:10413000140601D1232B08D0491CE8E7FF200A9977
:1041400041400A91002500F0E2FF00246C5428460B
:10415000FBF7FCFFA04204D0295D641C2029F9D0A4
:1041600000E0914D00262D962846904907F0EAFF81
:1041700000280E954ED02C4621AD2846FFF76BFE49
:10418000E11D2846FFF7D4FE2846FFF749FE3546D5
:104190001996344621A88088844228D221AE304620
:1041A000FFF76CFEF088269E012804D12DA8314629
:1041B00008F03CF80546299F38467D4907F085FF01
:1041C000002804D02DA8314608F030F805463046C6
:1041D000774907F07AFF002804D02DA8394608F067
:1041E00025F819902B9806F0ADFE641CD2E721A8A3
:1041F000FFF726FE199800280CD0009001952DA8F5
:1042000080216CA22B4608F076F801461AA808F027
:104210000DF80E902DA805F006FF00252D950E9E99
:10422000304669A107F08EFF002862D021AC2046FD
:10423000FFF711FE711D2046FFF77AFE2046FFF7BB
:10424000EFFD2C461895199521A8808884422AD222
:1042500021A8FFF713FE299F38465D4907F035FF77
:10426000269E002804D02DA8314607F0DFFF054622
:104270003046574907F029FF002804D02DA83946B9
:1042800007F0D4FF19903046494907F01EFF002877
:1042900004D02DA8394607F0C9FF18902B9806F0D6
:1042A00051FE641CD0E721A8FFF7CAFD002D3A4853
:1042B000014619D019990029014615D0284645A173
:1042C00007F003FF002834490ED101951998029098
:1042D0001899002900D0084600902DA880213FA2FF
:1042E0002B4608F008F801461AA807F09FFF04467D
:1042F00000E034462DA805F096FE2B48214607F035
:10430000E4FE0028244D01D000F030FD0A210E9477
:10431000204607F0B2FE401CC0B20A9000252C4691
:104320000A98844201D100F01EFD10941AA80A22B6
:104330000E9908F04DF80746FEF754FC064607F0C4
:10434000A5FD2C46002530953846FBF7FFFE2B4691
:1043500029461194884204D07A5C202A07D1491C4E
:10436000F8E714971D461C461293184667E0002490
:10437000880701D0E04300E088081D460206FF21BF
:1043800009068A4258D11BA006F080F8304607F093
:104390007DF92646274F3FE1D8D0000899DB000879
:1043A0002020202000000000B4E3000896DE000872
:1043B00083DE0008696D706F72742025730A25739F
:1043C000203D20257300000066726F6D2000000004
:1043D00095DE000850696B614F626A00696D706F0D
:1043E00072742025730A2573203D2025732E2573B2
:1043F00000000000496E64656E746174696F6E45FB
:1044000072726F723A20756E657870656374656458
:1044100020696E64656E742C206F6E6C79207375E4
:1044200070706F72742034207370616365730D0A4D
:104430000000000045E300081292149744B242B213
:10444000D3173046DB4907F0D3FA10201BA90856D2
:10445000001B15901996D84F1598854241DA18958A
:104460003046D64907F0ECF9054600280CD1304615
:10447000D24C2146D24A07F020FA3046214607F0B6
:10448000DFF9054607F002FD2DAC002626811794C2
:104490002E962D961BA807F057FD074601460C31B6
:1044A0002046FBF768FE384606F002F92846C54963
:1044B00007F082F907460C4621A8394606F07CFC35
:1044C00016907A1C7441199E2846BE49234607F06F
:1044D0008FFA28461699179A07F0B4FA189D6D1CA2
:1044E000B9E71298801514990C180026152E10D0D3
:1044F000B54885192046294607F024FE002806D035
:104500002846FBF723FEC0B2205C202817D0F61DFA
:10451000ECE70026122E26D0AC4885192046294605
:1045200007F010FE002808D02846FBF70FFEC0B2A7
:10453000205C2021014320290DD00936EAE730A86C
:1045400020223A23214607F086FE0446199E304673
:1045500039462A4652E0199E304629469C4C22464E
:1045600007F070FA50E020469AA107F0EBFD002812
:1045700000D115E2FEF778FD0546211D07F056FE35
:104580000446202218922846214607F021FF0246C1
:10459000199E3046914907F055FA28462146189A47
:1045A00007F016FF20468EA107F0CCFD002805D0AD
:1045B0000122002330468CA107F01AFA3A2228463D
:1045C000214607F005FF02462846894907F00AFE02
:1045D00001462846874A07F005FE014630A807F045
:1045E00025FE0446284606F0ADFC30463946824D8D
:1045F0002A4607F027FA304680A1224607F022FA21
:104600001BA8294607F01AFD30A8214607F088FEAE
:1046100001463046FCF79AFF30A805F004FD00255E
:104620002D952DA86A4907F001FE1790002E00D1A4
:10463000A3E13046614907F003F91290002819966A
:1046400000D1FBE0179F1797129C20465D496D4DE6
:10465000A8471890169120466B4E3146A8471590F2
:10466000149120463146A84707460E4621A83946F0
:1046700006F0A2FB054600237A1C734120466249DE
:1046800007F0B6F91498C0431599C943189A511800
:104690001891169948412046294607F0E8F8002865
:1046A00000D1C9E00546594907F00FFD0028199EC1
:1046B0000ED01898C3B21AAC30462146179AFCF7B0
:1046C000C9FD01462046524A07F08CFD074600E02E
:1046D000179F2846484907F0F8FC00282DD0189865
:1046E000C4B23A461AAF304639462346FCF7B2FD0B
:1046F00001463846464A474B9847024630463946B7
:104700002346FCF7A7FD044643482190304629493B
:1047100007F052F818994018303021AEB070384682
:1047200021463E4A3B4CA047014638463246A04708
:10473000014638463A4AA04707462846394907F015
:10474000C4FC002810D01898401CC3B21AAC199EA3
:10475000304621463A46FCF77DFD01462046324A66
:1047600007F040FD074600E0199E28462F4907F054
:10477000ACFC002800D166E71898401CC3B21AAD03
:10478000304629463A46FCF765FD01462846284A48
:10479000204CA0470246012330462946FCF75AFD2B
:1047A00001462846234AA047014628461E4AA047FC
:1047B000074648E708E3000845E300083BE3000834
:1047C00061300008D6E30008D4D80008A0D800085B
:1047D000D8D00008666F722000000000A4E3000833
:1047E00072616E6765280000697352616E676500CB
:1047F000A0DE000823E00008EAE300086C69737497
:104800005F696E00B9B700088BE300087EE200081C
:1048100068DD0008E5C100085F6C780035DE00083F
:10482000BBDD0008BCE2000842DD00087DE40008B2
:10483000AEDD0008A2DD0008FD4F199E1AA9002573
:104840003046179A2B46FCF705FD04463046F949D9
:104850002A462B4607F0CCF83046394607F007F8D1
:10486000F54907F032FC002857D03046F34906F0EE
:10487000FEFF1890F248014606F057F80546F14849
:1048800021903046F04906F097FF303021AEB070ED
:104890002DAF199819993A4617972346FCF7FEFC55
:1048A00016902846E949EA4CA0473146A047E94915
:1048B000A047054602460C323846169907F092FC8E
:1048C0000746284605F0F4FEDD48014606F02DF8BF
:1048D00005461AA9002319983A46FCF7BBFC07467F
:1048E0002846DD49A0473146199EA047DB49A0472D
:1048F000189D2946A047DA49A0472946A047D9492B
:10490000A047054602460C321798394607F06AFC64
:104910000446284605F0CCFE2AE018943046394675
:1049200006F0A5FFD04907F0D0FB00280AD02DAC37
:10493000304631462246189BFCF7B0FC0146204623
:10494000CA4A12E03046394606F091FFC8A107F086
:10495000BCFB00283DD02DAC304631462246189B8A
:10496000FCF79CFC01462046C24A07F03BFC04468B
:104970001AA8214607F05AFC05462DA805F053FB5E
:104980001199002904D01AA82A4607F02BFC0546E5
:10499000109C002E02D0304606F078FE641CBFE466
:1049A0002046B54907F0CEFB002827D020793A28C9
:1049B000199E02D0202800D026E630463946AE4C5B
:1049C000224607F03FF81BA8214607F037FB9C4C16
:1049D0001AE63046394606F04AFFA74907F075FB4C
:1049E000002829D02DA81899A44A07F0FBFB0346FC
:1049F0002DAA30463146FCF751FCB8E72046A04DC1
:104A0000294607F062FB0028199E00D0A4E5204645
:104A10009C4907F097FB002840D030AD284621463E
:104A200007F004FC044620222846214607F0D0FC6B
:104A300030469349824A93E53046394606F017FFDF
:104A4000914907F042FB00280AD02DAC2046189966
:104A50008A4A07F0C7FB03463046314622467FE7C5
:104A60003046394606F003FF884907F02EFB002840
:104A700024D02DAC20461899854A864EB04705466D
:104A80001998854906F0F3FE024620462946B047AC
:104A900001462046814AB047199E68E72046804972
:104AA00007F050FB00282DD0E11D30A807F038FC9E
:104AB000024630467B4906F0C5FF88E73046394656
:104AC00006F0D5FE784907F000FB002830D03046CC
:104AD000714906F0CCFE0546282107F01FFB00288F
:104AE00059D02DAE2827304629463A4607F055FCC6
:104AF00016902923304629463A4607F0ACFB054676
:104B00004F484BE02046694907F01CFB002821D0A4
:104B100030AD20223A232846214607F09CFB01466F
:104B2000284607F0FDFB044630463946574D27E03E
:104B30003046534906F0ADFE002800D1C8E02DAC48
:104B4000304631462246189BFCF7A8FB014620461A
:104B5000574A0AE72046574907F0F4FA002800D1DF
:104B600052E530AD20223A232846214607F073FB58
:104B70000146284607F0D4FB0446304639464A4DE4
:104B80002A4606F05FFF30464349224606F05AFFA8
:104B90001BA8294619E7169529480546189C294659
:104BA00007F093FA002800D0434D18954248294653
:104BB00007F08BFA17902DAE304621463F4A354D0F
:104BC000A8470446304616993D4AA8470246304653
:104BD0002146A84707463B48219019981A4906F0F4
:104BE000EBFD313021AC6070304639462246A84793
:104BF00001463046184AA847189A014617980028D7
:104C000000D02D4A3046234DA84701463046114A70
:104C1000A847014630462C4AA8470146304622465E
:104C2000A84701463046294AA8470446199E9FE6F0
:104C300045E3000814E30008EAE30008A4E30008E1
:104C4000D8D000085F6C780008E300085CDE00083C
:104C500061A90008BBDD00083CDE000852DE000848
:104C60004ADE000872DD00087EE2000873DD0008FD
:104C7000696600005FDD000898E200084ADD000870
:104C8000C1E3000876DE0008D8E20008BCE20008B4
:104C90002EDE0008E5C10008E2E3000855DD00084B
:104CA0006EDE00084BE300087DE4000869DE0008C2
:104CB00042DD000888DE000824E3000843DE000827
:104CC00053DD000842300A0096DD00088ADD000846
:104CD00030463746F24906F0DCFD00281BD02DACEB
:104CE000384639462246189BFCF7D8FA014620463A
:104CF000FC4AFD4EB04705463846F94906F0B7FD77
:104D0000024620462946B04701462046F74AB047AA
:104D100004463E462CE63846F54906F0BAFD002822
:104D20003E460AD02DAC304631462246189BFCF751
:104D3000B5FA01462046EF4A17E63046EE4906F03E
:104D4000A8FD00280AD02DAC304631462246189BDB
:104D5000FCF7A4FA01462046E84A06E6189B002B19
:104D600000D045E609E6002D00D1ECE113980028BB
:104D7000059F00D1C4E10020159017900A900646C7
:104D80002F4611950A242846214607F076F98642D7
:104D900000DBA2E11494199600242194384607F010
:104DA000B6F9411C21AD284605F000FE06463846FE
:104DB00007F0ADF939460746304618913A46FCF7F8
:104DC00052F8F455E248314605F0AFFD0746284653
:104DD00005F029F92D943D460C352846FBF7B6F928
:104DE0004019401E00780D2806D12846FBF7AEF981
:104DF0004019401E0021017039462878422808D108
:104E0000487B3038159001201790199E189F0D4649
:104E100057E116900E91139A908810909480D6883E
:104E200012971237A0B291680818FBF78FF9139AFE
:104E30000019441C9480A0B2B04209D291680918AC
:104E400006D0384607F041F9139A0028EAD000E06E
:104E5000C04C109890803846BD4907F036F90022C2
:104E60000028109202D01046164624E0A0B2B9499C
:104E7000884202D0002026461DE03846FBF766F93E
:104E80001399CA68441C002A05D008463946904741
:104E90001399086806E00868A2B2394605F0CAFB13
:104EA000139908600C308860C8880019C880287879
:104EB00016902DA80078189F2DA94E800F23159AC3
:104EC00018931A4002431698000110430870129C70
:104ED0000E3403222046A049FBF756F90028199EFC
:104EE000109D00D1C7E0032220469C49FBF74CF9F6
:104EF000002800D19CE00325204699492A46FBF76B
:104F000043F9002800D195E0204696492A46FBF750
:104F10003BF9002800D1AEE0032220469249FBF77E
:104F200033F9002800D187E0032220468F49FBF7A0
:104F30002BF9002800D181E0032220468C49FBF7A1
:104F400023F900287CD0032220468A49FBF71CF96C
:104F5000002877D0032220468749FBF715F900285F
:104F600072D0032220468549FBF70EF900286DD048
:104F7000032220468249FBF707F90028149D7AD0C6
:104F8000032220467F49FBF7FFF8002860D0032268
:104F900020467D49FBF7F8F800285BD00322204625
:104FA0007A49FBF7F1F80028039D64D003222046DC
:104FB0007749FBF7E9F800284ED0032220467549CF
:104FC000FBF7E2F80028189D55D0032220467249CD
:104FD000FBF7DAF8002841D0032220466F49FBF79F
:104FE000D3F800283CD0032220466D49FBF7CCF8CB
:104FF000002837D0032220466A49FBF7C5F800286D
:1050000032D0032220466849FBF7BEF800282DD095
:10501000032220466549FBF7B7F8002828D0032271
:1050200020466349FBF7B0F8002823D0002522E092
:10503000012520E002251EE004251CE005251AE0DC
:10504000062518E0072516E0082514E0092512E0DA
:105050000B2510E00C250EE00E250CE010250AE0D3
:10506000112508E0122506E0132504E0142502E0CE
:10507000152500E016252DA841782943179A002A06
:1050800001D080221143139A0E9D4170126A002AAA
:1050900008D02DA9099C20469047206809E0C04609
:1050A0004BE30008099C20682DA9042205F0C2FAF0
:1050B00020600C301399C861488B001D4883002084
:1050C0001790384607F023F80446284605F0F0FA12
:1050D000E019471C761C119D54E60A9D059F16E0B9
:1050E0004BE3000827DE0008E5C10008BBDD00082F
:1050F00030E300087CDD0008B0E2000883DD000832
:105100000498294605F02CFC049000250A950B987C
:10511000FBF71CF804461AA804F085FF0C98001948
:10512000411C0798814201D2FEF758FF01240498E0
:1051300005F0BEFA0F9805F0BBFA1BA806F0E2FED8
:10514000204631B0F0BD1AA804F06DFF0024EEE750
:10515000D8D00008FFFF0000A9E1000895E1000891
:10516000B1E10008BDE10008D9E10008A5E10008AF
:10517000B9E10008E5E10008CDE1000891E100088F
:10518000C9E10008A1E100089DE10008D1E10008A3
:1051900099E10008ADE1000884E10008C1E10008E0
:1051A000E1E10008C5E10008DDE10008D5E1000803
:1051B000B5E1000880B51F2207F00AF980BD7047ED
:1051C00080B508460D490A68D20704D10968090468
:1051D00005D4012100E0002106F032FA80BD084923
:1051E0000968490601D40221F6E7064909688904DD
:1051F00002D50021C943EFE70321EDE7100000507D
:105200001004005010080050F0B587B01C48016829
:105210000126314301600168314001910199026822
:1052200002210A43026002680A400192019A026860
:1052300004231A430260006818400190019800207E
:1052400006900490059102900196039005200507B1
:1052500001AC0C4F28462146B8470596F003019053
:1052600028462146B8477003019007482146B847B1
:105270004020019005482146B84707B0F0BDC04620
:10528000341002405D240008000800500004005063
:1052900010B5C2B008462B4905F0F0FBFDF780F8C9
:1052A00002A98022002A03D00880521E891CF9E737
:1052B0000124A12C0AD0601E02A9009181B2A3B2E0
:1052C00000208022FCF7EEFF641CF2E742B010BD24
:1052D000F0B5C3B00F461B49384605F0CFFB054675
:1052E00019A11B4E3846B04702901AA13846B04764
:1052F00001901AA13846B047044619A13846B04774
:1053000007462846FDF74CF803A98022002A03D05F
:105310000880521E891CF9E701980019BEB2029953
:1053200089B28F1985B2BE4209D203A80090A0B2FB
:10533000B1B2761CB3B22A46FCF7B4FFF3E743B030
:10534000F0BDC046EEE300086869676874000000BD
:1053500011AA0008776967687400000078300000BF
:1053600079300000F0B591B000200A9010900F90B5
:105370000E90E64E306801242043306030682040B3
:105380000B900B9830680227384330603068384003
:105390000B9028200C900F970B980D940520000778
:1053A0000CAD06902946FCF76FFE07970C97F8485E
:1053B00029462546FCF768FE7068204370607068D7
:1053C0000A9E20400C900C98FF200002D0490A68E9
:1053D00082430A60412081000F46FC37CD480760B8
:1053E000CD4C08230A200590072000020995EA0306
:1053F000CA4D0495256002916160A2600246E0609A
:10540000266166610397A761E36126626662A66210
:105410000598E062266363635D20215C00290893A0
:1054200005900DD0079B2354BC4D29681646402299
:1054300091432960099D2A0331462E46184674E09F
:1054400001925C202654099B1903D04AD068084376
:10545000D060D068009108400C900C9810681843F8
:105460001060106818400B9010960E9607980D90DB
:10547000054606200C900B9803270F970CA9069859
:10548000FCF702FE25210491A5484554A5490B6867
:10549000A54D1D400D603D030B682B4390271F4316
:1054A0000F60A24B11271F60A149099A0A60C663C9
:1054B0000999049A81540562099980220492102264
:1054C000984D05600D4647608260C6600499016191
:1054D00046618661C6610664436480330146483193
:1054E00068C14665866524214654079A1746059982
:1054F00062546065846220680168402291430160C3
:10550000EA02E1680A430F231B029A42334600D0A5
:10551000A3620490019881422A4600D81A46D20715
:105520001A46384600D1009A099E029F6368A56812
:105530003B402127BF022F40FB18256905401D4332
:10554000676937402F43A369039818403843E569DA
:1055500038272F400743256A304680262E403E4399
:105560004503A76A2F403743049E37601B0C042570
:1055700007952B400F252D020D4015431D43616AF1
:1055800010220A402A43616B089F39401143716021
:10559000C102F2698A43F2610A9921660599605451
:1055A000069DAF626420634CA047AF613220A047E4
:1055B0001120614EB0477820A047B120B0470527A1
:1055C0005E4C38460697A0473C252846A04728460B
:1055D000A047B220B0473846A0472846A0472846F3
:1055E000A047B320B0473846A0472846A0472846E2
:1055F000A0473846A0472846A0472846A047B420E1
:10560000B04703200590A047C0273846B047282060
:105610000490A0470898A0470798A047C120B0472A
:105620003846A047C220B0470D200890A0470A98EE
:10563000A047C320B0478D252846A0472A200290C6
:10564000A047C420B0472846A047EE20A047C52069
:10565000B0471A20A0473620B0473846A047E02080
:10566000B047079E3046A0472220A0470720A0470A
:105670000A20A0472E273846A0473020A0472520E3
:105680000390A0470298A0470498A04726252846E3
:10569000A0473846A0473A200490A0470A98A04760
:1056A0000998A0470598A04713200590A047E1203E
:1056B000214988473046A0471620A0470620A0472A
:1056C0000898A0472D273846A0472846A047232002
:1056D000A04727252846A0472846A0470398A0476B
:1056E0003846A0473B20A0470A98A0470998A04702
:1056F0003046A0470598A04704980F4DA847069844
:10570000A0472920A84711B0F0BDC0463410024080
:1057100008E400E000E100E0140100200030014056
:10572000B8000020080002400F80FFFF0008024080
:10573000840802406D2000086523000881230008CA
:10574000B0B50824534D2046A8472046A847204618
:10575000A8472046A847B0BDFEB50C480168022204
:1057600011430160006810400090009800200590EF
:1057700004900390029201200190000300900448DD
:105780006946FCF76BFE06B080BDC046341002408F
:1057900000040050F8B50446164906F07AF80028CF
:1057A00005D1144900222046134606F021F911497B
:1057B000204606F001F8054603280DD8AE000EA0DD
:1057C0008059114FB84711A08059B84713A080598C
:1057D000B84716A08059B847681CC117890F4118EF
:1057E00003229143421AD3170249204606F000F9DA
:1057F000F8BDC046A6E2000800080000080000004E
:1058000000000800080808002D75000808000000C6
:105810000000080008080800000800000000080058
:105820000808080000080000080000000808080038
:10583000000800000800000000000800B0B50120CA
:10584000C404144D2046A8472046A8472046A84730
:105850002046A847B0BDC04670470000B0B5012043
:10586000C4020C4D2046A8472046A8472046A8471A
:105870002046A847B0BDC046B0B5054C054D2046F2
:10588000A8472046A8472046A8472046A847B0BDBD
:10589000080808002D75000880B5704905F0D5FF8F
:1058A00005F050FB80BDC04670B50C460546394E2C
:1058B0000846314605F0C6F82846314605F07CFF1B
:1058C0000146284600F07AF80146204605F0A6FE7B
:1058D00070BDC04610B50446604905F0DAFF0028E7
:1058E00000D010BDFDF7C8FB02465C49204606F01B
:1058F00093F810BDB0B50C46054617490022134673
:1059000006F076F80448294605F003F801462046DB
:1059100005F084FEB0BDC046D8D00008F8B50C46EE
:10592000064600680C4905F073F8074630463946CC
:1059300000F044F8002807D0054630687A1CD317D9
:10594000054905F09BF902E004F0D2FF0546204628
:10595000294605F063FEF8BD1BE30008F8B50E46C6
:1059600004460C4D0846294605F06CF80A4F3046AF
:10597000394605F067F82046394605F0BBFE064675
:105980002046294605F018FF02462046314600F021
:105990003DF8F8BD0EE5000873E30008B0B50A460F
:1059A00004464349104605F04DF805462B4920466C
:1059B00005F04BFF294605F0CFFAB0BD10B50C46F7
:1059C000264905F042FF214605F0E4FA04F057FEAF
:1059D00010BDC046B0B50C4605463649204605F018
:1059E00017F801462846FFF7E9FF0146204605F073
:1059F00015FEB0BD10B50C46184905F026FF05F0A0
:105A0000D5FA0146204605F01BFE10BDF0B585B065
:105A1000174601910646114905F017FF044602A8F2
:105A2000394605F0C9F905460D49204604F0F0FF56
:105A3000B84207DA0121304605F0BCFF09A006F0A4
:105A400013F809E0019804F01AFE294604F038FF23
:105A50000146204605F0ACF805B0F0BD05E50008AC
:105A6000D6E300085B6572726F725D3A20696E64FE
:105A70006578206578636565646564206C656E672C
:105A800068206F66206C6973742E000070B50C4638
:105A900005460749204604F0D5FF0646054920463D
:105AA00004F0B6FF024628463146FFF7AFFF70BD4F
:105AB000FAE2000822E3000880B500F00DF880BD8E
:105AC00080B52F4905F040FF80BDC04680B5334901
:105AD00005F03AFF80BDC04680B5C449014A05F0D3
:105AE000B1FF80BD15E1000880B5FFF7F5FF80BD6F
:105AF00080B5012105F05EFF7B4805F0B5FF80BD54
:105B000080B5012105F056FF774805F0ADFF80BD57
:105B100080B5012105F04EFF734805F0A5FF80BD5B
:105B2000B0B50C460546794905F00EFF04492846F4
:105B300005F024FE024620460B4605F07BFDB0BD75
:105B400075E30008B0B50446A84D0846294604F0A0
:105B500095FF02462046294605F074FFB0BDC046B9
:105B600080B500F051F880BD10B5044636490022DA
:105B7000134605F03DFFC849204605F0E5FE10BD7F
:105B80006EE2000810B504462F490122002305F0FB
:105B90002FFFC549204605F0D7FE10BD56E200088C
:105BA00010B50C46624905F007FE0146204605F097
:105BB00047FD10BD10B50C46714905F058FE014671
:105BC000204605F045FD10BD10B50C46DD4905F039
:105BD0004EFE0146204605F03BFD10BD10B50446C3
:105BE00004490122002305F003FF03A1204605F02C
:105BF000ABFE10BD96E30008706C6174666F726D49
:105C00004869676800000000F8B504460E490025A1
:105C10000E4E2A462B46B047CA49CB4A0C4F204667
:105C2000B8475749574A2046B847134920462A469D
:105C30002B46B04782492046C34AB847EB433C490C
:105C4000044A2046B047F8BD65E20008F1B90008F3
:105C500045BA000819FCFFFF80B5FFF7D5FF80BDEE
:105C600010B5044604490022134605F0C1FE03A105
:105C7000204605F069FE10BD96E30008706C617463
:105C8000666F726D4C6F770080B5012105F092FE52
:105C9000C14805F0E9FE80BD80B5012105F08AFE0E
:105CA000BD4805F0E1FE80BD80B5012105F082FE12
:105CB000B94805F0D9FE80BD80B5012105F07AFE16
:105CC000B54805F0D1FE80BD80B5012105F072FE1A
:105CD000B14805F0C9FE80BD80B5012105F06AFE1E
:105CE000AD4805F0C1FE80BD49E00008B0B50C46E6
:105CF0000546064905F028FE0549284605F05CFDE5
:105D00000146204605F09CFCB0BDC0461FE20008DD
:105D1000C4E20008B0B50446054D0846294604F023
:105D200077FE0246C3172046294605F061FEB0BD46
:105D30002CE20008B0B50A4604461149104604F0AA
:105D40009DFE05460F4906F0C0F9002805D10EA1B9
:105D5000284606F0BAF9002809D0094920462A4603
:105D600005F070FE09A1204605F0EEFDB0BD012151
:105D7000204605F01FFE09A005F076FEB0BDC04626
:105D800051E200080AE50008696E0000706C617459
:105D9000666F726D5365744D6F6465005B657272FA
:105DA0006F725D204750494F206D6F6465207368A6
:105DB0006F756C6420626520276F757427206F7281
:105DC0002027696E272E000010B50A46044605A15B
:105DD000104604F053FE0246AF49204605F032FE5D
:105DE00010BDC04670696E4E616D6500B0E300087D
:105DF000B0B50A4604461249104604F03FFE054677
:105E0000104906F062F900280BD10F49284606F028
:105E10005CF9002805D10D49284606F056F90028FE
:105E200005D0074920462A4605F00CFEB0BD0121E9
:105E3000204605F0BFFD06A005F016FEB0BDC04629
:105E400086E30008DAE30008C8E3000893E20008EC
:105E50005B6572726F725D204750494F2070756CA0
:105E60006C2073686F756C642062652027757027DD
:105E70002C2027646F776E27206F7220276E6F6E3D
:105E800065272E0080B500F03BF880BD80B5024943
:105E900005F05AFD80BDC0466EE2000880B502499B
:105EA00005F052FD80BDC04656E2000810B50C4614
:105EB000414905F081FC0146204605F0C1FB10BDBB
:105EC00010B50C46464905F059FC024620460B46E3
:105ED00005F0B0FB10BDC04610B50C465E4905F09C
:105EE0006BFC0146204605F0ABFB10BD10B50C461F
:105EF000614905F0BCFC0146204605F0A9FB10BD38
:105F0000B0B504466449104D2A4605F09BFD5A4938
:105F100020462A4605F096FD7D20C2004E49002508
:105F200020462B4605F064FD234920462A462B4691
:105F300005F05EFD2A49054B20462A4605F044FD42
:105F4000B0BDC046B0E3000893E200080000E03FA7
:105F500080B5FFF7D5FF80BD80B5012105F02AFD92
:105F6000EA4805F081FD80BD80B5012105F022FDE4
:105F7000EB4805F079FD80BD80B5012105F01AFDE3
:105F8000EC4805F071FD80BD80B5012105F012FDE2
:105F9000ED4805F069FD80BD49E00008B0B5044654
:105FA000054D0846294604F033FD0246C317204636
:105FB000294605F01DFDB0BDFEE20008B0B504465F
:105FC000074D0846294604F007FD02460B462046C9
:105FD000294605F0F9FC03A1204605F0B5FCB0BD4B
:105FE00088E50008706C6174666F726D5365744467
:105FF0007574790010B50A4604461749104604F036
:1060000007FD0146204600F001F810BD10B50A4614
:106010000446CB17034905F0EBFC03A1204605F02D
:1060200093FC10BDDDE30008706C6174666F726DE7
:106030005365744672657175656E63790000000082
:1060400010B50A4604460449104604F0E1FC014636
:106050002046FFF7DBFF10BDDDE30008B0B50446C6
:10606000054D0846294604F009FD0246204629460A
:1060700005F0E8FCB0BDC04684E20008B0B50446B7
:10608000054D0846294604F0F9FC024620462946FB
:1060900005F0D8FCB0BDC046B0E300087047000072
:1060A00080B5012105F086FC214805F0DDFC80BDAE
:1060B00010B50A4604461649104604F08DFC01212D
:1060C000204605F077FC1A4805F0CEFC10BDC0460E
:1060D00010B50A4604460E49104604F07DFC012125
:1060E000204605F067FC124805F0BEFC10BDC04616
:1060F00010B50A4604460649104604F06DFC01211D
:10610000204605F057FC0A4805F0AEFC10BDC0461D
:1061100089E2000810B50C46012105F04BFC04484B
:1061200005F0A2FC0021204605F08AFA10BDC04609
:1061300076E0000880B5012105F03CFC01A005F0E7
:1061400093FC80BD5B6572726F725D20706C6174D0
:10615000666F726D4765745469636B2829206E659C
:10616000656420746F206265206F76657272696461
:10617000652E000010B50A4604460649104604F094
:1061800047FC0121204605F015FC6F4805F06CFC2A
:1061900010BDC0467AE4000810B50A460446064918
:1061A000104604F035FC0121204605F003FC66484A
:1061B00005F05AFC10BDC04681E40008F0B58DB072
:1061C0000C46064601AD17A119222846FAF74BFEE8
:1061D0003046294605F044FE00250B950A950995A1
:1061E000089508AF3046394606F072F93046394610
:1061F00006F05EF908980999FAF7B0FF06460F46CF
:106200000A98FAF789FF0E4B2A46FAF7FDF932464B
:106210003B46FAF7DFF8024620460B4605F00AFA3D
:106220000DB0F0BD040000820100110000706C612F
:1062300074666F726D4765745469636B000000008B
:1062400065CDCD417FB50C460546002003900290F8
:10625000019000906E462846314606F039F92846EE
:10626000314606F025F9044800994143029809187F
:10627000204605F0E5F97FBD00CA9A3B80B500F0E5
:1062800011F880BD80B5024905F05EFB80BDC046B7
:106290006EE2000880B5024905F056FB80BDC0469D
:1062A00056E20008B0B50446E120420253490025F9
:1062B00020462B4605F09CFB5849012220462B46E0
:1062C00005F096FB0249CB4A204605F0BBFBB0BD6A
:1062D000C4E2000880B5FFF7E5FF80BD80B501216D
:1062E00005F068FB184805F0BFFB80BD80B50121B3
:1062F00005F060FB144805F0B7FB80BD80B50121B7
:1063000005F058FB104805F0AFFB80BD49E00008E0
:1063100080B5012105F04EFB0B4805F0A5FB80BDC3
:1063200049E0000880B5012105F044FB064805F06E
:106330009BFB80BD49E0000880B5012105F03AFBD8
:10634000014805F091FB80BD49E0000870B50C469E
:1063500005460D4E0846314604F05AFB0246C31767
:106360002846314605F044FB08A1284605F0ECFA22
:106370001A49284605F0BEF904F081F90146204685
:1063800005F04CF970BDC04601E30008706C617403
:10639000666F726D526561644279746573000000C6
:1063A00070B50C4605462B4E0846314604F030FBCE
:1063B0000246C3172846314605F01AFB064928460F
:1063C00005F0C2FA0549284605F051FA0146204673
:1063D00005F03EF970BDC0461FE20008F6E1000876
:1063E000B0B50446054D0846294604F011FB0246A7
:1063F000C3172046294605F0FBFAB0BD9DE2000810
:10640000B0B50446054D0846294604F001FB024696
:10641000C3172046294605F0EBFAB0BD2CE2000870
:1064200070B50D4604460A49284604F0C9FA0646E6
:106430000849284604F0ECFA03460749204632464C
:1064400005F0A0FA05A1204605F07EFA70BDC04611
:1064500009E2000801E30008FFE10008706C6174C4
:10646000666F726D57726974654279746573000066
:1064700010B50A4604460749104604F0FFFA0246E2
:106480000549204605F0DEFA04A1204605F05CFA35
:1064900010BDC04609E20008FFE10008706C61749D
:1064A000666F726D577269746500000010B50C4616
:1064B000034804F06FF90146204605F0AFF810BD1F
:1064C000C12D000810B50C464C202449085AFAF793
:1064D00037FE00221D4BFAF72FF8024620460B46E6
:1064E00005F0A8F810BDC04610B50C4648201B4961
:1064F000085AFAF725FE0022144BFAF71DF8024657
:1065000020460B4605F096F810BDC04680B54C20DD
:106510001249085AFAF714FE00220C4BFAF70CF84D
:1065200002460B480B4603F0B1FF80BD80B5482002
:106530000A49085AFAF704FE0022044BF9F7FCFF57
:10654000024603480B4603F0A1FF80BD0000503F08
:1065500025DC000801480021C164704718000020B4
:1065600010B50C46034804F015F90146204605F025
:1065700055F810BD492E000810B50C46034804F02C
:1065800009F90146204605F049F810BD512E0008D2
:10659000F8B5009106681249124C3046A0470546EE
:1065A00011493046A047074610493046A0471049D8
:1065B000884200D00546BD420BDA6A1CD3170B494E
:1065C000304604F05BFBEB17CF482A4604F06FF926
:1065D00001E004F08DF90146009805F01FF8F8BDC0
:1065E0002EE1000811AA000834E100081DE30008AC
:1065F000013665C4D8D0000810B50C46034804F035
:10660000C9F80146204605F009F810BD692E0008BA
:1066100010B50C4604F06CF90146204604F0FEFF6C
:1066200010BD000010B50C46034804F0B3F8014655
:10663000204604F0F3FF10BD852E0008B0B58AB0E7
:106640000C460246002901D0A07900E00220002576
:10665000002A03D09179042900D1D568072812D0E7
:1066600006282AD16846202101800C34002D03D54C
:106670002046F9F76BFD4519605D694608701E48B4
:1066800004F053F935E0684620210180204610309F
:10669000002D0AD5217B627B12025118A27BE37B7D
:1066A0001B029A18120451184D19405D6946087072
:1066B0001148012204F0A8F81BE00938FD21084226
:1066C00002D004F015F914E0E4680C49204605F006
:1066D00054F96D460AA125222846FAF7C4FB204644
:1066E000294605F0BDFB20680F4904F0ABF903F023
:1066F000C6FF0AB0B0BDC046D8D000080EE50008FD
:106700000C00108101000002070000040F001500BA
:10671000005F5F6B6579005F5F6765745F5F005F57
:106720005F726573000000004FE40008B0B50C46CE
:106730003449204604F086F905465449204604F0C1
:1067400081F901462846FFF779FF0146204604F00B
:1067500065FFB0BDF0B58DB00C46019029492A4EB9
:106760002046B047029029492046B047054628A157
:10677000204604F083F9074627492046B047002DFC
:106780003ED00446A87907280CD006281FD1207BCC
:106790000299C9680C356854019839462A4605F0B3
:1067A00051F92DE0A87BE97B2A7B6B7B247C029E40
:1067B000F6681035AC551B029A1809020818000437
:1067C0008318019839462A4605F0DCF818E00938A4
:1067D000FD21084214D1ED6810492846029A05F0BF
:1067E000CCF80F492846224605F0C7F803AC0DA1A6
:1067F00025222046FAF737FB2846214605F030FBD4
:106800000DB0F0BD10E5000845AA00082CE3000813
:106810006F626A5F7374720075E300080EE500082A
:1068200073E300080C001081010010010700000252
:106830000D001500005F5F6B6579005F5F76616C2E
:10684000005F5F7365745F5F0000000070B50C4609
:106850000CA10D4E2046B0470C492046B0470546D6
:106860000BA12046B04706460BA1204604F0D0F805
:1068700030462946FFF7E2FE0146204604F0CEFEF0
:1068800070BDC046656E640045AA00082CE3000890
:10689000737461727400000073746570000000000E
:1068A00070B50C4606461749204604F0CBF8002880
:1068B0000BD005468079072811D0062813D004286C
:1068C00003D1EA681048002114E00121304605F0A8
:1068D00071F80EA003F0DAFD04F00AF80CE0284687
:1068E00003F0CDFE08E00C352846F9F72FFC0246F0
:1068F0000548294603F088FF0146204604F08EFE35
:1069000070BDC04675E30008D8D000084572726FAC
:10691000723A20696E7075742061726720747970A4
:1069200065206E6F7420737570706F727465642E5D
:106930000D0A0000F0B58DB00D46039048A1284621
:1069400004F09CF8044647A10495284604F08DF80D
:10695000064645480027C76409970B970BAD2846A4
:10696000214605F063FC014625222846069105F0E4
:106970002FFD01463D4803F0D8FF044601200002E8
:1069800005900796304604F011FB874245D20894E3
:1069900000250A953046394604F0FCFA06460AAC52
:1069A00025222046069905F013FD0246204631496E
:1069B00005F018FC0C95002E1BD00246B079062875
:1069C00007D005280CD0042813D1F3680CA805992A
:1069D00003E00C360CA80599334605F08CFC07E063
:1069E000F0683169009001910CA8059905F083FCCD
:1069F00005460AAE3046294605F018FC04460CA8A8
:106A000003F011FB0898214603F0AAFF0446304624
:106A100003F009FB7F1C079EB4E721460C3109AD4A
:106A2000284605F003FC264604460BA803F0FBFAB3
:106A3000304603F03DFE0E4E039F38463146224657
:106A400005F000F83846314604F011FF04462846A8
:106A500003F0E9FA0498214604F0FAFD0DB0F0BD08
:106A6000666D74007661720018000020D8D00008AE
:106A7000DEE200089EDE0008F0B5C1B00C46054617
:106A80005C49204603F0C4FF07460120010201AE25
:106A90003046FAF70FFA6A463020108017700A491C
:106AA000304603F0FFFC584F28463946324604F082
:106AB000C9FF2846394604F0DAFE0146204604F0B4
:106AC000C7FD41B0F0BDC04644E4000810B50C4617
:106AD000012104F06FFF05A003F0D8FC03F008FFCC
:106AE0000146204604F09AFD10BDC0465B45727217
:106AF0006F725D206275696C742D696E20646973B4
:106B000074206973206E6F7420656E61626C6564B9
:106B10002E0D0A00B0B50C4605461449204603F078
:106B200091FF00280AD08179052911D0042905D1C7
:106B3000C26801691046FAF7D8FA0EE00CA004F01A
:106B400093FF0121284604F035FF134B134A08E058
:106B5000C26801691046FAF703F9FAF767FB0246C3
:106B60000B46204604F066FDB0BDC046FAE20008C0
:106B70005B6572726F725D20636F6E7665727420F2
:106B8000746F20646F75626C65207479706520661F
:106B900061696C642E000000FF69F8C0A583F5FFF1
:106BA00070B5C0B00C4605461249204603F030FFD0
:106BB0000646012001026846FAF77CF9012E03DB44
:106BC00068460FA1324602E0724268460AA103F00D
:106BD00069FC0D4E6A462846314604F033FF2846CC
:106BE000314604F044FE0146204604F031FD40B039
:106BF00070BDC04675E300082D307825303278002E
:106C00003078253032780000DDE2000810B50C46FF
:106C10000A49204603F016FF002807D00146807974
:106C20000938FD22104202D1C96800E0002101208C
:106C3000C0078143204604F003FD10BD2CE300088B
:106C4000B0B50C4605461D49204603F0FBFE002862
:106C50000CD08179091F032908D8C04679440979E5
:106C600049008F44011E0C10C16820E01FA004F0F1
:106C7000FBFE0121284604F09DFE1B4917E00C3065
:106C800004F072F812E0017B427B12025118827B01
:106C9000C37B1B029A181204511801290BD1017CE5
:106CA00005E0C26801691046FAF79CFA01462046E1
:106CB00004F0C6FCB0BD02A0D9E7C046FAE2000865
:106CC00056616C75654572726F723A20696E7661B5
:106CD0006C6964206C69746572616C20666F7220E7
:106CE000696E742829000000013665C45B65727204
:106CF0006F725D20636F6E7665727420746F2069A9
:106D00006E742074797065206661696C642E000071
:106D1000F0B587B00C4606462249204603F092FEA5
:106D2000002813D0054680790A2831D0062809D1D9
:106D30000C351DA130462A4604F084FE1C4803F0A1
:106D400033FD28E00938FD21084202D003F0D0FDD0
:106D500021E0EE681749304604F077FD1649884275
:106D600016D06D4615A11C222846FAF77CF830464D
:106D7000294605F075F83068174F394603F062FE72
:106D800003F07DFC05463046394604F0C5FD03E0BE
:106D9000284603F074FC05462046294604F03EFCD4
:106DA00007B0F0BDFAE200085F736F626A0000008E
:106DB000692E0008FDE30008512E0008080000823B
:106DC000010000040A001000005F5F697465725FD3
:106DD0005F005F5F726573004FE40008B0B50C465A
:106DE00005461449204603F02DFE002809D081797C
:106DF000072910D0062904D10C30F9F7A7F901466C
:106E000013E00121284604F0D5FD0BA003F03EFB62
:106E10000020C14309E0017B427B12025118827BB2
:106E2000C07B0002801800044118204604F008FCD2
:106E3000B0BDC046FAE200085B4572726F725D2019
:106E40006C656E3A206172672074797065206E6F90
:106E50007420737570706F72740D0A0010B50C4653
:106E6000012104F0A7FD05A003F010FB03F040FD95
:106E70000146204604F0D2FB10BDC0465B4572724D
:106E80006F725D206275696C742D696E206C697318
:106E900074206973206E6F7420656E61626C656426
:106EA0002E0D0A0010B50C466449204603F0E6FD9D
:106EB0000178204604F0C4FB10BDC046F0B585B093
:106EC0000A4604465D49104603F0CFFD029004F0E7
:106ED0006DF80390401E00903E48014603F025FDEA
:106EE0000546002601960398864265DA02983146E7
:106EF00004F050F807460021204604F05BFD002F07
:106F00000AD0B879072803D1384603F055FC37E09A
:106F10000938FD2108422AD00495FCF7A5F805465A
:106F20003846464903F0CCFC384603F0A8FB01463E
:106F3000284603F03DFE284603F0C4FD00280AD091
:106F400002462046254F394604F07CFD284603F0D2
:106F5000F9FF049D15E03B4804F086FD0121204621
:106F600004F028FD284603F0EDFF049D08E0F868D2
:106F700004F07EFD0028CFD00146174803F086FAC2
:106F8000164F2046394604F072FC002812D0014604
:106F9000284603F0E5FC05460098864204DA2846B8
:106FA0000F4903F0DDFC05462046394604F0B4FCE9
:106FB00001200190761C96E70198012804D129460A
:106FC0000C31054803F062FA284603F071FB05B066
:106FD000F0BDC046D8D000083DDD0008DEE2000864
:106FE0009CDE000870B50A4604461449104603F0BA
:106FF00029FD06460021204604F0DCFCFCF734F8AD
:107000000546304603F03BFB0146284603F0D0FD21
:10701000284603F057FD002804D00146084803F035
:1070200035FA06E0074804F01FFD0121204604F070
:10703000C1FC284603F086FF70BDC04675E300081A
:1070400044E4000852E30008F8B50C4600911049EA
:10705000204603F0DDFC06460E49204603F0D8FC2E
:1070600007460D4803F096FB0546F317C468204613
:107070000749324604F0BCFCFB17204605493A4656
:1070800004F0B6FC0098294604F0C8FAF8BDC046E2
:107090002EE1000834E10008512E0008B0B50A4680
:1070A00004460BA1104603F0E9FC054600212046EA
:1070B00004F080FC2046294604F02EFC012806D16D
:1070C00005A004F0D1FC0121204604F073FCB0BD02
:1070D00061726750617468005B6572726F725D20E7
:1070E00064656C3A206F626A656374206E6F206617
:1070F0006F756E642E0000007FB50C4605463D4955
:10710000204603F09FFC00280FD0817900220392D3
:1071100007290DD005290DD0042915D1C36803A86E
:107120000B21174A05F0E7F815E00022039213E05F
:10713000103010E0C16800690091019003A80B2194
:107140000E4A05F0D8F806E00939FD23194203D1AB
:10715000C06804F08DFC02460A4E2846314604F011
:1071600071FC03A802F05FFF2846314604F07FFB64
:107170000146204604F06CFA7FBDC046B9E2000823
:107180001CE20008DDE2000810B50A460446194971
:10719000104603F057FC002811D08079001F0C28FE
:1071A00026D8C0467844007940008744061012145F
:1071B000211618211A21211C1E00364816E03648D7
:1071C00004F052FC0121204604F0F4FB10BD3048CD
:1071D0000CE02BA00AE01BA008E024A006E01DA004
:1071E00004E00FA002E009A000E003A004F03CFCD2
:1071F00010BDC046FAE200083C636C61737320273F
:1072000066756E6374696F6E273E00003C636C6147
:10721000737320276D6574686F64273E000000005B
:107220003C636C617373202762756974696E5F6675
:10723000756E6374696F6E5F6F725F6D6574686F92
:1072400064273E003C636C61737320276279746528
:1072500073273E003C636C61737320276D65746116
:10726000206F626A656374273E0000003C636C61B6
:10727000737320276F626A656374273E0000000005
:107280003C636C6173732027737472273E000000A7
:1072900063E1000873E100082DE00008B0B5044682
:1072A0000EA10022134604F0A3FBED48056D0E4924
:1072B000204604F0C5FA04460C49284604F076FA44
:1072C000002809D0054609482E2104F04FFF014649
:1072D0002868224603F0E8FCB0BDC04669735F70C1
:1072E0006572696F640000006DE400086BE40008DB
:1072F000B0B58EB004460B4D0846294603F0A2FBFC
:1073000002462046294604F038FB01AD06A1322290
:107310002846F9F7A8FD2046294604F0A1FD0EB045
:10732000B0BDC046CDE3000810001083010000028C
:10733000080010811500000208001E0000616C7733
:107340006179730063616C6C732E617070656E643B
:107350000066756E5F746F646F000000F0B597B0E3
:107360000D460446254E0846314603F06BFB0746A2
:107370000D49284603F04CFB0546204631463A4667
:1073800004F0FBFAEB17204607492A4604F030FBCD
:107390006D4606495B222846F9F765FD20462946D9
:1073A00004F05EFD17B0F0BD73E40008DCD0000807
:1073B000F0B591B00D4604461049284603F042FB53
:1073C00007460F4E2846314603F03CFB0546204653
:1073D0000A493A4604F0D1FA204631462A4604F0DA
:1073E000CCFA6D46074941222846F9F73CFD204674
:1073F000294604F035FD11B0F0BDC046CDE30008CC
:107400009BE3000838D1000880B5012104F0D2FACE
:10741000014804F029FB80BD49E0000804462046ED
:1074200002F01EFC204600F003F8F8E7FFF7F6FF35
:10743000B0B5FFB0BFB00C4D2C6D0C4904F0BCF9D9
:1074400002460B460AA1204604F0D2FA6C460A49CD
:107450000A4A2046F9F707FD286D214604F000FD91
:107460007FB03FB0B0BDC0461800002036E3000832
:107470005F5F7469636B00007CD10008F602000056
:1074800080B5FFF7D5FF80BDF8B50A4604460BA1CD
:10749000104603F0BDFA0546C7170B4E204602F012
:1074A000DFFB2046FFF7C4FF2046314604F084F995
:1074B000281A38468841F1DAF8BDC046756E7469FD
:1074C0006C5F6D730000000036E3000810B5144CCB
:1074D000A068382101401348082920D0102919D16B
:1074E000E16803220A401049032A00D00846022A14
:1074F00000D00146E0684004400E4843E168490678
:10750000490F491CF9F73EF9E168490F491CF9F7A1
:1075100039F910BD20688004410F0348C84010BDF0
:1075200000100240001BB7000024F40080B584B0B6
:10753000039001A90020087017200290FFE702982D
:10754000002816D4FFE703990298C14001200140AA
:1075500001A801700078002803D0FFE700F01EF8B2
:1075600002E000F009F8FFE7FFE70298401E0290F2
:10757000E5E704B080BD000081B001200003184998
:1075800008600099491C00910099491C00910099DC
:10759000491C00911349086001B0704781B0012077
:1075A00000030F4908600099491C00910099491C8B
:1075B00000910099491C00910099491C0091009983
:1075C000491C00910099491C00910099491C0091A7
:1075D0000099491C00910349086001B07047C046FA
:1075E0001804005028040050806A01684A68032388
:1075F0009A434A60016E10220A4302665D2101220D
:107600004254704770470000BCB57149CA6B846A28
:1076100000680068800622D4206841682025A943BC
:10762000416041680223994341606421204600F093
:1076300019F8002802D0206E28432066A068002890
:1076400007D1002001902068C168019180680190F5
:1076500001980020E0875D2001212154206EBCBDEF
:1076600018000020FEB516460F4605460324E10229
:107670003A46334600F05CF800282BD128465C30AF
:107680000090534BD86B301AC219524840684001E1
:10769000010D5143D86B0190029129688B681B063C
:1076A0000FD57B1CFAD04A48C36B01981B1A934232
:1076B00018D2029B0298401E0290002BEED11A466F
:1076C000ECE70320410228463A46334600F030F802
:1076D000002805D0286E2021014329662046FEBDE2
:1076E0000024FBE74868E022904348604120800086
:1076F0006A6882420BD1A8680122D303984202D063
:107700009202904203D10868402290430860012011
:107710004203AB6A934205D10B6893430B600B683D
:1077200013430B600021009A11705070D2E7C046DD
:10773000FCB5E04DEC6B1B1B9F18264B5B682324AC
:107740005C43230D7B43EE6B0193056803465C337A
:107750000093AB680B4213D003235C02A14200D11B
:107760002C7B541CF5D0D34CE46BA41BBC420AD236
:10777000019B019C641E0194002BEAD11F46E8E79F
:1077800000231846FCBD6968E022914369604121ED
:10779000890042688A420BD181680122D403A14248
:1077A00002D09202914203D129684022914329607C
:1077B00001214A03806A904205D1286890432860DD
:1077C0002868104328600020009A10705170D8E794
:1077D0001800002010000020F0B587B0B44A546DA6
:1077E000264624367378012BFCD15D27D35D012B0F
:1077F000F8D15C23D55C012D00D1BEE0D55D012D13
:1078000000D0B8E0002800D1B5E00D0400D1B2E00E
:1078100004930325D5554425002353531366D1877C
:10782000462553539187029090631364D364059364
:107830001365106801210691CD039168A94208D112
:1078400001684025A94301600699890305680D4335
:1078500005604B4B4B4D4C49E562216363630599D1
:10786000A1634168494B1940039041600721090217
:10787000D5688D42049B17D806988102A5698D4270
:1078800012D1D18F03984568C90705D13F490D40F2
:107890004560D18F480806E0069989030D4345608D
:1078A000D18F4908481CD087D08F317801295CD00E
:1078B000069D35707178012953D100900220019006
:1078C00070700598E06327683868A8433860A06C3A
:1078D000E16C4160206D059000282E4602D0606D5D
:1078E000A16D4160039D0C35206C1C210140304688
:1078F000884027490E6806430E6000987860A668A5
:10790000102E2946029800D00146B960102E00D0F2
:107910002846F86038680E2101433960069E30021F
:10792000646C2168C90302D5216801432160059D6B
:10793000002D039C02D02968014329603868304338
:1079400038602068400603D420684021014321604C
:1079500060682021014361606068019908436060AC
:1079600009E0059830708020E063106E102101431B
:1079700011660698D0550020D05407B0F0BDC0461F
:10798000E97500080976000805760008FFBFFFFFCB
:1079900004000240F0B585B003A908705C25444E90
:1079A000715D012900D180E0012777554149CC6BF9
:1079B0005D22B35C012B75D1009403230292B35472
:1079C00044230022F2523266F7874623F252B787E9
:1079D00003ABB3633264F2640192326533683A46B2
:1079E000FF03B468BC4207D11C684027BC431C603D
:1079F00094031F6827431F601C68640603D41C6837
:107A0000402727431F60F4682B4FBC4219D303A8BB
:107A10000488DC60801CB063F38F5B1EF3873368DF
:107A20001746F48F002C26D09C68A40701D4CC6B99
:107A3000F7E70488DC60801CB063F48F641EF48771
:107A4000EFE71873B06B401CB063F38F5B1EF387D6
:107A500033681746F48F002C0DD09C68A40701D41E
:107A6000CC6BF7E700781873B06B401CB063F48FF1
:107A7000641EF487EEE7019CE1430D48009AFFF78E
:107A8000F1FD0B4B002801D02020186698680028D3
:107A9000029A06D104941868C16804918068049021
:107AA0000498186E00207055B75405B0F0BDC0465C
:107AB000140100201800002001070000B0B588B0B4
:107AC0000546474903F0D3FE0446464904F03AFB15
:107AD00000280AD02046FAF7B9F900280DD0012174
:107AE000284603F067FF404804E00121284603F0E0
:107AF00061FF45A003F0B8FF70E0002506950595ED
:107B0000049503952046FAF7FFF9059503210291A4
:107B100001902046FAF7CEF901A9FAF79FFC01215E
:107B20000805324A13680343136012680240079243
:107B300007982F488268D20709D1C2682D4B13409D
:107B4000C36002692C4B1A40D218521C02614A05CC
:107B5000C3681343C3604B0304681C42FCD003603A
:107B6000C368C3688368DB070BD1C368C368234C51
:107B70001C40C460C368134203D0826AF0231343DD
:107B8000836202698A4302614A070369934303617E
:107B900042690723134343614269702313434361DE
:107BA000426804239A434260426808239A43426031
:107BB0008268134B13400A079A188260826A0F2367
:107BC0009A438262090242698A43426181680D4A8E
:107BD0000A40511C81600168C907FCD008B0B0BDE3
:107BE000B0E3000881E10008F3E000084010024023
:107BF00000240140C73FFFFFFFFFFF3F3CC2FEFFE5
:107C0000E8FFFF6FE8FFFF7F5B6572726F725D20B8
:107C10006E6F74206D6174636820616463207069A5
:107C20006E2E000070B50446EC4903F020FE861C61
:107C3000FBF71AFA0546314604F0F8FA06465549AC
:107C400004F043FA002801D0012678E0524930467A
:107C500004F03BFA002801D0504E70E05049304605
:107C600004F033FA002801D04E4E68E04E49304609
:107C700004F02BFA002801D04C4E60E04C4930460D
:107C800004F023FA002801D04A4E58E04A49304611
:107C900004F01BFA002801D0484E50E04849304615
:107CA00004F013FA002801D0464E48E04649304619
:107CB00004F00BFA002801D0444E40E0444930461D
:107CC00004F003FA002801D0424E38E04249304621
:107CD00004F0FBF9002801D0404E30E04049304626
:107CE00004F0F3F9002801D03E4E28E03E4930462A
:107CF00004F0EBF9002801D03C4E20E03C4930462E
:107D000004F0E3F9002801D03A4E18E03A49304631
:107D100004F0DBF9002801D0384E10E03849304635
:107D200004F0D3F9002801D0364E08E03649304639
:107D300004F0CBF9002801D1064600E0334E284676
:107D400003F000F93248816A0F229143B20E0A43D0
:107D50008262310242698A43426181682D4A0A4047
:107D6000111D816001684907FCD5006C80B2F9F7EC
:107D7000B5F92949F9F702F97321C905F9F7FEF8B0
:107D8000F9F754FA02460B462449204603F01CFE3C
:107D900070BDC0461FE100082FE10008020000048A
:107DA00035E100080400000838E100080800000C74
:107DB0003FE100081000001042E10008200000141C
:107DC00046E10008400000184AE100088000001C5D
:107DD0004EE100080001002052E1000800020024EA
:107DE00012E100080004002823E100080008002C2C
:107DF00031E100080010003037E1000800200034B5
:107E00003AE100080040003841E100080080003CF1
:107E100000240140E8FFFF7F3333534075E300083F
:107E200070B504461C4903F022FD06461B49204656
:107E300003F01DFD3046FAF73DF80546002806D14F
:107E40000121204603F0B6FD154803F00DFE304633
:107E5000FAF75AF8002806D10121204603F0AAFDBE
:107E6000104803F001FE0B20000728180A21C84122
:107E7000052810D8C1B22F22CA40D1070BD08000EC
:107E800009A109580E4A13680B4313600DA1085845
:107E900011680140116070BDB0E3000851E20008B4
:107EA000F3E00008D7E00008010000000200000035
:107EB0000400000008000000010000002000000095
:107EC00024100240FEFFFFFFFDFFFFFFFBFFFFFF4F
:107ED000F7FFFFFFFEFFFFFFDFFFFFFFF0B587B0FB
:107EE0000546894903F0C3FC06468849284603F045
:107EF000BEFC07463046F9F7A9FF002807D001214C
:107F0000284603F057FD824803F0AEFD3CE03046C2
:107F1000F9F7D0FF0446002806D10121284603F0D6
:107F200049FD7B4803F0A0FD3046F9F7EDFF06461A
:107F3000002806D10121284603F03CFD754803F0D6
:107F400093FDA662384602F0B9FF07460F4928465E
:107F500003F08DFC05460E4904F0B7F8002801D067
:107F6000012006E00B49284604F0AFF8411E884185
:107F7000400000210691049105900297019603911B
:107F800001A92046FAF76AFA07B0F0BD86E30008B7
:107F9000DAE30008C8E3000870B504465A4903F064
:107FA00066FC0646F9F786FF0546002806D1012142
:107FB000204603F0FFFC564803F056FD3046F9F723
:107FC000A3FF0646002806D10121204603F0F2FC5B
:107FD000504803F049FDAE6170BDC046B0E30008F3
:107FE00070B50446484903F042FC0646F9F762FFC3
:107FF0000546002806D10121204603F0DBFC444859
:1080000003F032FD3046F9F77FFF0646002806D11F
:108010000121204603F0CEFC3E4803F025FDAE6270
:1080200070BDC04670B50446374903F020FC0646D3
:10803000F9F740FF0546002806D10121204603F04C
:10804000B9FC334803F010FD3046F9F75DFF0646F2
:10805000002806D10121204603F0ACFC2D4803F096
:1080600003FD28693040801B4242424102490023FF
:10807000204603F0BDFC70BDC4E20008F0B587B037
:108080000446214903F0F3FB07462049204603F04C
:10809000EEFB05463846F9F7D9FE002807D0012146
:1080A000204603F087FC1A4803F0DEFC29E038463E
:1080B000F9F700FF0646002806D10121204603F00B
:1080C00079FC134803F0D0FC3846F9F71DFF07464A
:1080D000002806D10121204603F06CFC0D4803F076
:1080E000C3FCB762284602F0E9FE00210691059123
:1080F0000491022103910290019701A93046FAF7F9
:10810000ADF907B0F0BDC046B0E3000851E2000889
:10811000F3E00008D7E00008F0B58DB00446F1495F
:1081200003F02CFBF8F71CFE0290EF49204603F009
:1081300043FB0746ED490194204603F098FB0646B1
:10814000FBF7C8FD04463046FBF722FD0546E8482C
:1081500084420ED0E748844215D0E748844215D0C7
:10816000E648844215D0E648844216D10120C00278
:1081700011E0E448016802221143016000681040E8
:108180000790079809E00120C00304E00120800463
:1081900001E001204004FAF753F93846F8F793FF5D
:1081A0000146D948F8F727FFF9F707F8401E21687C
:1081B000D64BD34A944215D0CD4A944201D1702275
:1081C0009143CB4A94420FD0CA4A94420CD0CB4A36
:1081D000944209D0C84A944206D02160E0623F210F
:1081E000A16209E07022914319402160E0623F21C1
:1081F000A162C3498C4205D0BF498C4202D0BF491D
:108200008C4201D100212163616901221143616126
:1082100021688023039399432160012D06950596DB
:10822000049210D0042D10D0102D10D0402D10D05D
:1082300011028D420FD091028D420ED011038D425A
:108240000DD1062111E000210FE011460DE00221C1
:108250000BE0032109E0042107E0052105E01104FA
:108260008D4201D0082100E00721A94A525C264630
:1082700018369359A74D695C08273D468D401D432C
:108280009551F8F72BFF01460298F8F777FEF8F7BB
:1082900094FF049A1104069B8B4226D0042B1146AE
:1082A00000D1BAE0102B46D0402B5AD001210A024F
:1082B000934258D08A0293426BD00A0393426AD009
:1082C000012B32D1226A8A432262216A6368A26941
:1082D0008B4DAC4205D0884DAC4202D0874DAC42AC
:1082E00079D18A4D2B400F2576E08B4D7335216A6D
:1082F00029402162216A636D814A944205D07E4AF9
:10830000944202D07D4A944202D162682A4062605F
:10831000814AD21C134060221A436265A26DA06597
:108320000320000481432162069B01200004834254
:108330004FD0394671E0216A102291432162216AAF
:108340006368A2696E4DAC4205D06B4DAC4202D061
:108350006A4DAC424AD1F025A9430325AD02AB4397
:1083600046E0032159E0216A91432162216A636852
:10837000E269634DAC4205D05F4DAC4202D05F4D27
:10838000AC4240D103252D03AB430F252D02A94359
:108390003BE0052141E0236A93432362226A65683A
:1083A000E369574FBC4205D0534FBC4202D0534FF4
:1083B000BC4201D189038D43656058490B400321BC
:1083C0004D035B19E36120640803824322620621A6
:1083D00023E0072121E00325A94363604E4B1A40A7
:1083E0006032A26160632162002116E03025A9435A
:1083F00063604A4B1A4003235B03D218A261A06357
:108400002162022109E0414D29406360424B1A403C
:108410006032E261E063216204213E48405C042551
:108420002A4682403A48405C8159914381516068B4
:108430007021884360600F2000056168814361609E
:10844000A06803998843A0602D48844202D0049814
:10845000400300E03248059E60643046FBF73AFC7A
:1084600000281ED007463046F9F7F0FC30460026BB
:108470000A96F9F749FD0B96022107AA43C21E4846
:10848000874217D01B48874213D01D48874211D01E
:108490001A488742069D10D0154887420CD1012109
:1084A0000BE020A003F0E0FA0121019803F082FA2A
:1084B00015E02946069D00E031460C910598F9F734
:1084C000F9FC07A9F9F7CAFF206A2843206220684F
:1084D000012108432060C803616C014361640DB051
:1084E000F0BDC04688E50008DDE30008B0E3000801
:1084F00000040040002000400048014000440140CA
:10850000002C01403C10024000247449FFFCFFFF96
:108510000CD5000815D500088CFFFEFFFF8CFFFE70
:10852000002000025B6572726F725D3A20696E69AD
:10853000742050574D20706F7274206661696C64AE
:108540002E000000F8B504462F4903F017F90090FB
:108550000E462B49204603F08AF90546FBF7BAFB85
:1085600000280ED007462846FBF712FB0446009869
:108570003146F8F7F5FB024638462146FBF71AFC70
:10858000F8BD224803F070FA0121204603F012FAE8
:10859000F8BDC046F8B50446184903F00DF9074682
:1085A0001749204603F063F90546FBF793FB0028C3
:1085B0001BD006463846F8F786FD01461148F8F705
:1085C0001AFDF8F7FAFD401EF0620F49204603F04D
:1085D000D5F8F8F7C5FB04462846FBF7D9FA01465B
:1085E00030462246FBF7E6FBF8BD084803F03CFAAC
:1085F0000121204603F0DEF9F8BDC046DDE30008A6
:10860000B0E300080024744988E50008B2E00008DF
:1086100080B5D949CA6B0249002303F0E9F980BD4E
:1086200036E3000880B50846024902F0F1F9F9F78F
:108630001DFD80BD7AE40008B0B50846064902F089
:10864000E7F904460025A54205DA7D20C000F9F7C8
:108650000DFD6D1CF7E7B0BD81E40008F0B591B0E9
:108660000446404903F0A8F806463F49204603F077
:10867000A3F8F1B2012903D0022903D13C4902E059
:108680003A4900E00021002962D0394CA14266D16C
:1086900001267304029037498A681A438A608A68FF
:1086A0001A40099209980868304308600868304009
:1086B00009900896002507950695059502200190DA
:1086C000049004200390099805200007009003AF50
:1086D0003946F9F7C3FE0896079506950595019862
:1086E00004900820039000983946F9F7B7FE224815
:1086F0000168FF229143016030072049086010950E
:108700000F950C200E900D950C950B9502980A90E4
:10871000099509A92046F9F701FF0920C0026168FF
:1087200081436160A0682A218843A06020683043AB
:108730002060E0698002FCD5E0694002F9D520683C
:10874000202101432160300221680143216006E0BD
:108750000121204603F02EF909A003F085F911B09C
:10876000F0BDC0462CE200089DE200080038014040
:1087700000440040341002401CE400E000E100E04E
:108780005B6572726F725D20555341525420696E61
:108790006974206661696C642E000000F0B585B0D4
:1087A00006463C4903F008F8C0B2BC4D012804D08D
:1087B000022805D11235B74F04E01135B64F01E05C
:1087C00000252F461E490396304602F0F5FF064667
:1087D000FAF74AFC0446384600F040F9074604958B
:1087E0002878864200DB064602942046314602F095
:1087F000DDF8054639463246F8F735FB1149039C4A
:1088000020462A4603F01EF920460E4903F02FF8B1
:108810000190B919049D2878821B3846F8F723FB8C
:108820002878801B2870C0B200213954029802F0C9
:1088300089FB05492046019A03F004F905B0F0BD13
:1088400001E30008C4E20008F6E1000870B505463F
:108850000F4903F00CF804460E49284602F0ACFF1D
:10886000C0B2012803D0022803D18A4D02E0E54DB1
:1088700000E0002500262046F7F768FC864206D275
:10888000A05DA862E8694006FCD5761CF3E770BDE0
:10889000FFE100082CE2000870470000F8B5364CF4
:1088A000E06B401CE0632079012807D1207B002881
:1088B00004D1606BE16B081AC82800D2F8BD2F48BC
:1088C0002F4DA847216B2FA003F010FE01F0B6FA40
:1088D00033A0A8470026A665E66566703F20C5025E
:1088E0003648006880022840354FC119E06A01F01F
:1088F00067FE324C206880022840C11931A001F087
:108900005FFE01F069FE0120C0072F490A6802439B
:108910000A6008682DA01A4FB84724683248B84743
:108920003248B847A002284025494418671E20460F
:10893000F7F70CFC86420FD2A05D0A2808D1B85D7B
:108940000D2801D10A2003E00D2002F0ADFAA05D50
:1089500002F0AAFA761CEAE72448094DA847224CFF
:108960002046A84722A0A84728A0A8470348A84710
:108970002046A847F9F778FC18000020F4DD00082D
:10898000BDCF00085B696E666F5D3A2072656369F2
:10899000657665642073697A653A2025640D0A005E
:1089A0005B696E666F5D3A2057726974696E672005
:1089B000666C6173682E2E2E200D0000E075FF1F7F
:1089C00000F0FF070A0A0000142002405B204F4B12
:1089D000205D3A20577269746520666C6173682067
:1089E0006F6B21200D0000001BDE0008BDDD0008BC
:1089F0005B204F4B205D3A2050726F6772616D694A
:108A00006E67206F6B21200D000000005B696E66B1
:108A10006F5D3A2052657374617274696E672E2EB1
:108A20002E200D000120C006014908607047C04695
:108A300008ED00E010B504460748214603F045FB69
:108A4000002801D0002004E01F21204603F015FB80
:108A5000401C80B210BDC046D8D0000810B5904967
:108A6000884207D0674988420DD1674C206C0028A6
:108A70000BD010BD644C606C0028FAD1402003F08C
:108A80009BF8606410BD002010BD402003F094F8F6
:108A9000206410BD00440040003801401800002050
:108AA000F0B593B05748C169890600D49EE0416A89
:108AB000554C2170217801F029F9A08A402804D36F
:108AC00052484021F8F7F6F9002021784F4D2954FB
:108AD000461CA68220780A2800D087E003A84021FF
:108AE000F8F7E8F920790028029653D1474D284637
:108AF000F7F72CFB811E0026002904D46A5C0A2AA1
:108B000003D0491EF7E7324600E04A1CA918821A32
:108B1000019203AF3846F8F7A6F90198C0194670DC
:108B20003B49384603F00EFB06460127002805D0D6
:108B30002772206B401C03F03FF8E06203A835A1C8
:108B400003F0C3FA00281FD00220207300202072F7
:108B5000EFF3108072B6206D02F098FD3F20C00246
:108B60002F490968890208407F2292020A40101AA0
:108B70002C49401803F03AFDE062002838D062B674
:108B800029A004F01BFA01E0002E35D02771E06B1C
:108B900003AD029EA078002801D10120A070207BA7
:108BA000002801D0401E2073E06B6063276BA76331
:108BB000B9192163E66A207A012808D10191491C7C
:108BC000304604F00BFA0646E062019C00E00C46D9
:108BD000F0192946029AF8F746F9002030550A4C58
:108BE0000020A08209484021F8F764F913B0F0BDD5
:108BF00019A004F0E3F9FEE720790128029EC9D00C
:108C0000EEE7C04600380140180000207800002040
:108C100096DE0008696D706F72740D0A0000000026
:108C2000E075FF1FFF0F00005B696E666F5D2069D6
:108C30006E20646F776E6C6F6164206D6F64652C5D
:108C40002073656E6420707974686F6E20706C6537
:108C50006173652E0D0000005B6572726F725D209E
:108C60006E6F20656E6F75676820636F6465206244
:108C70007566662C20706C6561736520726573651E
:108C80007420746865206465766963652E0D000044
:108C900080B50348416AC9B201F038F880BDC046CA
:108CA00000440040F8B50C46C969471804250BA6D6
:108CB000781942787F2111407A5D0F2A09D8062958
:108CC00007D1A16840884018314603F0FEF900281A
:108CD00001D12D1DECE72846F8BDC0462D3100001E
:108CE00070B50A18121F095C09094B1C041F0020EB
:108CF000002C0CD415782D09AB4200D1401C012664
:108D00009657002E03D4121F241F8D42F0D8C0B2F4
:108D100070BD0000F0B58BB01C4604920291099022
:108D200000260A96194614310AAD284603F07EFA49
:108D3000014628222923284603F08DFA002800D175
:108D4000D2E0002C01D0A57900E002252A210446BA
:108D500003F0E4F905906748214603F0B6F90028CE
:108D6000069401D0002404E02C21204603F085F96C
:108D7000441C0F2D00D1641EE0B207900999486A87
:108D8000896AC969FFF7ACFF034628460D380228F7
:108D900007D30598002804D11198181A079988421A
:108DA00030D101950598002800D01C4603940AA8EC
:108DB000069903F03BFA0746002425460798A84287
:108DC0000BD02C21384603F0E1F906464B4903F05D
:108DD000B9F9002805D16D1CF0E7009408940794B8
:108DE0001DE0E843079940180890701C009001248A
:108DF0008D4212D2FAF740F907902C21069803F021
:108E0000C5F90CE010992C200322099C22543A4801
:108E1000079A01F03BFB002666E000200790049DC6
:108E20000998083009900398C6B2002E2BD00898F4
:108E3000864200DC0024200605D00AA82D4903F054
:108E4000F5F9074607E02C21069803F09FF907463D
:108E50003A2103F09BF9099803F076F8394601F0BE
:108E60002FFD0746E0B2012807D10798394602F0E6
:108E700073F8384601F01CFC03E02846394601F03F
:108E800097FE761ED1E70598002821D0FAF7F4F86E
:108E900004460798002815D002F088F80646471EB9
:108EA0000025B5420ADA0798394602F073F8014600
:108EB000204602F051F87F1E6D1CF2E7079802F081
:108EC00041F8049D132228460099234601F0E0FE54
:108ED00001980F2807D10AA0029901F01AFD014656
:108EE000284601F065FE039E0AA801F09CF8F0B246
:108EF0000BB0F0BDD8D00008FCDC000825E000086D
:108F000073656C6600000000F0B587B09F79032F91
:108F100001D1002543E014460D460646187B597BD7
:108F200009020818997BDA7B120251180904081803
:108F30000690987C0590D87C0490187C0390587C0F
:108F400002900021284602F035FD0D2F01D00C2F94
:108F500004D121682846069A904713E0029800023F
:108F60000399401804990902059A891809040B18F5
:108F7000D8690699081A80B272680090284621467E
:108F800001F0F2F82068074901F05CFD01F077FB81
:108F90000546206800680449002201F0FBFC2846D1
:108FA00007B0F0BDC1E30008299F0008F8B50446EA
:108FB0002D300090257E0834002D38D0204602F058
:108FC000C3FF0746002803D0BE79032E01D104E079
:108FD000022600980078002804D0384601F068FB8B
:108FE0006D1EE9E730460938FD21084203D1F968D2
:108FF0000FA001F04BFA301F0328EED87844007917
:109000004000874401040A10F96812A008E0FA68D9
:109010003B690EA001F03AFADFE739460C310A4805
:1090200001F034FAD9E7384601F0C6FBD5E7F8BDC0
:109030003C6F626A65637420617420307825303239
:10904000783E0D0A000000003DDD000825660D0A8F
:109050000000000025640D0A0000000001480862BD
:10906000002070471AFCFFFFBCB514465C21104677
:1090700003F054F8002812D000200190009001ADB8
:109080006A462846214600F067FF0146009ABC4820
:1090900001F0BAFB0446284600F0C5FF08E0204670
:1090A000F7F754F80246B648214601F0ADFB0446F6
:1090B0002046BCBD80B5134608460122194600F083
:1090C000E9FD002080BD00000148086200207047D3
:1090D0001BFCFFFF10B5084600241146224600F095
:1090E000D9FD204610BD80B50868114602F014FC79
:1090F000002080BD80B50868114602F0FBFA00230D
:10910000002804D08079821E501E824100E01A4659
:109110009B4801F0CCFB80BD70B514460D46086835
:1091200006681149304601F0A9FC002815D0014617
:10913000934801F0FAFB0D4901F012FC214601F0C1
:109140000FFC044602460C3228680068064901F00C
:10915000B6FD204601F0ACFA04E003493046224651
:1091600001F0ADFD002070BD81E3000829E000089A
:10917000F8B514460F460546114602F08AFB002852
:1091800033D11B4E306D214602F083FB0146306D1A
:10919000002908D0214602F0ADFA024628462146B1
:1091A00002F0EBFB21E0214602F0B6FA002815D0D0
:1091B0000646104801F0EEFA214601F081FB092134
:1091C00001F0C2FB0146286801F0F2FC2846214666
:1091D00002F036FB314602F043FE06E02C2003216C
:1091E000395405A0214601F051F90020F8BDC046D0
:1091F00018000020852E00084D6F64756C654E6F59
:1092000074466F756E644572726F723A204E6F20AD
:109210006D6F64756C65206E616D656420272573C4
:10922000270D0A00F0B585B001920C460646486A43
:10923000896AC969455C2046083002F085FEC76826
:1092400001F036FA1E4803900F202840303002A962
:1092500088711C4802907A427A413068002301F0FC
:109260000DFD002F03D1019801F07EFD206200204A
:1092700005B0F0BD10B510460C4601F075FD20623A
:10928000002010BD00207047BCB515460C46496A49
:10929000A26AD269895C0A4A01920F220A403032DE
:1092A00069468A71074A0092006801F0B1FB0143E8
:1092B00003D1284601F058FD20620020BCBDC04605
:1092C000736530005F5F656CB0B50868114602F0E9
:1092D00011FA044601F0D3F905460921204601F0B0
:1092E00033FB0B21284601F02FFB2846B0BD0020A0
:1092F00070470000F0B585B0144650784F2809D06B
:10930000782803D06F2805D0582826D10021204680
:109310000A4619E002AD302028702046F6F716FF05
:10932000871E0026082F314601D80B21091A019506
:109330006D1CE819F7F7BEFDA11C28463A46F7F761
:1093400092FD019831463246F6F72EFF0246C317CA
:109350000B4801F0ACFA05B0F0BD2E21204602F01A
:10936000DDFE002808D0204603F0E9FD024604484F
:109370000B4601F093FAEEE7204601F0F5FCE5E735
:10938000D8D00008F0B589B005920D46486A896AC0
:10939000C969FFF7A5FC012800950AD0022844D12D
:1093A0000835284602F0D0FD0446284602F0CCFDE0
:1093B00006E00835284602F0C7FD044601F098FA99
:1093C00002270021002807913D4601D085790146FA
:1093D000002C01D0A7790794281F46424641042D4E
:1093E000069106D1CC682046F7F76DFE049004255F
:1093F0000DE00024052D049409D10699C868096977
:10940000F7F7AEFC0490F7F7BFFE04460525052FDD
:10941000029414D00020042F1CD10798C06801903A
:10942000F7F751FE0390042716E000200225029072
:10943000069007902F460646019004900BE007998E
:10944000C8680969F7F78CFC0390F7F79DFE019057
:10945000052701E001900390DF48059C214602F0BA
:1094600034FE002816D0062D21D1062F1FD1002052
:10947000089006990C31079A0C3208AD284602F084
:10948000B1FE0146D54801F050FA0446284600F0E6
:10949000CAFD70E0D248214602F017FE00280FD026
:1094A000012F02981BD1002E26D0424247E0052D05
:1094B00001D0052F1CD104980399F7F706FD52E05F
:1094C000C848214602F001FE00281FD0052D01D01A
:1094D000052F31D104980399F7F750FD43E0052D8E
:1094E00001D0052F0FD104980399F7F73FFD3AE01B
:1094F000029801990A1822E0052D04D10120C10724
:10950000049848402FE00199421A18E0B6A021467D
:1095100002F0DBFD002817D00024039D28462146D9
:10952000F7F7C3FD00281AD02C200121009A11540E
:10953000AEA001F0CFFB1EE0029A01984243D31780
:10954000A64801F0B4F915E0B1A0214602F0BDFD36
:10955000002819D004980399F7F78BFD1EE00498B2
:109560002946F7F748FDF7F761FE02469B480B4690
:1095700001F094F90446069801F09AF8079801F072
:1095800097F8204609B0F0BDA2A0214602F09DFD4B
:10959000002809D004980399F7F779FD0246401E88
:1095A00082418E480023CCE79B48214602F08DFD86
:1095B000002807D002980199F7F704F9CB178748DC
:1095C0000A46BEE795A0214602F07FFD00280ED096
:1095D0007F20C1050024049D0198844205DA2846B5
:1095E000F7F7CCFC0146641CF6E70846BBE78CA005
:1095F000214602F06AFD002806D002980199F7F78B
:10960000E1F80246C3179BE78648214602F05DFD5C
:10961000002805D184A0214602F057FD00284ED035
:10962000BD420BD1072D13D0062D3AD106980C3030
:1096300007990C3102F049FD04466CE00120C0435B
:10964000A91F0024814266D3B91F8142EAD262E099
:10965000069A107B517B09020818917BD27B12027B
:10966000511809040818079B197B5A7B12025118DC
:109670009A7BDB7B1B029A18120451180024884243
:1096800049D107991031069A1032002842D04B1C5C
:10969000551C401E097812788A4219462A46F4D091
:1096A00039E004980399F7F761FC0146F7F766FC87
:1096B0005E49F7F7DEFC0446401E84412BE05CA0C7
:1096C000214602F002FD002806D0049D2846039E94
:1096D0003146F7F7DCFC0BE056A0059902F0F5FCEB
:1096E000002824D0049D2846039E3146F7F7C1FC8C
:1096F000044628463146F7F739FC0146F7F73EFCA9
:109700004A49F7F7B6FC0443601E844133480023FE
:10971000224616E701244348059902F0D6FC0028AA
:1097200001D0E2B23DE7E0B24242424139E742A015
:10973000059902F0CAFC002803D00298019A024061
:10974000FDE63EA0059902F0C0FC002803D0029877
:10975000019A0243F3E63AA0059902F0B6FC00280C
:1097600002D00198C243EAE636A0059902F0ADFCAA
:10977000002803D0029A01980241E0E632A0059940
:1097800002F0A3FC002803D0029A01988240D6E69A
:109790002E48059902F099FC002807D00199481E2F
:1097A0008141029A501E82410A40FAE628480599F2
:1097B00002F08BFC002804D0029A01980243501E4C
:1097C000EEE62448059902F080FC002801D00198BB
:1097D000AAE70024CFE6C04627E00008D8D000085A
:1097E0002BE0000825E000082F0000005A65726F8A
:1097F0004469766973696F6E4572726F723A20645C
:1098000069766973696F6E206279207A65726F007C
:109810003C0000003E0000009EDE00082A2A0000F6
:109820002F2F000060E10008213D0000BD37863584
:109830003E3D00003C3D0000260000007C00000092
:109840007E0000003E3E00003C3C000063DE00085D
:109850007EDE00088FDE0008F0B58DB004920F4662
:109860000846083002F070FB0446002801D0A679B3
:1098700000E002263868039005682849284601F070
:109880001AF900282DD0019602942449284601F0A7
:10989000F5F80546E548294601F047F8064605A8CB
:1098A0002021F7F707FB00960C3600242C212846D0
:1098B00002F0E3FB84420DDC05A82C22314602F0C5
:1098C0006FFC049902F001FC002801D07868039035
:1098D000641CEBE7009800F0EBFE38680568029C1A
:1098E000019E1E49284601F0E6F80028039F04D097
:1098F0001A49284601F0B9F807460B2E03D1092171
:10990000204601F021F800253846049922462B46CE
:1099100000F0F6FB28460DB0F0BDC04681E300081C
:10992000B0B515460C460BA1104602F0CEFB014621
:109930002068002903D0F44901F0EEFF08E0294631
:1099400001F07EFF024620680068EF4901F0ACF9A3
:109950000020B0BD246F726967696E0047E400089B
:10996000B0B514460D4618A1104602F0AEFB002813
:1099700003D017480122002308E016A1204602F078
:10998000A4FB002805D012480022134600F08FFFE8
:10999000B0BD2868214601F0ADFE00F070FE002841
:1099A00000D0B0BD6868214601F0A4FE00F067FE5B
:1099B0000028F6D12C20012129548348214600F0AB
:1099C00065FD0020B0BDC046547275650000000002
:1099D000D8D0000846616C736500000010B50C46D5
:1099E000064808620846083002F0AEFA01462068D0
:1099F000006801F013FE002010BDC04619FCFFFFF7
:109A0000F0B58BB015460E46074600240A94664909
:109A1000104602F05AFB002804D00836304602F007
:109A200093FA08E06149284602F04FFB002809D06C
:109A30005F4800F0B9FE04460AA800F0F4FA204698
:109A40000BB0F0BD3846294601F0B0FE07460028AD
:109A500006D13068294601F0A9FE0746002822D029
:109A60003846294601F0C0FE002805D17068294615
:109A700001F0BAFE00287FD00997074680790328B5
:109A80007BD0F9F7AFF80890026800950194304652
:109A9000099D29463B46FFF73DF92C21715C0029C1
:109AA0000AD0089D75E02C200121315447A0294699
:109AB00000F0ECFC0024BFE7059030462C30069007
:109AC00030462946089D2A4607973B46FFF71CFA71
:109AD0000446002834D0A0790B2831D10921204632
:109AE00000F032FFE0683349039001F07DFE074645
:109AF000F9F778F80146002F1CD004910498026809
:109B00002C48009005980190304603993B46FFF79A
:109B100001F904990698007800280BD13046039982
:109B2000049A3B46FFF7F0F90499002802D000F0B0
:109B3000BFFD0499084601F0A9FD384600F0B8FDC4
:109B40002E461DA1099D284601F091FE002801D056
:109B500001F0C0F81B49284601F09BFE002808D000
:109B60001849284601F028FE002802D00620069950
:109B70000870079F35460CE000272C200221315445
:109B80001148294600F082FC0024002F254600D110
:109B900052E7384600F08CFD002D00D14CE72846F6
:109BA00001F074FD48E7C046D8D0000824E300085F
:109BB00061300008EDE100085F5F7379734F7574E1
:109BC0000000000036E20008D6DC00084572726F23
:109BD000723A206D6574686F642027257327206EA4
:109BE0006F20666F756E642E0D0A0000BCB51446BA
:109BF0005C21104602F092FA002810D0002001905B
:109C000001AD6A462846214600F0A6F901460748FC
:109C100000F08BFE0446284600F005FA04E00348F5
:109C2000214600F082FE04462046BCBDD8D0000884
:109C3000BFF34F8F084809490160BFF34F8F00BF42
:109C4000FDE7C046BFF34F8F034804490160BFF3EF
:109C50004F8F00BFFDE7C0460CED00E00400FA05A1
:109C600010B5044604A101F0A7FD014303D005A1EE
:109C7000204601F069FE10BD69735F7065726F6404
:109C800000000000706C6174666F726D47657454FB
:109C900069636B00F0B587B004920591426A816AEE
:109CA0000391CD690192575D0F26374000680690F9
:109CB00004681549204600F0FEFE0290002804D0FA
:109CC0001149204600F0D1FE069001984219781CF7
:109CD00001215156002903D511783140884201D025
:109CE000121DF5E7039800900498002801D00E2378
:109CF00000E010230298002800D03346069805990A
:109D000000F02AF807B0F0BD47E40008B0B50C46F3
:109D1000774D0F49884201D0002101E029461231D8
:109D20000C4A904201D00D4600E01135FEF796FE38
:109D30002978445429783F2904D3411C4022F7F75D
:109D400092F8B0BD491C297000224254B0BDC046F3
:109D50000044004000380140F0B589B003930492FC
:109D60000D4605900846F6F7F1F9064600200290E8
:109D7000069006AC2046314600F018FE0746202229
:109D8000294602F08BF92046314600F00FFE0546C9
:109D90002822394602F0A7F90598294601F006FD68
:109DA00000283ED001900E9800902E21284602F007
:109DB000DDF90446029808903846F6F7C7F90146DF
:109DC00008A800F0F3FD054605942046F6F7BEF915
:109DD00006463846F6F7BAF9864207D2BC5D0598C2
:109DE000F6F7B4F9281A8455761CF2E72846F6F7F8
:109DF000ADF906460098079005980399049A00F07B
:109E000081FD07A9042200F015FC721C294600F010
:109E100011FC01460198006800F0CAFE08A800F095
:109E200002F906A800F0FFF809B0F0BD0021802972
:109E300003D000224254491CF9E77047FEB525A023
:109E400003F0BCF82A4D00222A622A4801680292D7
:109E5000009201923F20C0028A0210407F218902B5
:109E60001140254E3268002A06D532460C3A234B63
:109E70001360234B13603268224A8018C70A481EB9
:109E8000C40AE01B401C6F62A862287C00281DD118
:109E900001202874F7F7B4FF002815D1FD00A74270
:109EA0000DD83068F82188432843174908433060AB
:109EB000F7F7A6FF002802D108357F1CEFE73068CE
:109EC0000221884330600A4D009828740FA003F0E7
:109ED00075F8FEBD5B696E666F5D3A2065726973E9
:109EE000696E6720666C6173682E2E2E200D00004F
:109EF00018000020E075FF1F142002402301674571
:109F0000AB89EFCD00F0FFFF020001005B204F4B5B
:109F1000205D3A2065726973696E6720666C6173B3
:109F200068206F6B21200D0080B5002805D0817955
:109F3000132902D1C06801F005F8002080BD80B56A
:109F4000002807D0024680790C2803D10846114624
:109F500000F014FE002080BDFEB5009206461CA253
:109F60001C4B1D4CA04701461CA21D4B3046A04770
:109F700001461CA21C4B3046A0470546F6F7E6F802
:109F80000146304600F012FD0646002427462846CA
:109F9000F6F7DCF8874217D2E85D5C2810D17A1911
:109FA000517878290CD101A8002101710F4B019340
:109FB00092788270FF1CEA5DC2700A46F6F7F4F8E8
:109FC00030557F1C641CE2E7009804603046FEBDFB
:109FD0005C6E0000BBDD0008F1C300085C7200008D
:109FE0001BDE00085C74000099DB0008307830301C
:109FF00070B50C4605460846F6F7A8F82968401CD7
:10A0000086B208462146324600F014FB28602046FE
:10A01000314600F02DFA70BD80B50846042100F0ED
:10A0200027FA80BD704710B50068002804D0046886
:10A0300000F03EFB2046F8E710BD0000F0B59BB0F5
:10A0400015460E4604460846F6F780F8421C0AA854
:10A050003146F6F708FF02A82021F6F72BFF2E2144
:10A06000304602F00AF8401B471C00200090C54310
:10A0700001976D1CBD423EDA02A80AA92E2202F009
:10A080008FF8002C36D0266802A9304600F00AFD71
:10A090000A2824D102A9304600F0E7FC00261A96CF
:10A0A000002817D001F054FB064601F01FFF01F015
:10A0B00023FC3046114901F047FC206802AF092219
:10A0C0003946334600F0E4FD20463946019F01F051
:10A0D000BCFB06461AA8FFF7A6FF344608E009387D
:10A0E000FD21084206D102A9304600F0BEFC04461C
:10A0F000002CBED1009C20461BB0F0BDEDE1000855
:10A10000F8B51E4615460F4601F050FB002813D047
:10A1100004462E21384602F029F80746002E03D0C7
:10A12000284600F0ACFA05462846394600F0C8FB40
:10A130000146206800F03CFDF8BD000070B50C46FB
:10A14000054607A001F0C1FF002801D0012605E067
:10A15000002628462146324600F010F9304670BDF0
:10A160006578697428290000F0B599B01D460590FE
:10A17000588B06900E9201910D910DAE3446083425
:10A180001C212046F6F796FE00200390B085179517
:10A190001E9816900494204601F0BDFE2C360796BA
:10A1A00016990698814200DBC3E06648814200D1DF
:10A1B000BFE01798C2698F1801210C9179560029C8
:10A1C0000FD50DAE3046FEF7F1FE03983083079EA3
:10A1D00030800F980C30119010980C3012907978D4
:10A1E00017987A88806882184806C00D56490B581F
:10A1F0000DA905989847002803D00146049801F05E
:10A20000C5FE1598514988424E495CD000280DD0B2
:10A210004F4988420DD04F49884211D11799169E57
:10A220003046FEF73FFD3018079E00E01698011DEE
:10A2300049E01799169E3046FEF734FD811941E03A
:10A240001799CE69169A935D0F24089423400993B9
:10A2500001280B9202961BDB92190A92498B002669
:10A26000042213460B9AD2188A4213DA0A9AD21899
:10A270000C9C1457002C06D51278089C2240099C8F
:10A28000A24200D8761C1A1D74B2A042E9DC01E09B
:10A29000039B1E46002813D50B99029A8918091FA3
:10A2A000CA180C9C1457002C06D51278089C224022
:10A2B000099CA24200D1761E1B1F72B29042EFDBB6
:10A2C0000B981918079E00201590179A528B9142EF
:10A2D00000DB1C4916913178002900D160E77170CC
:10A2E0003C1D06460220C0432156301D241F002974
:10A2F000F7D5002E01D01AA000E017A000F0C6F894
:10A3000060787F307F2101401529164903D8400627
:10A31000C00D154909586388A868C21813A000F039
:10A32000B5F8361F241DBC42E3D90020079E3070CB
:10A3300036E70DA8FEF73AFE049801F0E3FD019818
:10A3400019B0F0BD6179FEFF20D5000819FCFFFFB0
:10A350001BFCFFFF1AFCFFFF202D3E200000000029
:10A3600020202000A9E1000874D4000825732025CE
:10A370007320090928232564290D0A00F0B58FB040
:10A380000446084610435CD00E460192002002901D
:10A390000E9004A82821F6F78DFD27682A4D38462F
:10A3A000294600F088FB0028039015D02749304645
:10A3B00001F0C8FE002806D12549304601F0C2FE52
:10A3C00004AD002813D00EA83A22314601F0E5FF73
:10A3D0000546206804AA01E004AA3846294600F090
:10A3E0002DFC2068294600F02DFB05461035002E77
:10A3F0000CD0284600F08EFC28463146F9F7C8FDFF
:10A4000000280DD113A000F041F811E0019908884F
:10A410006883891CE961425AEA804018801CA86060
:10A42000029800902046214622462B46FFF79CFECC
:10A430000398002802D004A800F05EFC0EA8FFF7E5
:10A44000F2FD0FB0F0BDC04640E2000869DE000832
:10A4500088DE00085B6572726F725D3A2053796E18
:10A46000746178206572726F722E0D0A0000000010
:10A4700080B50A463F21C902624B1B689B020B4014
:10A480006149591800F0C2F880BDC04683B0C0B51C
:10A4900003AF0EC703A9009102F038F888BC01BCD5
:10A4A00003B0004782B07CB50D460692079306AB19
:10A4B000019301210C0221462A4602F031F8FF28BF
:10A4C0000ADD05460648074EB04707A02946B047B3
:10A4D0000DA02146B047FEE77CBC01BC02B000479E
:10A4E00030DC00088DA40008496E666F3A20627562
:10A4F00066662073697A6520726571756573743A52
:10A500002025640D0A000000496E666F3A206275CE
:10A5100066662073697A65206E6F773A2025640D30
:10A520000A000000F0B591B0039302920C4601902E
:10A530000025109504AF3846F9F78DFC38462146C2
:10A54000F9F7F6FC3846F9F76BFCED4F2E4604A8F8
:10A550008088864226D204A8F9F790FC099C0298CC
:10A56000214601F0B2FD002808D0280605D110A828
:10A570003946224601F036FE07466D1C03982146F7
:10A5800001F0A3FD002800D06D1E280605D110A8FB
:10A590003946224601F026FE07460E9800F0D2FC0E
:10A5A000761CD4E704A8F9F74BFC0198394601F072
:10A5B0003DFE044610A8FFF736FD204611B0F0BD61
:10A5C000B0B50C460546F5F7C1FD024628462146C2
:10A5D00000F01CF8B0BD0000F8B51024094D0A4E7B
:10A5E000134F002C0CD03F20C00229688902014083
:10A5F0008819396A002200F005FC3862641EF0E711
:10A60000F8BDC046E075FF1F00F0FF07F8B514461F
:10A610000D460646064F002C08D03278396A284687
:10A6200000F0F0FB3862641E761CF4E7F8BDC0460B
:10A6300018000020FEB50192029104468688B018E9
:10A6400082B20020014600F005F90546A17900F02C
:10A650007BF9A168284600F03DF92F460C372146CA
:10A660000C3138463246F6F7FEFBB8190299019ACA
:10A67000F6F7F9FB204600F01BF82846FEBD10B5A2
:10A68000002813D004468079092802D1E06801F03F
:10A6900033F9A28821460C31002000F0DBF8A168D4
:10A6A00000F018F9A17900F04FF910BD002010BD9D
:10A6B00010B5044600F004F8204600F027F810BD5D
:10A6C00010B500281BD0817909290ED0122916D186
:10A6D000017B427B12025118827BC37B1B029A18BA
:10A6E000120451181030884710BDC468204601F08C
:10A6F000F3F80549204601F05FF8002800DD10BDA1
:10A70000204600F0C3FF10BDAFE4000880B500286C
:10A7100004D081880C3189B201F03AFA80BD7CB551
:10A720001C4615460E4600F0FDFB00210091314607
:10A730002A46234600F001F87CBDF8B51C4600927D
:10A740000F46054618460C3001F036FA064685607D
:10A75000848006983060B771002C01D1214603E057
:10A76000601E03218843011D37460C373846F6F733
:10A77000A1FB0099002903D038462246F6F773FB67
:10A780003046F8BD80B583B2814803210022FFF72F
:10A79000C6FF80BD80B500F063FF02467C480B21F8
:10A7A00000F0B0F880BDC04680B5024678480A2166
:10A7B00000F0A8F880BDC046F8B50446807B009044
:10A7C000E67B277B657B0CA0FFF760FE2802C019A3
:10A7D0003102009A891809040E18103407A5002EBA
:10A7E00006D021782846FFF751FE761E641CF6E756
:10A7F00004A0FFF74BFEF8BD622700005C7825300F
:10A8000032780000270D0A00F8B51446009105467D
:10A81000571D3846FFF7B6FF294600F051F80721CB
:10A8200000F092F8064605460C3528463946F6F7FC
:10A8300041FB0099200EF073200CB073200A707356
:10A840003473002903D0281D2246F6F70CFB30464E
:10A85000F8BD0000BCB513460A4600280AD00446DD
:10A86000808898420CD120460C3011461A46F6F7E3
:10A87000FAFA10E046480321FFF751FF04460AE0C8
:10A88000A179A06825680095FFF757FF0546204687
:10A89000FFF73CFF2C462046BCBDC046E0B5019307
:10A8A000009205216A460823FFF739FF8CBDE0B509
:10A8B0000193009204216A460823FFF730FF8CBD04
:10A8C00010B50446084600F02DFB0146204600F076
:10A8D00001F810BDE0B5002801D081608CBD0022D8
:10A8E00000920323084619461346FFF726FF8CBD46
:10A8F00080B52748022100221346FFF710FF80BDD4
:10A90000D8D00008E0B5019201AA0423FFF707FFA1
:10A910008CBDB0B50C460546084600F0EDFF092198
:10A9200028462246FFF7EEFFB0BDB0B50C460546FF
:10A930000846F5F70BFC401C83B206212846224648
:10A94000FFF7EDFEB0BD000080B5002801D0817199
:10A9500080BDFD4800221346FFF7E1FE80BDC046E2
:10A960007CB50A4604460020019021460C3101AD19
:10A97000284601F037FC0146F348FFF7D6FF0646AC
:10A980002046FFF795FE2846FFF74DFB30467CBD7D
:10A99000D8D0000870B5002807D014460D460668C8
:10A9A0002146A847002E3046F9D170BD10B50446A7
:10A9B000481CFFF7E7FE2168206001600C3010BDE5
:10A9C00080B5002805D000F03DF8002800D01030F8
:10A9D00080BD002080BD000080B500F033F8024645
:10A9E00009490A48002A0DD09379042B04D0052B7D
:10A9F00008D1D068116980BDD0681169F6F775FB80
:10AA0000F6F714FC80BDC04664CDCDC1000080FFC8
:10AA100080B500F017F802460020C1430848002A1C
:10AA20000CD09379052B04D0042B07D1D068116981
:10AA300080BDD0681169F6F7D5FBC11780BDC0464F
:10AA4000013665C410B50446084600F06BFA0146AD
:10AA5000206800F001F810BD002804D082688A4206
:10AA600002D00068F8E70020704780B5FFF7EAFFE2
:10AA7000002801D0C06880BD002080BD80B50028BE
:10AA800005D0FFF7DFFF002800D00C3080BD00208C
:10AA900080BD000080B50249FFF7D4FF0C3080BDB7
:10AAA000EBE2000880B5FFF7CDFF002801D08079E8
:10AAB00080BD022080BD80B5FFF7C4FF411E8841E4
:10AAC00080BD00007FB504462749FFF7EBFF002556
:10AAD0000295411E052914D87944097949008F440B
:10AAE0003C101002203720492046FFF791FF034613
:10AAF0000020039003AE20211D4A304601F0FBFBED
:10AB00001DE00938FD21084227D117492046FFF7EB
:10AB1000ACFF002103910090019103AE202115A20A
:10AB20000AE011492046FFF757FF002203920090E8
:10AB3000019103AE20210D4A304601F0DCFB0146B5
:10AB4000204600F0C5F905463046FFF76CFA04E0F0
:10AB500005492046FFF792FF054602A8FFF763FA72
:10AB6000284604B070BDC04675E30008B9E200088D
:10AB70001CE200083078256C6C78000010B50029C4
:10AB800015D0002203461B688B4204D0002B1A46C6
:10AB9000F9D1002108E00B6804688C4200D1036001
:10ABA000002A00D0104603600846FFF781FD10BD63
:10ABB000FEB50C4607461B4D0029294600D0A1686A
:10ABC0003E683046FFF748FF002812D00197002C5E
:10ABD000284600D0A068029400243746002E29465B
:10ABE00000D0B968814207D03E68002E3C46F4D1BF
:10ABF00014E03C602660FEBD3846FFF761FD029D13
:10AC0000AA8829460C313846FFF724FEA979FFF7B8
:10AC10009BFE002C019900D0214608600298FFF7A6
:10AC200075FDFEBD3F420F0010B504460846FFF714
:10AC300035FE01462046FFF7BBFF10BD7CB504463C
:10AC40000D480190002A16D016460D46002001A995
:10AC50000422FFF7FFFD28223146FFF7EBFC12210B
:10AC6000FFF772FE2946FFF72BFE002803D00146AE
:10AC70002046FFF79DFF7CBDF9AC000810B50446E7
:10AC80000846FFF714FE01462046FFF791FF10BD6E
:10AC900010B50446084611461A46FFF733FE014632
:10ACA0002046FFF785FF10BD10B504460846114643
:10ACB000FFF72FFE01462046FFF77AFF10BD10B5C3
:10ACC000044608461146FFF730FE01462046FFF7CE
:10ACD0006FFF10BD10B5002806D004461A48214663
:10ACE00001F0F3F9002800D010BD02482146FFF71B
:10ACF000CDFB10BD3DDD000810B5044600680028FE
:10AD000001D0FFF7D5FC6069002801D0FFF7D0FC27
:10AD100010BD0000B0B504460B480146FFF705FE24
:10AD200020600025A5800C30A060F5F70FFAE560E3
:10AD30002561401CE080FFF7DBFD60610C30A56100
:10AD4000E06125626562B0BDD8D00008E0B500239F
:10AD500000930D23FFF700F88CBDE0B500230093AE
:10AD60000C23FEF7F9FF8CBD10B50446F5F7EEF99C
:10AD700080B22118491E0978002912D00C490D4AC9
:10AD80005118421E0020002A06D0A35CDB00CB58DD
:10AD9000C0185031521EF6E722782D2A03D14042C6
:10ADA00010BD002010BDD2008958401810BDC0460B
:10ADB00080FEFFFF80D5000870B50D4604460020D8
:10ADC000A07208340E4E642D0FD364212846F5F787
:10ADD000D9FC6321C943414349194900715A217083
:10ADE000090A6170A41E0546EDE76800305A20701C
:10ADF000000A60700A2D00D2641C204670BDC04657
:10AE00008EE50008FEB50646254F7878082840D321
:10AE10000192029100257D705F202C460146583931
:10AE200008D4395C2A0251182A0E23029C18401EAD
:10AE30000D46F3E7EFF3108072B6387C00281ED180
:10AE4000012000903874F6F7DBFF002802D00020C4
:10AE5000387414E002988019124A1168009E314338
:10AE600011600560BFF36F8F4460F6F7C9FF0D4AAC
:10AE70001168B143116000213974002802D000200C
:10AE80007870FEE7EFF3108072B678780299083197
:10AE9000019A3B1858241A55401C78700846FEBD8C
:10AEA0001800002014200240C2B20349CA600A6898
:10AEB0005206FCD57047C0461C38014080B5034996
:10AEC00001F003F9411E884180BDC0460AE5000833
:10AED000F8B50E460546002000906C4680210CA275
:10AEE0000F4B204601F007FA07462046314601F095
:10AEF0009DF9024628463946FFF7E1FE28463946C5
:10AF0000FFF7BCFD05462046FFF78DF82846F8BD43
:10AF10005B7072696E74427566665D257300000031
:10AF200075E30008014606480A78002A04D0212368
:10AF300043439818491CF7E70121C9078843704724
:10AF40000515000010B50446FFF76DF804212046F2
:10AF500000F01EFE10BD0000FEB50F460446164967
:10AF6000FFF756FD064668463146FFF725FF0546C2
:10AF70003846FFF784FB07462946FFF7A1FC204629
:10AF80003946FFF715FE721CD31720460A49FFF712
:10AF900075FEFEBD1FB5044601A8FFF70DFF014673
:10AFA0002046FFF74FFD04B010BD000080B50249F8
:10AFB000FFF72EFD80BDC046D6E3000810B50C4655
:10AFC0000348FFF7E7FB0146204600F027FB10BDD2
:10AFD0009931000810B50C460348FFF7DBFB01462A
:10AFE000204600F01BFB10BD6132000810B50C4676
:10AFF0000348FFF7CFFB0146204600F00FFB10BDD2
:10B000006134000810B50C460348FFF7C3FB014646
:10B01000204600F003FB10BD9534000810B50C4627
:10B020000348FFF7B7FB0146204600F0F7FA10BDD2
:10B030001135000810B50C460348FFF7ABFB01467D
:10B04000204600F0EBFA10BDD936000810B50C46CA
:10B050000348FFF79FFB0146204600F0DFFA10BDD2
:10B06000E136000810B50C460348FFF793FB014694
:10B07000204600F0D3FA10BD7537000810B50C4615
:10B080000348FFF787FB0146204600F0C7FA10BDD2
:10B090009D38000810B50C460348FFF77BFB0146BE
:10B0A000204600F0BBFA10BDE539000898B0012534
:10B0B0002902974A10680691084310600020079003
:10B0C000F7F7A6F8934E00280FD1306C0121084302
:10B0D0003064306C0840109010980807F16B014301
:10B0E000F163F16B01401091109803200890400229
:10B0F000894C2168814368020590081820608748C0
:10B100004168062048438649F5F73CFB801C0995B9
:10B11000AF026169394201D0401EFAD1B0683821CE
:10B120000840F268102803D1089B1A40032A01D076
:10B13000082843D13068B068084010282ED1F06844
:10B14000784A0240F01C82425FD1F648006840070E
:10B15000800F5ED0072004900003B2680390024382
:10B16000B2600F221202B3689343B3603268920157
:10B1700000D4B8E0B268022002900243052001909A
:10B180008243B260E94DEB6BEB4AB4680C40102C83
:10B1900054D0EC6BE41A9442F7D9A4E0099B18064A
:10B1A0003268824332605806E04AD36B3468044206
:10B1B00013D0D46BE41A022CF8D926E009980004C5
:10B1C000326802433260D948C26B33689B03B2D401
:10B1D000C36B9B1A642BF8D917E0F368D44C1C405E
:10B1E000F31C2343F360D34B5B1C34681C43346073
:10B1F000099B1B07F4681C43F460D36B346804425A
:10B20000A3D1D46BE41A022CF8D9EFF3108072B6F4
:10B21000FEE7C44B186802220243052082431A60ED
:10B22000C248C26BC44BBF4C246807252540022D81
:10B2300090D0C46BA41A9C42F5D954E0B948036875
:10B24000049C2340032B12D3B6480368029C23437B
:10B25000019CA3430360EB6BB2480468049804406C
:10B26000022C04D0EC6BE41A9442F5D93BE0B268AE
:10B2700003988243B260B0688006400F1ED0B26867
:10B280000A40AE48082A1ED0B2680A40102A2ED1C1
:10B29000F168089A1140032900D0A948F1684906CD
:10B2A000490F491CF5F76EFAF1684904490E484305
:10B2B000F168490F491CF5F765FA04E0306880042D
:10B2C000410F9F48C840984AB1688B093C211940FA
:10B2D0009C4B5B581F211940C84050601068F6F71E
:10B2E00097FF002820D0EFF3108072B6FEE7B06819
:10B2F000084020288C4A02D10998C003E4E7B068CE
:10B300000840182801D00798DEE77D200002DBE71F
:10B310000020024000100240007000401000002099
:10B3200040420F00737F3EE0706D0899884370655E
:10B3300020200890F7F7E4F8099C2046F7F7E0F89A
:10B34000A003316C01433164316C014010911098BD
:10B35000706B20437063706B204010900F94002638
:10B360000E960D960C9602980B9005980A901098E0
:10B370000198000707900AAD2946F7F76FF80F9478
:10B380000E960D960C9602980B900A9707982946F0
:10B39000F7F764F8FF2000066B490A6882430A60E9
:10B3A000E0066A490860179616960C2015901496C8
:10B3B00013961296E120400211901096644D10A948
:10B3C0002846F7F7ABF8049A5007A9688143A960AB
:10B3D0005006A9688143A9606007296881432960F4
:10B3E0000920C002696881436960A8682A218843EE
:10B3F000A860286820432860E8698002FCD5E869D5
:10B400004002F9D5286808990843286028680699F9
:10B41000084328604FA001F0D1FD3F20C1025548EC
:10B420000068800208405449425CFF2A03D0451856
:10B430006878FF285AD15C4801F0C0FD5B485C4C3D
:10B44000A0475C48A0475C48A0475C48A0475CA078
:10B45000A0476048A04760A0A04700F00BF9054650
:10B4600032480565B84F684A2846394600F025FA43
:10B470002846394600F0E4F90446644D4035F007AB
:10B4800021D12E46614F20372046394600F001FA7F
:10B49000002804D1204639465D4A00F00EFA2046C5
:10B4A000394600F0CDF905465A493A4600F0CAFA45
:10B4B0002846A6493546324600F0AEFA0B20400138
:10B4C0003518099EDBE71948046D5349204600F002
:10B4D00023F9002803D00146204600F0C1FC13499F
:10B4E000086DC86100F0A2FBFEF7A2FB00F0C2F8F5
:10B4F0000E490865C861297869290DD11FA001F09E
:10B500005DFD28482946FFF710FA084988610C308C
:10B5100000F0DEFAFEF78CFB294600F0A1FC0348A0
:10B52000C069DFE700200240100000201800002062
:10B530008C80C11FFFFFFF0088130000001BB700B5
:10B540000024F400CCD4000818E400E000E100E09E
:10B55000003801405B696E666F5D3A2073746D332D
:10B560003220686172647761726520696E69742047
:10B570006F6B0D00E075FF1F00F0FF075B696E66E3
:10B580006F5D3A20636F6D70696C696E67207468D7
:10B590006520707974686F6E207363726970742EA1
:10B5A0002E2E0D00D8D00008D7DD0008F7DB0008EC
:10B5B0008DA400089BDB0008C5DB0008B0DB000899
:10B5C00053544D333247303D3D76312E332E320DBC
:10B5D0000A000000DDDB00083D3D3D3D3D3D3D3DB9
:10B5E0003D3D3D3D3D3D3D3D3D3D3D3D3D3D3D3D8B
:10B5F0003D3D3D3D3D3D3D3D3D3D3D3D3D3D3D3D7B
:10B600003D3D3D0D0A0000009F2B0008F8D90008C1
:10B610006130000884E20008ABE3000810B50A4678
:10B6200004460E491046FFF74BF901462046FFF746
:10B63000BFFA10BD80B50949FFF7F6FA80BDC046D4
:10B6400080B50A46CB170549FFF718FB80BDC046F9
:10B6500080B50A460149FFF732FB80BDC1E300080F
:10B6600010B500F075F8044600F046F9204600F0E9
:10B670003DFC10BD80B50348FFF7F2FF02490865A5
:10B6800080BDC046A92B000818000020F0B587B087
:10B6900004460CA100F0A8F800280DD001900BA0E2
:10B6A00002A90A46E8C8E8C200781070204600F0F7
:10B6B000D7FB0198FEF7FCFF204600F011F807B019
:10B6C000F0BDC0465F5F64656C5F5F000400008290
:10B6D00001000900005F5F64656C5F5F00000000AF
:10B6E00010B504460068FFF72DFC0421204600F049
:10B6F0004FFA10BDB0B50C4600F058F8002809D03C
:10B7000005462E21204600F031FD01462868FFF74E
:10B7100099F9B0BD0020B0BD70B50D4606460A4986
:10B7200000F0B7F8002400280CD00749304600F09C
:10B730008CF8294600F084F8002803D0034900F073
:10B7400084F80446204670BD0EE2000848E2000876
:10B7500070B50646F7F788FC0446B04705463749FA
:10B76000324600F059F96B4900222846134600F092
:10B770003FF92046FFF7E6FB284670BDB0B50C4602
:10B7800000F014F8002809D005462E21204600F0CC
:10B79000EDFC01462868FFF71FF9B0BD01490248DA
:10B7A000B0BDC046FD3F8FC0A245B6F380B50122B3
:10B7B000FEF744FC80BD0000B0B50C46FFF7F6FF75
:10B7C00000280AD005462E21204600F0CFFC014675
:10B7D0002868FFF71DF9C117B0BD0020C14301481B
:10B7E000B0BDC046013665C470B50A4605462E2177
:10B7F000104600F0BBFC044628462146FFF77AFFBE
:10B80000002803D0FEF73BFF054614E00B4928460D
:10B8100000F01BF8002500280DD0FFF799FF002845
:10B8200009D006462146FFF765FFFEF728FF0546CB
:10B830003046FFF755FF284670BDC046FDE30008BF
:10B8400080B50022FEF7FAFB80BDB0B50C46FFF7CD
:10B85000ADFF002809D005462E21204600F086FCC9
:10B8600001462868FFF701F9B0BD0020B0BDB0B5B2
:10B870000C46FFF79BFF002809D005462E212046E5
:10B8800000F074FC01462868FFF7F8F8B0BD00200E
:10B89000B0BDB0B50C46FFF789FF00280BD00546B8
:10B8A0002E21204600F062FC01462868FFF7CAF806
:10B8B000411E8841B0BD0120B0BDB0B50C46054663
:10B8C0001046FEF771FF2146FEF7FAFF0146286891
:10B8D000FFF76EF9B0BD0000B0B504460D4D294626
:10B8E000FFF76AFF0B460021421E8B412046294686
:10B8F00000F07EF8B0BDC046B0B50446054D2946FF
:10B90000FFF75AFF0023421C4B412046294600F016
:10B910006FF8B0BDAFE40008B0B50C46FFF746FFC6
:10B9200000280FD005462E21204600F01FFC0146BE
:10B930002C682046FFF786F801462046FFF71EF9DF
:10B940000020B0BD0120B0BDF8B50446FFF74CFFA4
:10B95000002811D0817B0091C67B077B457BFEF7D9
:10B96000A7FE2802C0193102009A891809040A1892
:10B9700002D0002120469047F8BD80B50123FEF794
:10B98000BFFB80BDF8B51C4615460E46FFF70EFFFF
:10B9900000280DD007462E21304600F0E7FB3E6818
:10B9A00029462246FEF730FF01463046FFF700F9F0
:10B9B000F8BD000080B50A460249002300F018F8DF
:10B9C00080BDC04636E20008F8B51C4615460E4656
:10B9D000FFF7ECFE00280AD007462E21304600F083
:10B9E000C5FB014638682A462346FFF71DF9F8BD16
:10B9F000F8B51C4615460E46FFF7D8FE00280AD0BB
:10BA000007462E21304600F0B1FB014638682A4631
:10BA10002346FFF733F9F8BD70B514460D46FFF71E
:10BA2000C5FE00280DD006462E21284600F09EFBBC
:10BA3000356808212246FEF765FF01462846FFF7D4
:10BA4000B7F870BD70B514460D46FFF7AFFE00287D
:10BA500009D006462E21284600F088FB01463068B2
:10BA60002246FFF72CF970BD80B5FFF733F980BD92
:10BA7000B0B588B004460CA1FFF7B6FE002810D080
:10BA8000FEF716FE01AD0AA11B222846F5F7EBF9D9
:10BA90002046294600F0E4F90C492046FFF7E7FE6E
:10BAA00000E0002008B0B0BD5F5F7374725F5F009C
:10BAB000080000820100000409000F00005F5F73AE
:10BAC00074725F5F005F5F72657300004FE400088F
:10BAD000F0B58FB00546009005AC20212046F5F763
:10BAE000E9F9FEF7ABF923492046884700260E9670
:10BAF000099621480D90214A204629469047E08822
:10BB000004A901910880608B03AD28801C49204660
:10BB1000884702271B4A2846394690472046154940
:10BB200088470E96099618480D902046009D294694
:10BB3000124A904720461249884701983946114ACF
:10BB4000904702A8067001210E4A904720460949F5
:10BB500088470E96099608480D900C480890204694
:10BB60002946064A9047204605498847FEF734FD96
:10BB70000FB0F0BD15AD000825A00008913F0008EA
:10BB8000F9AC000871A4000819A00008F19F000892
:10BB9000B0B50C46AB4DA978012900D1FEE7EFF313
:10BBA000108172B600F0F0FCE01C0321884362B6FD
:10BBB000A96C081AA864B0BD80B50E498A78012A1C
:10BBC00000D1FEE7C01C032290438A6C12188A64DD
:10BBD000CB6C934200D2CA64EFF3108172B600F0CE
:10BBE00005FD62B6002800D080BD03A0FEF74EFC24
:10BBF000FEE7C046180000205B6572726F725D3A06
:10BC0000204E6F206865617020737061636521202C
:10BC1000506C656173652072657365742074686526
:10BC2000206465766963652E0D0A0000F0B589B061
:10BC30007E49049103900568002004A90422FEF7C0
:10BC400009FE1121FEF780FE7949FEF739FE002832
:10BC500003D001462846FEF7ABFF7649764A039C9F
:10BC60002046FFF7D9FE2068FEF714FF0546734F04
:10BC700000268023204639463246FFF783FE70496E
:10BC800020463246009633463E46FFF7B1FE28680E
:10BC9000FEF7FCFB6B4908780028FCD00D78009F6C
:10BCA0000F7008A80570039C2068FEF7F3FE019052
:10BCB00020466049FFF7C9FD029020463146FFF754
:10BCC00075FD00280AD03146064608462E2100F0B0
:10BCD0004DFA01463068FEF773FE0746039858494F
:10BCE000FFF76AFD064658A02946FEF7CFFB7F2DD9
:10BCF00005D00A2D11D00D2D0FD0082D3FD138467B
:10BD0000F4F724FA002840D0054653A0FEF7BEFB06
:10BD1000E819401E0024047081E04CA0FEF7B6FB39
:10BD2000002E37D000200190079006A90A20087045
:10BD30000122384600F08EF9039D2846444C2146E6
:10BD4000FFF795FD014607AE30463A4600F04AFA45
:10BD5000024628462146FFF775FE3046FEF763F996
:10BD60003878092801D0202846D13A48FEF78EFBC2
:10BD70003846FEF75BF8314E3249019C51E008A984
:10BD80000122384600F066F902E03448FEF77EFBF7
:10BD9000002444E03878002821D03846F4F7D6F95A
:10BDA000C019401E00783A2819D101260024039DAD
:10BDB0002846234932462346FFF71AFE05A90A20E2
:10BDC00008703846324600F045F9284620493A4680
:10BDD000FFF738FE3846FEF729F81E481DE00398A5
:10BDE0003946029A9047044601980068FEF74EFBD8
:10BDF0003846FEF71BF812E00022039C204610494B
:10BE00001346FFF7F5FD20461149FFF730FD0146C7
:10BE10002046029A904704460448FEF737FB074E37
:10BE20000849012C00D036E709B0F0BD22DE000839
:10BE3000EBE2000879E300083DA10008E3E2000816
:10BE400014E2000818000020256300000D0A00001D
:10BE5000CDE200081DDE0008200800009CDE00087E
:10BE600080B50A460021FEF789FA80BD1FB5044659
:10BE70001C49FFF7A1FC411E01A8FEF79DFF0146EA
:10BE80002046FFF7DDFC04B010BDC046B0B5044647
:10BE9000144900252A462B46FFF7AAFD03492046F0
:10BEA0002A462B46FFF7A4FDB0BDC0468BE3000831
:10BEB000FEB504460B49FFF77FFC06460F46684671
:10BEC0003146FEF779FF05460023721C7B41204670
:10BED0000449FFF78DFD044A20462946FFF7EDFC93
:10BEE000FEBDC046D6E300086130000810B5044628
:10BEF000026810680249FEF74DFD204610BDC0469D
:10BF00003F9F000810B504460068FEF7D1FB60684B
:10BF1000FEF7CEFB10BD70B50446012005020026D9
:10BF2000304631462A46FEF795FC206040223046D6
:10BF30003146FEF78FFC6561268221680C31606016
:10BF40000C30A160E06070BDB0B5018A002400290A
:10BF500019D0491E0182C1688A1EC2600122D243E3
:10BF6000895E8268511A81600846FEF788FB0028C6
:10BF700009D0054680790938FD21084202D1E868D8
:10BF8000FFF7AAFC2C462046B0BD0000F8B50D46D0
:10BF90000446008A401C20828E880C368879093835
:10BFA000FD21084202D1E868FFF7A6FCE068811C89
:10BFB000E160B1B2CE1C03218E4306802168A068E7
:10BFC000411A8F190C3F61698F4209D90A480B4DFC
:10BFD000A8470BA03946A847616911A0A847FEE70A
:10BFE00029463246F4F73FFFA0688019A060284632
:10BFF000FEF75EFBF8BDC04686DC00088DA4000895
:10C00000496E666F3A20737461636B2073697A6559
:10C0100020726571756573743A2025640D0A0000FD
:10C02000496E666F3A20737461636B2073697A6539
:10C03000206E6F773A2025640D0A000010B5044683
:10C040000348FEF772FC01462046FFF79FFF10BD34
:10C05000D8D0000870B515460E460446F4F776F8B9
:10C0600021180022AA4203DAB35C8B54521CF9E770
:10C07000401900212154204670BDB0B50C4605463C
:10C08000F4F764F801460020002906D02A78A2427D
:10C0900000D1401C491E6D1CF6E7B0BDF8B5154631
:10C0A0000E460090002427463046F4F74FF88742AA
:10C0B00007D2F05DA84202D000990855641C7F1C8D
:10C0C000F2E7002100980155F8BD80B50246002036
:10C0D000002A07D0002905D01046F4F73EF80146A3
:10C0E0004042484180BD70B514460E46054608469C
:10C0F000F4F72CF80021814207DA725CA24204D0E6
:10C100006A54725C491CA242F5D1284670BD0021D8
:10C11000425C491C0A2AFBD1481E7047B0B50C4648
:10C120000546F4F713F800220146904204D0AB5CB8
:10C13000521CA342F9D1511E814201D30020B0BD4F
:10C140000120B0BDB0B505460020002D0DD00C4635
:10C1500000290AD02046F3F7F9FF02462846214677
:10C16000F4F712F8014640424841B0BDB0B50D4663
:10C170000446F3F7EBFF611E012805DB0A5C401E55
:10C18000AA42F9D12018441C2046B0BD10B504467F
:10C19000FFF7ECFFA04202D0411E00220A7010BD42
:10C1A000F8B516460D4600900846F3F7CFFF00217C
:10C1B0000A460F460B4683420EDAEC5C002F04D091
:10C1C0006C54491C01275B1CF5E7B442FAD0009F70
:10C1D000BC54521C0027F6E70023009883546B548C
:10C1E000F8BD0000F8B514460D4606460E4F084649
:10C1F000B8473946074620468847C1193046FEF7FA
:10C20000D5FB064628460849884702463046294657
:10C21000F4F729FE20460449884702463046214665
:10C22000FFF718FFF8BDC0464D010008B0B50C4639
:10C2300005460846F3F78AFF01462846FEF7B6FB97
:10C2400005462046F3F782FF024628462146F4F7CA
:10C250000AFE2846B0BDFEB51E4617460D460446EA
:10C260000846F3F773FF01462046FEF79FFB029056
:10C270002846F3F76BFF00242146814204DA6A5C0A
:10C28000BA4203D0491CF8E7019101E001910C4644
:10C290006A1E074631463B46012F04DBD65C5F1E13
:10C2A0008E42F8D100E00746661CAD1900220299C3
:10C2B000B418BC4203DAAC5C8C54521CF8E700257D
:10C2C000029CA554002B00DC02950199814200DB01
:10C2D00002950298FEBD70B514460D460646084606
:10C2E000F3F734FF01463046FEF760FB294622464D
:10C2F000FFF7D4FE70BD81B078B514460D460593A6
:10C3000005A900912946FEF751FB0646009B2946E8
:10C31000224600F005F9304678BC02BC01B008475F
:10C32000F0B58FB00D4604460846F3F70FFF410005
:10C330002046FEF73BFB029003AE3046F7F78BFD3D
:10C3400030462946F7F7F4FD3046F7F769FD002639
:10C35000314603A88088814217D2019103A8F7F7DC
:10C360008DFD0027089DBCB22846F3F7EFFEA042E2
:10C3700005D9285D029988557F1C761CF3E70D9836
:10C38000FEF7E0FD0199491CE3E703A8F7F758FD24
:10C390000021029881550FB0F0BD70B514460D46CE
:10C3A00006460846F3F7D2FE0021884204D06A5CB4
:10C3B000A24202D0491CF8E70146814200D301465F
:10C3C0003046FEF7F3FA29462246FFF78CFE70BD91
:10C3D00070B514460D4606460846F3F7B7FE01460B
:10C3E0003046FEF7E3FA29462246FFF7D9FE70BD34
:10C3F000F0B587B01E4614460F4601900846114618
:10C40000F3F783FE002826D0054600200290002F77
:10C4100048D0002C46D02046F3F798FE069000281E
:10C4200040D0002E00D1214E00970594049630464E
:10C43000F3F78CFE0146069803910F1A002601249B
:10C44000002D0AD0069828180599F3F75EFE0546D8
:10C45000E419761EF4E7029724E0009F3846F3F7CC
:10C4600075FE01190198FEF7A1FA05460290002E0B
:10C4700014D038460599F3F748FE04463946C71BE1
:10C4800028463A46F3F755FEE8190499F3F773FE88
:10C490000699671803994518761CE8E72846394637
:10C4A000F3F769FE029807B0F0BDC046D8D0000887
:10C4B00010B50C460C49FFF77FF97D22D20000230E
:10C4C000F4F7ABFC01485043A06010BD40420F00A0
:10C4D00010B50C460449FFF76FF97D22D200002306
:10C4E000F4F79BFC03C410BD36E300080FB410B58D
:10C4F00003A9044B044A029800F07AF910BC08BC66
:10C5000004B01847A9AE00080000002010B5024B87
:10C51000024A00F06DF910BDA9AE0008000000202D
:10C520007CB51D4616460C0001D0611E00E00021BE
:10C5300001910090054B6A462946304600F058F9B3
:10C54000002C02D0009A002111707CBD29CF000878
:10C550002021020C01D010211046020A01D0104601
:10C560000839020901D01046091F820801D010467F
:10C57000891E420801D0881E7047081A70470000C3
:10C58000004870470C00002030B5002805D0164C3C
:10C59000021F20680023014605E0084630BD904296
:10C5A00003D8034640680028F9D1002B00D0596811
:10C5B000002B0AD01C68D51AA54204D11268A41811
:10C5C0001A461C6002E05A6000E02260002807D092
:10C5D0001468851AA54203D105686419146040687F
:10C5E0005060184630BD000004000020F1B50E4C2C
:10C5F0000F480C4E001B0D4FC508ED0000221146E0
:10C60000009800F0B3FC002803D13068002801D066
:10C610000020F8BD3C600020256060600120306093
:10C62000ECE70000080000207C010020040000204E
:10C63000781B002001480068704700000C000020B3
:10C6400002E008C8121F08C1002AFAD170477047DB
:10C65000002001E001C1121F002AFBD17047000039
:10C6600001490860704700000C000020F0B51FB4BD
:10C6700086B00998089A030D0021024314D051484E
:10C68000514A1818504305141198012810981AD0CF
:10C69000281A401C00264D4F4D49009601910490E8
:10C6A000002812DA444211E01198012449A301281C
:10C6B00001D11098C1430698119A84600360C2604A
:10C6C00041600BB0F0BD4042E4E704462105002084
:10C6D0003F4A001C51410391029012E0E00707D04D
:10C6E00032463B4601990098F3F726FF01910090EE
:10C6F00032463B4610461946F3F71EFF06460F46E4
:10C700006410002CEAD10498039B0028029A09992E
:10C71000089806DAF3F710FF019B009AF3F70CFF75
:10C7200005E0F3F771FF019B009AF3F76DFF0446F4
:10C730000E460022284BF3F7FFFF03D80020C0432A
:10C74000014607E00022254B20463146F3F742FE22
:10C75000F3F7D2FF102409E0002C0ADB0A220023A1
:10C76000F3F75AFD079B30321A55641E02460A43FE
:10C77000F2D11122641C079B121B1C19119B012B67
:10C7800003D0012308430ED10AE0084304D011204E
:10C7900010900020119077E71098151A6D1E0BE08D
:10C7A0001098824202DD00236D1C03E0824201DA10
:10C7B00000236D1E002BEED0069811998260C16097
:10C7C00030C07EE701FCFFFF104D00000000144068
:10C7D0000000F03F300000000000F0430000E03FA8
:10C7E00030380A2801D2012070470020704700002D
:10C7F000FFB597B00646002518E2252877D100241A
:10C800002746FD49049400E00443761C3278012059
:10C81000203A90400842F7D130782A280ED00222E0
:10C82000307801463039092916D804990A2359432A
:10C83000303940181443761C0490F1E7189802C868
:10C8400004911890002904DA01204003044348426F
:10C85000049002200443761C30782E2814D1042042
:10C8600004437078761C2A2809D11898761C80C851
:10C87000189009E00A214F43303FC719761C3078E1
:10C88000014630390929F5D930786C2810D006DCFA
:10C890004C281AD068280ED06A2817D104E07428D2
:10C8A00013D07A2812D110E00120400504430CE097
:10C8B0000121090501E0032109050C43717881423A
:10C8C00003D1012000052418761C761C30781190C5
:10C8D00066280BD013DC58287DD009DC00287BD0DB
:10C8E0004528F6D04628F4D047281AD1A5E118E00B
:10C8F000632835D0642870D0652812D19DE1702856
:10C900006CD008DC6728F1D069287BD06E280DD068
:10C910006F2806D1BAE073282ED0752871D07828F8
:10C9200059D01A9A199990476D1C7EE16002400F08
:10C93000022809D003280DD00428189801680DD0CA
:10C940000D60001D189070E11898EA1701680D60DD
:10C950004A60F6E7189801680D80F2E70D70F0E77D
:10C9600018986A4601781172001D189000205072C4
:10C9700002A80090012005E0189802C81890002035
:10C980000091C04361070DD5002101E00199491CC8
:10C990000191B94212DA8142F8DB009A515C002918
:10C9A000F4D10BE0002101E00199491C0191814281
:10C9B000FADB019A0099895C0029F5D10199049864
:10C9C0001A9B471A21463846199A00F097FA01999E
:10C9D000401945180BE04FE02CE113E04EE00098C1
:10C9E00000990078491C00911A9A1999904701986A
:10C9F000401E0190401CF2D1214638461A9B199ADC
:10CA000010E137E00A200021009001916002410FFF
:10CA1000022907D0189A01CA1892C217944603290E
:10CA200008D00AE01898C01DC108C90005C91891AE
:10CA3000944607E000B2C2179446042902D140B2DE
:10CA4000C1178C4600226146944506DA0A46002149
:10CA5000404291418C462D2102E0210504D52B2135
:10CA60006A461173012103E0E10701D02021F7E7B5
:10CA7000029155E00A200AE0102008E01020009002
:10CA80000021042004430191082703E0082000212D
:10CA9000019100906002410F022907D0189A01CA43
:10CAA000189200229446032908D008E01898C01D67
:10CAB000C108C90005C91891944603E080B2042951
:10CAC00000D1C0B200210291210729D51199702906
:10CAD00006D0009A1021019B4A401A4305D00EE06F
:10CAE00040216A461173012108E06146014306D0E6
:10CAF00030216A4611731199517302210291009AF3
:10CB00000821019B4A401A430AD16146014301D1E1
:10CB1000610705D530216A46117301217F1E0291FC
:10CB20001199582904D035A10E910DA90D910DE050
:10CB300037A1F9E76146019B009AF3F76DFB0E9B65
:10CB40008C469B5C0D9A521E0D92137061460143F8
:10CB5000F0D10D9805A9081A20300190600703D57F
:10CB600001200004844300E001270198874201DD91
:10CB7000381A00E000200199009041180298091825
:10CB80000498401A0490E00306D421461A9B199A8F
:10CB9000049800F0B3F94519002706E003A81A9A93
:10CBA000C05D199990476D1C7F1C02988742F5DB88
:10CBB000E0030CD521461A9B199A049800F09EF9BF
:10CBC000451904E01A9A3020199990476D1C009974
:10CBD000481E00900029F5DC08E00D980D990078BA
:10CBE000491C0D911A9A199990476D1C0199481E7C
:10CBF00001900029F1DC63E1092801003031323372
:10CC00003435363738396162636465660000000088
:10CC10003031323334353637383941424344454672
:10CC20000000000000F05AF94519761C3078002801
:10CC300000D0E2E528461BB0F0BD600700D406270F
:10CC40001898C01DC108C90048680A680831C30F98
:10CC5000DB071891190001D09CA108E0210501D53E
:10CC60009BA104E0E10701D09AA100E09AA1430052
:10CC700011985B08109165280CD006DC452809D076
:10CC800046281DD0472841D141E0662818D06728A2
:10CC90003CD13CE00021112F01DB112000E0781C89
:10CCA0000191009008A911A8FFF7E0FC13990591E4
:10CCB0000021119A15927F1C12980197009150E063
:10CCC0000120C00703900120019008A9009711A836
:10CCD000FFF7CCFC139A149905920022119B009245
:10CCE00012981593059A0192002901D0104602E08E
:10CCF000791C40180190381A01D5019804E040428F
:10CD0000401E0090781C0190C01B029043E0012F50
:10CD100000DA01270021112F01DD112000E0384643
:10CD20000191009008A911A8FFF7A0FC13990591A3
:10CD3000119A0021129815920091019721070CD4A5
:10CD40000599B94201DB019900E00191012904DD57
:10CD5000159A491E515C302906D0B84201DA011DEE
:10CD600005DA0121029115E00199491EEDE700283D
:10CD700005DC0099411800910199091A03E0019A14
:10CD8000411C914200DD01910099401A401C029023
:10CD90000120C0070390200706D402990198814220
:10CDA00002DB0020C043029000206946C87707AF2D
:10CDB000012103980337C907884224D0022011902B
:10CDC0002B201290039800280CDA404203902D206B
:10CDD000129007E00A210398F3F7D4FC30317F1E4C
:10CDE000039039701199481E11900029F2DC0398C4
:10CDF0000028EFD1791E1298087030782021084061
:10CE00004530BF1E387006A8C01BC01D0390109887
:10CE10000078002800D00120019941180298C0171D
:10CE20000918039809180498401A401E0490E0035A
:10CE300006D421461A9B199A049800F05FF8451908
:10CE400010980078002803D01A9A199990476D1C01
:10CE5000E00324D521461A9B199A049800F04EF855
:10CE600045191CE00098002807DB009905988842C6
:10CE700003DD1598405C199901E0199930201A9A40
:10CE8000904700986D1C401C00900298401E029034
:10CE9000002804D11A9A2E20199990476D1C0199E7
:10CEA000481E01900029DDDC05E038781A9A7F1CC5
:10CEB000199990476D1C0399481E03900029F4DCD2
:10CEC00021461A9B199A0498ACE600002D00000038
:10CED0002B0000002000000000000000F8B5044610
:10CEE00000251E461746880404D405E03946202054
:10CEF000B0476D1C641EF9D52846F8BDFFB5044641
:10CF0000002581B01E46C80301D5302700E0202748
:10CF1000880404D505E038460399B0476D1C641EAB
:10CF2000F9D5284605B0F0BD4A68002A06D00A683F
:10CF3000531C0B6010704868401E4860704730B545
:10CF400083B00446FFF776FB0546002000900246BA
:10CF50000190012321466846F3F702FA2846FFF7BD
:10CF60007FFB0199009803B030BD0000F8B50B308D
:10CF7000C608F600104D19E02068B04215D3B04243
:10CF80000BD96368871B201D0093F3F76CFFA01972
:10CF9000009B07604360286004E060682860201DF3
:10CFA000F3F761FF201D2660F8BD251D2C68002CBD
:10CFB000E2D10020F8BD00000400002010B50446B6
:10CFC00001E0FDF771FF2078641C03490028F8D1C7
:10CFD0000A20FDF769FF10BD00000020F3B583B003
:10CFE00005001AD028680190284680380290C76F43
:10CFF00004983E1F864200D906462846FFF7C4FA29
:10D0000004460091324629460498FFF7AFFF019984
:10D01000002806D0016005B0F0BD0498FFF7E6FADD
:10D02000F9E729600299002CCF670AD021686218BD
:10D03000291F8A4202D9291B091F216000996160BA
:10D04000E9E7024A00991160E5E7000004000020CA
:10D05000004040404040404040404141414141400B
:10D0600040404040404040404040404040404040C0
:10D07000400502020202020202020202020202024F
:10D080000220202020202020202020020202020254
:10D0900002029090909090901010101010101010AC
:10D0A00010101010101010101010101002020202B8
:10D0B00002028888888888880808080808080808FC
:10D0C00008080808080808080808080802020202F8
:10D0D0004000000051D0000800000000280010832C
:10D0E000010000020B001081010000020B00108102
:10D0F000180000020B001085210000020B000085C3
:10D100002300000425002F0000706572696F645FC2
:10D110006D730063616C6C732E617070656E64007A
:10D1200066756E5F746F646F003000310069735F05
:10D13000706572696F6400001800108301000002BE
:10D140000600108113000002060010811C0000027E
:10D1500006002500007768656E0063616C6C732EB5
:10D16000617070656E640066756E5F7768656E00ED
:10D1700066756E5F746F646F00000000600200826D
:10D18000010000040D00008311000004160000855A
:10D190001B0000041D0020851B0020010D00100253
:10D1A000280000022E000004330000823700000433
:10D1B0004400000D44000007460011810D001105D8
:10D1C0001B000108480001074B00028E000011817E
:10D1D0001D0011051B000108480001074B001281CA
:10D1E0004D00120144002201440022054B001208A8
:10D1F000550012054B00020257000204160002857A
:10D200004B0002041D00018B4B0011011D00110594
:10D210004B000108480001074B0012811600120361
:10D2200061000208480002074B0013814D00130102
:10D2300044002301440023054B0013085500130547
:10D240004B00030257000304680003826800038553
:10D250001B0003041D00028B4B0012011600120379
:10D260006D000208480002074B0013814D001301B6
:10D2700044002301440023054B0013085500130507
:10D280004B000302570003046D00038546000304AE
:10D290001D00028B4B0012011600120372000208DF
:10D2A000480002074B0013814D0013014400230185
:10D2B000440023054B001308550013054B000302DF
:10D2C0005700030472000385460003041D00018B10
:10D2D0004B0011011D00110546000108480001071F
:10D2E0004B001281160012036D000208480002076D
:10D2F0004B0003826D0003074B0014814D001401A5
:10D3000044002401440024054B0014085500140572
:10D310004B0004025700040468000482680003857F
:10D320001B0003041D00028B4B00120116001203A8
:10D3300072000208480002074B0013814D001301E0
:10D3400044002301440023054B0013085500130536
:10D350004B00030257000304680003857C000304AC
:10D360001D00018B4B0011011D0011057C000108FF
:10D37000480001074B0012811600120372000208D8
:10D38000480002074B0013817E0023014D0023015A
:10D3900044003301440033054B00230855002305A6
:10D3A0004B00130257000308850003074B0004825B
:10D3B000680014814D001401440024017E00240102
:10D3C00072001408550014034D0004028700038501
:10D3D0001B0003041D0000868F00008C33009200A8
:10D3E000005F5F63616C6C732E6C656E006C656EC4
:10D3F000006E6F6E65006D6F6465003000696E666B
:10D400006F5F696E6465780072616E67650069744C
:10D410006572005F6C30005F6C302E5F5F6E657808
:10D42000745F5F00690032003D3D0031005F5F6363
:10D43000616C6C73002B005F5F736C6963655F5F89
:10D4400000616C7761797300746F646F0077686551
:10D450006E00706572696F645F6D730033005F5FAB
:10D460007469636B003E005F5F7365745F5F002DDE
:10D470003100000095E10008B1E10008BDE10008BD
:10D48000D9E10008A5E10008B9E10008E5E10008DC
:10D49000CDE1000891E10008C9E10008A1E1000820
:10D4A0009DE10008D1E1000899E10008ADE1000824
:10D4B00084E10008C1E10008E1E10008C5E10008DD
:10D4C000DDE10008D5E10008B5E10008000000003A
:10D4D000000000000000000000000000000000004C
:10D4E000000000000000000000000000010000003B
:10D4F000020000000300000004000000060000001D
:10D500000700000008000000090000000000000003
:10D510000404043C3C00000800000008000800006F
:10D52000EF92000861990008019A0008ED9B00083D
:10D5300059980008F5920008759200082592000895
:10D5400085930008D5900008DD99000889920008AD
:10D55000E7900008F59000085D900008C990000869
:10D560001991000821990008C9920008B590000897
:10D570006990000885920008719100080000000081
:10D58000000000000000000001000000000000009A
:10D590000200000000000000030000000000000086
:10D5A0000400000000000000050000000000000072
:10D5B000060000000000000007000000000000005E
:10D5C000080000000000000009000000000000004A
:10D5D00000000000000000000A0000000000000041
:10D5E00014000000000000001E0000000000000009
:10D5F00028000000000000003200000000000000D1
:10D600003C00000000000000460000000000000098
:10D6100050000000000000005A0000000000000060
:10D620000000000000000000640000000000000096
:10D63000C8000000000000002C01000000000000F5
:10D640009001000000000000F40100000000000054
:10D650005802000000000000BC02000000000000B2
:10D660002003000000000000840300000000000010
:10D670000000000000000000E803000000000000BF
:10D68000D007000000000000B80B00000000000000
:10D69000A00F000000000000881300000000000040
:10D6A0007017000000000000581B00000000000080
:10D6B000401F0000000000002823000000000000C0
:10D6C0000000000000000000102700000000000023
:10D6D000204E000000000000307500000000000037
:10D6E000409C00000000000050C30000000000004B
:10D6F00060EA00000000000070110100000000005E
:10D700008038010000000000905F01000000000070
:10D710000000000000000000A086010000000000E2
:10D72000400D030000000000E09304000000000032
:10D73000801A06000000000020A107000000000081
:10D74000C02709000000000060AE0A0000000000D1
:10D7500000350C0000000000A0BB0D000000000020
:10D76000000000000000000040420F000000000028
:10D7700080841E0000000000C0C62D0000000000D4
:10D7800000093D0000000000404B4C00000000007C
:10D79000808D5B0000000000C0CF6A000000000028
:10D7A00000127A00000000004054890000000000D0
:10D7B00000000000000000008096980000000000BB
:10D7C000002D31010000000080C3C90100000000ED
:10D7D000005A62020000000080F0FA02000000001F
:10D7E0000087930300000000801D2C04000000004F
:10D7F00000B4C40400000000804A5D050000000081
:10D80000000000000000000000E1F505000000003D
:10D8100000C2EB0B0000000000A3E11100000000BB
:10D820000084D717000000000065CD1D0000000037
:10D830000046C323000000000027B92900000000B3
:10D840000008AF2F0000000000E9A4350000000030
:10D85000000000000000000000CA9A3B0000000029
:10D860000094357700000000005ED0B20000000098
:10D8700000286BEE0000000000F2052A0100000005
:10D8800000BCA0650100000000863BA10100000073
:10D890000050D6DC01000000001A711802000000E0
:10D8A000627265616B00000000636F6E74696E7573
:10D8B0006500000000000000000000000000000003
:10D8C0000000000001000000020000000300000052
:10D8D000040000007768696C65000069660000005C
:10D8E0000000656C69660000002A2A000000000044
:10D8F00000007E00000000000000002A0000000080
:10D90000000000002F0000000000000000250000C3
:10D910000000000000002F2F000000000000002B7E
:10D9200000000000000000002D00000000000000CA
:10D93000003E3E000000000000003C3C00000000F3
:10D940000000002600000000000000005E00000053
:10D9500000000000007C00000000000000003C000F
:10D96000000000000000003C3D000000000000003E
:10D970003E00000000000000003E3D0000000000EE
:10D980000000213D000000000000003D3D000000BF
:10D9900000000000253D000000000000002F3D00B9
:10D9A0000000000000002F2F3D0000000000002DAF
:10D9B0003D000000000000002B3D000000000000C2
:10D9C000002A3D000000000000002A2A3D0000005F
:10D9D000000000206E6F74200000000020616E6463
:10D9E0002000000000206F7220000000000020696D
:10D9F0006D706F72742000007F707961010000000B
:10DA00000100000000000000000000000000000015
:10DA100000000000000000006D61696E0000000061
:10DA200000000000000000000000000000000000F6
:10DA300000000000600100007400009601000096E4
:10DA40000C00008214000004210000822600000463
:10DA500032000082360000044300008247000004C8
:10DA60005300008257000004640000826900000433
:10DA700075000082790000048F000082930000820C
:10DA80009C001083A7000002AF001083B5000002C5
:10DA9000AF000082C3000081CB000007D0001183DB
:10DAA000D2000102AF000182DA000086E300E60046
:10DAB0000050696B615374644C6962006D61636806
:10DAC000696E65006D616368696E652E54696D6588
:10DAD0000074696D65006D616368696E652E41440F
:10DAE0004300616463006D616368696E652E475031
:10DAF000494F0070696E006D616368696E652E50F4
:10DB0000574D0070776D006D616368696E652E55C5
:10DB10004152540075617274006D616368696E658D
:10DB20002E524742007267620050696B6153746401
:10DB30004C69622E4D656D436865636B6572006D5F
:10DB4000656D007267622E696E6974007267622E7D
:10DB5000656E61626C650068656C6C6F2032007088
:10DB600072696E74006D656D2075736564206D61FA
:10DB7000783A006D656D2E6D6178005472756500A0
:10DB80003200666C6F77696E67007267622E666C32
:10DB90006F77002D3100000000090050696B615063
:10DBA000695A65726F3D3D76312E322E300D0A0076
:10DBB00050696B615374644C69623D3D76312E3817
:10DBC0002E360D0A0050696B6153746444657669A2
:10DBD00063653D3D76312E382E360D0A0070696B37
:10DBE000617363726970742D636F72653D3D763148
:10DBF0002E382E360D0A003D3D3D3D3D3D5B7069A2
:10DC00006B61736372697074207061636B616765C7
:10DC10007320696E7374616C6C65645D3D3D3D3D60
:10DC20003D3D0D0A0025302E3266206B420D0A0064
:10DC30004F766572666C6F774572726F723A2073B9
:10DC40007072696E746620627566662073697A65A3
:10DC5000206F766572666C6F772C20706C656173CF
:10DC60006520757365206269676765722050494B4E
:10DC7000415F535052494E54465F425546465F53AA
:10DC8000495A450D0A004F766572666C6F7745728A
:10DC9000726F723A2070696B6120564D2073746107
:10DCA000636B206F766572666C6F772C20706C6585
:10DCB00061736520757365206269676765722050BE
:10DCC000494B415F535441434B5F425546465F5376
:10DCD000495A450D0A004E616D654572726F723A80
:10DCE000206E616D652027257327206973206E6F74
:10DCF0007420646566696E65640D0A005479706508
:10DD00004572726F723A20257328292074616B6501
:10DD10007320256420706F736974696F6E616C2065
:10DD2000617267756D656E7420627574202564205C
:10DD30007765726520676976656E0D0A0025730D3B
:10DD40000A003020524554200A0030204E454C2015
:10DD5000310A0028290A30204A4D5020310A00306B
:10DD6000204A455A20310A0030204A4D50202D319A
:10DD70000A000A30204A455A20320A003020425216
:10DD80004B0A00302043544E0A00302052415320A9
:10DD900073656C660A0030204F55542073656C66BD
:10DDA0000A0030204E45572073656C660A0030200B
:10DDB00052415320246F726967696E0A002D2D2D20
:10DDC0002D5B636F646520696E20666C6173685DAE
:10DDD0002D2D2D2D2D0D005B696E666F5D3A206235
:10DDE0006F6F742066726F6D206669726D776172F5
:10DDF000652E0D003D3D3D3D3D3D3D3D3D3D3D3DA7
:10DE00003D3D5B50726F6772616D65725D3D3D3D7A
:10DE10003D3D3D3D3D3D3D3D3D3D3D0D002E2E2ECC
:10DE200020003E3E3E20003020474C422000302063
:10DE30004445462000302044454C200030205255B7
:10DE40004E20003020434C5320000A3020455354CC
:10DE500020002E5F5F6E6578745F5F0A30204F553B
:10DE600054200020616E6420006465662000676CA9
:10DE70006F62616C200072657475726E2000206F95
:10DE80007220002061732000636C61737320002096
:10DE90006E6F74200020696D706F72742000250011
:10DEA0006974657228005F5F696E69745F5F282915
:10DEB00000706C6174666F726D5265616428290030
:10DEC000706C6174666F726D5365744D6F64652814
:10DED0002900706C6174666F726D456E61626C656D
:10DEE000282900656E61626C65282900706C617478
:10DEF000666F726D44697361626C6528290064699C
:10DF00007361626C65282900706C6174666F726D54
:10DF10005772697465282900706C6174666F726D40
:10DF200048696768282900706C6174666F726D4774
:10DF300065745469636B282900706C6174666F7234
:10DF40006D526561644279746573282900706C6153
:10DF500074666F726D57726974654279746573285F
:10DF60002900696E6974282900706C6174666F728B
:10DF70006D4C6F77282900706C6174666F726D53F9
:10DF800065744672657175656E6379282900706CD9
:10DF90006174666F726D53657444757479282900D5
:10DFA00073657450696E2870696E3A7374722900D3
:10DFB0005F5F7365745F5F286F626A3A616E792C88
:10DFC0006B65793A616E792C76616C3A616E792C69
:10DFD0006F626A5F7374723A737472290073657446
:10DFE00049642869643A696E742900736C656570C8
:10DFF0005F7328733A696E742900736C6565705F8E
:10E000006D73286D733A696E74290063616C6C5F7F
:10E01000616C776179732866756E5F746F646F3AAF
:10E02000616E7929002A002B002C002D005B65729F
:10E03000726F725D20747970653A20617267206E2C
:10E040006F20666F756E642E005B6572726F725D15
:10E0500020706C6174666F726D206D6574686F649A
:10E06000206E65656420746F206265206F7665722E
:10E07000726964652E005B6572726F725D20504933
:10E080004B415F5354445F4445564943455F554EA9
:10E0900049585F54494D455F454E41424C45206EBD
:10E0A00065656420746F20626520656E61626C65D1
:10E0B0002E005B6572726F725D3A2063616E206E36
:10E0C0006F7420666F756E642050574D20686172C2
:10E0D00064776172652E005B6572726F725D206E8F
:10E0E0006F74206D61746368206770696F20706958
:10E0F0006E2E005B6572726F725D206E6F74206DA4
:10E1000061746368206770696F20706F72742E008D
:10E1100050413130005041300050423000504430C6
:10E1200000504131310050423100504431006131E2
:10E13000003132006132003133003134005041345B
:10E140000031350050413600504137005041380011
:10E15000504139002A3D002B3D002D3D002F3D0050
:10E160003D3D003C636C6173732027666C6F617486
:10E17000273E003C636C6173732027696E74273EF1
:10E1800000504100474C4200504200504300504470
:10E1900000444546005245460042524B0044454C1F
:10E1A000004E454C004E554D004E4F4E0043544ED0
:10E1B0000052554E00494D50004A4D5000535452A4
:10E1C0000052415300434C5300524554004F5054A9
:10E1D00000455354004C5354004F55540042595479
:10E1E000004E4557004A455A005B005D005F5F697D
:10E1F0006E69745F5F007265616444617461007789
:10E2000072697465446174610064617461005F5F88
:10E210006C6962005F5F7368696E620025640070FC
:10E220006C6174666F726D52656164006964006D43
:10E230006574686F64005F5F657272436F64650048
:10E240005F5F66697273745F62797465636F64653A
:10E25000006D6F646500706C6174666F726D456E01
:10E2600061626C65006973456E61626C6500706C1B
:10E270006174666F726D44697361626C6500776882
:10E28000696C65006E616D6500756E69785F7469B3
:10E290006D65006E6F6E6500656C7365006261751B
:10E2A000645261746500666C6F77537461746500C5
:10E2B000636F6E74696E756500256600646566003F
:10E2C00072656600726561644275666600736865B2
:10E2D0006C6C5F6275666600656C6966005F5F62A4
:10E2E0007566005F5F7368627566005F5F73686381
:10E2F000666700737472696E6700617267006368B5
:10E30000006C656E67746800626C6F636B44656572
:10E3100070746800646565707468005F5F69746537
:10E32000725F690054696E794F626A006F626A00B9
:10E33000627265616B007469636B00657869744231
:10E340006C6F636B00626C6F636B00676C6F626114
:10E350006C005B6572726F725D207072696E743AE8
:10E360002063616E206E6F74207072696E74207607
:10E37000616C005F5F76616C005F5F736868646CFE
:10E38000005F5F676C0070756C6C00626F74746F17
:10E390006D006E756D0069734F6E0066756E5F7708
:10E3A00068656E006172675F696E006D61696E001D
:10E3B00070696E0040616E6E6F6E746174696F6E2D
:10E3C0000072657475726E00646F776E0066756EAC
:10E3D0005F746F646F00746F7000757000667265B3
:10E3E00071006465636C65617200666F7200636FD3
:10E3F0006C6F72006F70657261746F72005F636C36
:10E40000737074720063666F726D617428666D74E8
:10E410003A7374722C2A766172292D3E73747200DD
:10E420006368722876616C3A696E74292D3E737444
:10E4300072006865782876616C3A696E74292D3EA1
:10E44000737472002573005F5F72756E4173005FB5
:10E450005F7265730062797465732876616C3A61E6
:10E460006E79292D3E6279746573005F5F63616C1C
:10E470006C7300706572696F645F6D7300636C61CB
:10E480007373006765744475747928292D3E666C32
:10E490006F617400666C6F6174286172673A616EB7
:10E4A00079292D3E666C6F6174006C656674005F3F
:10E4B000726566636E74006765744368616E6E654D
:10E4C0006C28292D3E696E74006C656E2861726738
:10E4D0003A616E79292D3E696E7400696E74286107
:10E4E00072673A616E79292D3E696E7400696428FD
:10E4F0006F626A3A616E79292D3E696E7400696DAA
:10E50000706F7274006C697374006F7574005F5F74
:10E510006B6579005F5F6E6578745F5F28292D3EBB
:10E52000616E79005F5F736C6963655F5F286F621E
:10E530006A3A616E792C73746172743A616E792CE7
:10E54000656E643A616E792C737465703A696E74A5
:10E55000292D3E616E790069746572286172673A8F
:10E56000616E79292D3E616E79005F5F6765745F2A
:10E570005F286F626A3A616E792C6B65793A616ED9
:10E5800079292D3E616E7900647574790000303010
:10E590003031303230333034303530363037303857
:10E5A0003039313031313132313331343135313646
:10E5B000313731383139323032313232323332342C
:10E5C0003235323632373238323933303331333212
:10E5D00033333334333533363337333833393430F8
:10E5E00034313432343334343435343634373438E7
:10E5F00034393530353135323533353435353536D6
:10E6000035373538353936303631363236333634BB
:10E6100036353636363736383639373037313732A1
:10E620003733373437353736373737383739383087
:10E630003831383238333834383538363837383876
:10E640003839393039313932393339343935393665
:10E65000393739383939000078E6000800000020E1
:10E660001800000040C6000890E6000818000020CE
:10E67000601E000050C600080000000000000000FE
:10E680000000000000000000040000000024F4006E
:04000005080000C12E
:00000001FF
